LX51 LINKER/LOCATER V4.66.1.0                                                           03/30/2017  09:01:59  PAGE 1


LX51 LINKER/LOCATER V4.66.1.0, INVOKED BY:
C:\KEIL_V4\C51\BIN\LX51.EXE .\main.obj, .\Interrupt.obj, .\LPF.obj, .\SystemInit.obj, .\TimerInit.obj, .\ADCInit.obj, .\
>> WDTInit.obj, .\GPIOInit.obj, ..\Library\FU68xx_Hardware_Driver\Source\FU68xx_CFG.LIB, ..\Library\FU68xx_Hardware_Driv
>> er\Source\FU68xx_Flash.LIB, ..\Library\FU68xx_Hardware_Driver\Source\FU68xx_OSC.LIB, ..\Library\FU68xx_Hardware_Drive
>> r\Source\FU68xx_Power.LIB TO ADC


CPU MODE:     8051 MODE
MEMORY MODEL: SMALL WITH FLOATING POINT ARITHMETIC


INPUT MODULES INCLUDED:
  .\main.obj (MAIN)
         COMMENT TYPE 0: C51 V9.52.0.0
  .\Interrupt.obj (INTERRUPT)
         COMMENT TYPE 0: C51 V9.52.0.0
  .\LPF.obj (LPF)
         COMMENT TYPE 0: C51 V9.52.0.0
  .\SystemInit.obj (SYSTEMINIT)
         COMMENT TYPE 0: C51 V9.52.0.0
  .\TimerInit.obj (TIMERINIT)
         COMMENT TYPE 0: C51 V9.52.0.0
  .\ADCInit.obj (ADCINIT)
         COMMENT TYPE 0: C51 V9.52.0.0
  .\WDTInit.obj (WDTINIT)
         COMMENT TYPE 0: C51 V9.52.0.0
  .\GPIOInit.obj (GPIOINIT)
         COMMENT TYPE 0: C51 V9.52.0.0
  ..\Library\FU68xx_Hardware_Driver\Source\FU68xx_CFG.LIB (FU68XX_OSC)
         COMMENT TYPE 1: C51 Compiler
  ..\Library\FU68xx_Hardware_Driver\Source\FU68xx_CFG.LIB (FU68XX_POWER)
         COMMENT TYPE 1: C51 Compiler
  C:\KEIL_V4\C51\LIB\C51FPS.LIB (?C?FPDIV)
         COMMENT TYPE 1: A51 / ASM51 Assembler
  C:\KEIL_V4\C51\LIB\C51FPS.LIB (?C?FCAST)
         COMMENT TYPE 1: A51 / ASM51 Assembler
  C:\KEIL_V4\C51\LIB\C51FPS.LIB (?C?FPGETOPN)
         COMMENT TYPE 1: A51 / ASM51 Assembler
  C:\KEIL_V4\C51\LIB\C51S.LIB (?C_STARTUP)
         COMMENT TYPE 1: A51 / ASM51 Assembler
  C:\KEIL_V4\C51\LIB\C51S.LIB (?C?ULDIV)
         COMMENT TYPE 1: A51 / ASM51 Assembler
  C:\KEIL_V4\C51\LIB\C51S.LIB (?C?LNEG)
         COMMENT TYPE 1: A51 / ASM51 Assembler
  C:\KEIL_V4\C51\LIB\C51S.LIB (?C?LSTXDATA)
         COMMENT TYPE 1: A51 / ASM51 Assembler
  C:\KEIL_V4\C51\LIB\C51S.LIB (?C?LSTKXDATA)
         COMMENT TYPE 1: A51 / ASM51 Assembler
  C:\KEIL_V4\C51\LIB\C51S.LIB (?C?LIMUL)
         COMMENT TYPE 1: A51 / ASM51 Assembler
  C:\KEIL_V4\C51\LIB\C51S.LIB (?C_INIT)
         COMMENT TYPE 1: A51 / ASM51 Assembler


ACTIVE MEMORY CLASSES OF MODULE:  ADC (MAIN)

BASE        START       END         USED      MEMORY CLASS
==========================================================
C:000000H   C:000000H   C:00FFFFH   000979H   CODE
I:000000H   I:000000H   I:00007FH   00000EH   DATA
X:000000H   X:000000H   X:00FFFFH   00003CH   XDATA
I:000020H.0 I:000020H.0 I:00002FH.7 000001H.1 BIT
I:000000H   I:000000H   I:0000FFH   000001H   IDATA


MEMORY MAP OF MODULE:  ADC (MAIN)
LX51 LINKER/LOCATER V4.66.1.0                                                         03/30/2017  09:01:59  PAGE 2




START     STOP      LENGTH    ALIGN  RELOC    MEMORY CLASS   SEGMENT NAME
=========================================================================

* * * * * * * * * * *   D A T A   M E M O R Y   * * * * * * * * * * * * *
000000H   000007H   000008H   ---    AT..     DATA           "REG BANK 0"
000008H   00000DH   000006H   BYTE   UNIT     DATA           ?DT?INTERRUPT
00000EH.0 00001FH.7 000012H.0 ---    ---      **GAP**
000020H.0 000020H.1 000000H.2 BIT    UNIT     BIT            ?BI?EXTERNALFASTCLOCKCONFIG?FU68XX_OSC
000020H.2 000020H.3 000000H.2 BIT    UNIT     BIT            _BIT_GROUP_
000020H.4 000020H.4 000000H.1 BIT    UNIT     BIT            ?BI?INTERNALFASTCLOCKCONFIG?FU68XX_OSC
000020H.5 000020H.5 000000H.1 BIT    UNIT     BIT            ?BI?SYSTEMFASTCLOCKMCDCONFIG?FU68XX_OSC
000020H.6 000020H.6 000000H.1 BIT    UNIT     BIT            ?BI?SYSTEMFASTCLOCKSPD2CONFIG?FU68XX_OSC
000020H.7 000020H.7 000000H.1 BIT    UNIT     BIT            ?BI?LVDPOWERDOWNDETECTCONFIG?FU68XX_POWER
000021H.0 000021H.0 000000H.1 BIT    UNIT     BIT            ?BI?LVDPOWERDOWNWARNIECONFIG?FU68XX_POWER
000021H.1 000021H   000000H.7 ---    ---      **GAP**
000022H   000022H   000001H   BYTE   UNIT     IDATA          ?STACK

* * * * * * * * * * *   C O D E   M E M O R Y   * * * * * * * * * * * * *
000000H   000002H   000003H   ---    OFFS..   CODE           ?CO??C_STARTUP?0
000003H   000021H   00001FH   BYTE   UNIT     CODE           ?PR?MAIN?MAIN
000022H   000022H   000001H   ---    ---      **GAP**
000023H   000025H   000003H   BYTE   OFFS..   CODE           ?INTERRUPT?00023
000026H   000032H   00000DH   BYTE   UNIT     CODE           ?C_INITSEG
000033H   000035H   000003H   BYTE   OFFS..   CODE           ?INTERRUPT?00033
000036H   0002A3H   00026EH   BYTE   UNIT     CODE           ?C?LIB_CODE
0002A4H   0003F4H   000151H   BYTE   UNIT     CODE           ?PR?TIM0_INIT?TIMERINIT
0003F5H   0004D5H   0000E1H   BYTE   UNIT     CODE           ?PR?ADC_ISR?INTERRUPT
0004D6H   000563H   00008EH   BYTE   UNIT     CODE           ?PR?ADCDATAINIT?ADCINIT
000564H   0005EFH   00008CH   BYTE   UNIT     CODE           ?C_C51STARTUP
0005F0H   00065CH   00006DH   BYTE   UNIT     CODE           ?PR?ADC_INIT?ADCINIT
00065DH   0006B9H   00005DH   BYTE   UNIT     CODE           ?PR?ADCGETCONVERSIONVALUE?ADCINIT
0006BAH   000711H   000058H   BYTE   UNIT     CODE           ?PR?GPIOINIT?GPIOINIT
000712H   000760H   00004FH   BYTE   UNIT     CODE           ?PR?_WATCHDOGCONFIG?WDTINIT
000761H   0007A5H   000045H   BYTE   UNIT     CODE           ?PR?_VREFCONFIG?FU68XX_POWER
0007A6H   0007E5H   000040H   BYTE   UNIT     CODE           ?PR?_LVRPOWERDOWNRESETCONFIG?FU68XX_POWER
0007E6H   000825H   000040H   BYTE   UNIT     CODE           ?PR?_LVWPOWERDOWNWARNCONFIG?FU68XX_POWER
000826H   000858H   000033H   BYTE   UNIT     CODE           ?PR?EXTERNALFASTCLOCKCONFIG?FU68XX_OSC
000859H   00087CH   000024H   BYTE   UNIT     CODE           ?PR?TIM0_ISR?INTERRUPT
00087DH   00089AH   00001EH   BYTE   UNIT     CODE           ?PR?_LPF?LPF
00089BH   0008B8H   00001EH   BYTE   UNIT     CODE           ?PR?VHALFCONFIG?FU68XX_POWER
0008B9H   0008D3H   00001BH   BYTE   UNIT     CODE           ?PR?INTERNALFASTCLOCKCONFIG?FU68XX_OSC
0008D4H   0008ECH   000019H   BYTE   UNIT     CODE           ?PR?SYSTEMFASTCLOCKMCDCONFIG?FU68XX_OSC
0008EDH   000905H   000019H   BYTE   UNIT     CODE           ?PR?SYSTEMFASTCLOCKSPD2CONFIG?FU68XX_OSC
000906H   00091DH   000018H   BYTE   UNIT     CODE           ?PR?SYSTEMINIT?SYSTEMINIT
00091EH   000933H   000016H   BYTE   UNIT     CODE           ?PR?EXTERNALSLOWCLOCKCONFIG?FU68XX_OSC
000934H   000942H   00000FH   BYTE   UNIT     CODE           ?PR?SYSTEMFASTCLOCKCONFIG?FU68XX_OSC
000943H   000951H   00000FH   BYTE   UNIT     CODE           ?PR?LVDPOWERDOWNDETECTCONFIG?FU68XX_POWER
000952H   000960H   00000FH   BYTE   UNIT     CODE           ?PR?LVDPOWERDOWNWARNIECONFIG?FU68XX_POWER
000961H   00096CH   00000CH   BYTE   UNIT     CODE           ?PR?WDT_INTI?WDTINIT
00096DH   000974H   000008H   BYTE   UNIT     CODE           ?PR?WATCHDOGREFRESH?WDTINIT
000975H   003FFAH   003686H   ---    ---      **GAP**
003FFBH   003FFFH   000005H   BYTE   OFFS..   CODE           ?CO?MAIN?0

* * * * * * * * * * *  X D A T A   M E M O R Y  * * * * * * * * * * * * *
000000H   00003BH   00003CH   BYTE   UNIT     XDATA          ?XD?ADCINIT



OVERLAY MAP OF MODULE:   ADC (MAIN)


FUNCTION/MODULE                             BIT_GROUP   DATA_GROUP 
--> CALLED FUNCTION/MODULE                 START  STOP  START  STOP
LX51 LINKER/LOCATER V4.66.1.0                                                         03/30/2017  09:01:59  PAGE 3


===================================================================
TIM0_ISR/INTERRUPT                         ----- -----  ----- -----

*** NEW ROOT *****************************

ADC_ISR/INTERRUPT                          ----- -----  ----- -----
  +--> _LPF/LPF

_LPF/LPF                                   ----- -----  ----- -----

*** NEW ROOT *****************************

?C_C51STARTUP                              ----- -----  ----- -----
  +--> MAIN/MAIN
  +--> ?C_INITSEG

MAIN/MAIN                                  ----- -----  ----- -----
  +--> SYSTEMINIT/SYSTEMINIT
  +--> TIM0_INIT/TIMERINIT
  +--> ADC_INIT/ADCINIT
  +--> WDT_INTI/WDTINIT
  +--> _WATCHDOGCONFIG/WDTINIT
  +--> ADCGETCONVERSIONVALUE/ADCINIT
  +--> WATCHDOGREFRESH/WDTINIT

SYSTEMINIT/SYSTEMINIT                      ----- -----  ----- -----
  +--> SYSTEMFASTCLOCKCONFIG/FU68XX_OSC
  +--> EXTERNALSLOWCLOCKCONFIG/FU68XX_OSC
  +--> _VREFCONFIG/FU68XX_POWER
  +--> VHALFCONFIG/FU68XX_POWER

SYSTEMFASTCLOCKCONFIG/FU68XX_OSC           20H.2 20H.2  ----- -----

EXTERNALSLOWCLOCKCONFIG/FU68XX_OSC         20H.2 20H.2  ----- -----

_VREFCONFIG/FU68XX_POWER                   20H.2 20H.2  ----- -----

VHALFCONFIG/FU68XX_POWER                   20H.2 20H.3  ----- -----

TIM0_INIT/TIMERINIT                        ----- -----  ----- -----

ADC_INIT/ADCINIT                           ----- -----  ----- -----
  +--> ADCDATAINIT/ADCINIT

ADCDATAINIT/ADCINIT                        ----- -----  ----- -----

WDT_INTI/WDTINIT                           ----- -----  ----- -----

_WATCHDOGCONFIG/WDTINIT                    20H.2 20H.2  ----- -----

ADCGETCONVERSIONVALUE/ADCINIT              ----- -----  ----- -----

WATCHDOGREFRESH/WDTINIT                    ----- -----  ----- -----

?C_INITSEG                                 ----- -----  ----- -----



PUBLIC SYMBOLS OF MODULE:  ADC (MAIN)


      VALUE       CLASS    TYPE      PUBLIC SYMBOL NAME
      =================================================
      00000020H.2 BIT      ---       ?_VREFConfig?BIT
      00000020H.2 BIT      BIT       ?_WatchDogConfig?BIT
LX51 LINKER/LOCATER V4.66.1.0                                                         03/30/2017  09:01:59  PAGE 4


      00000000H   NUMBER   ---       ?C?CODESEG
      010000E0H   CODE     ---       ?C?FCASTC
      010000DBH   CODE     ---       ?C?FCASTI
      010000D6H   CODE     ---       ?C?FCASTL
      01000039H   CODE     ---       ?C?FPDIV
      01000114H   CODE     ---       ?C?FPGETOPN2
      01000149H   CODE     ---       ?C?FPNANRESULT
      01000153H   CODE     ---       ?C?FPOVERFLOW
      0100012BH   CODE     ---       ?C?FPRESULT
      0100013FH   CODE     ---       ?C?FPRESULT2
      01000150H   CODE     ---       ?C?FPUNDERFLOW
      01000277H   CODE     ---       ?C?LIMUL
      0100022CH   CODE     ---       ?C?LNEG
      01000246H   CODE     ---       ?C?LSTKXDATA
      0100023AH   CODE     ---       ?C?LSTXDATA
      0100019AH   CODE     ---       ?C?ULDIV
      00000000H   NUMBER   ---       ?C?XDATASEG
      010005ABH   CODE     ---       ?C_START
      01000000H   CODE     ---       ?C_STARTUP
      00000020H.0 BIT      ---       ?EXTERNALFASTCLOCKCONFIG?BIT
      00000020H.2 BIT      ---       ?ExternalSlowClockConfig?BIT
      00000020H.4 BIT      ---       ?INTERNALFASTCLOCKCONFIG?BIT
      00000020H.7 BIT      ---       ?LVDPOWERDOWNDETECTCONFIG?BIT
      00000021H.0 BIT      ---       ?LVDPOWERDOWNWARNIECONFIG?BIT
      00000020H.2 BIT      ---       ?SystemFastClockConfig?BIT
      00000020H.5 BIT      ---       ?SYSTEMFASTCLOCKMCDCONFIG?BIT
      00000020H.6 BIT      ---       ?SYSTEMFASTCLOCKSPD2CONFIG?BIT
      00000020H.2 BIT      ---       ?VHALFConfig?BIT
      0100087DH   CODE     ---       _LPF
      010007A6H   CODE     ---       _LVRPowerDownResetConfig
      010007E6H   CODE     ---       _LVWPowerDownWarnConfig
      01000761H   CODE     ---       _VREFConfig
      01000712H   CODE     ---       _WatchDogConfig
*SFR* 000000D0H.6 DATA     BIT       AC
*SFR* 000000E0H   DATA     BYTE      ACC
      010005F0H   CODE     ---       ADC_Init
      010003F5H   CODE     ---       ADC_ISR
      02000000H   XDATA    ---       ADCData
      010004D6H   CODE     ---       ADCDataInit
      0100065DH   CODE     ---       ADCGetConversionValue
*SFR* 000000F0H   DATA     BYTE      B
*SFR* 00000086H   DATA     BYTE      CFGKEY
*SFR* 000000D5H   DATA     BYTE      CMP_CR0
*SFR* 000000D6H   DATA     BYTE      CMP_CR1
*SFR* 000000DAH   DATA     BYTE      CMP_CR2
*SFR* 000000D7H   DATA     BYTE      CMP_SR
*SFR* 000000D0H.7 DATA     BIT       CY
*SFR* 00000082H   DATA     WORD      DP
*SFR* 00000083H   DATA     BYTE      DPH
*SFR* 00000082H   DATA     BYTE      DPL
*SFR* 000000F8H   DATA     BYTE      DRV_OUT
*SFR* 000000A8H.7 DATA     BIT       EA
*SFR* 000000A8H.4 DATA     BIT       ES0
*SFR* 000000D9H   DATA     BYTE      EVT_FILT
*SFR* 000000A8H   DATA     BIT       EX0
*SFR* 000000A8H.2 DATA     BIT       EX1
      01000826H   CODE     ---       ExternalFastClockConfig
      0100091EH   CODE     ---       ExternalSlowClockConfig
*SFR* 000000D0H.5 DATA     BIT       F0
*SFR* 000000D0H.1 DATA     BIT       F1
*SFR* 00000084H   DATA     BYTE      FLKEY
*SFR* 000000E8H   DATA     BYTE      FOC_SET0
*SFR* 000000E9H   DATA     BYTE      FOC_SET1
*SFR* 000000E8H.7 DATA     BIT       FOCEN
*SFR* 00000080H   DATA     BIT       GP00
LX51 LINKER/LOCATER V4.66.1.0                                                         03/30/2017  09:01:59  PAGE 5


*SFR* 00000080H.1 DATA     BIT       GP01
*SFR* 00000080H.2 DATA     BIT       GP02
*SFR* 00000080H.3 DATA     BIT       GP03
*SFR* 00000080H.4 DATA     BIT       GP04
*SFR* 00000080H.5 DATA     BIT       GP05
*SFR* 00000080H.6 DATA     BIT       GP06
*SFR* 00000080H.7 DATA     BIT       GP07
*SFR* 00000090H   DATA     BIT       GP10
*SFR* 00000090H.1 DATA     BIT       GP11
*SFR* 00000090H.2 DATA     BIT       GP12
*SFR* 00000090H.3 DATA     BIT       GP13
*SFR* 00000090H.4 DATA     BIT       GP14
*SFR* 00000090H.5 DATA     BIT       GP15
*SFR* 00000090H.6 DATA     BIT       GP16
*SFR* 00000090H.7 DATA     BIT       GP17
*SFR* 000000A0H   DATA     BIT       GP20
*SFR* 000000A0H.1 DATA     BIT       GP21
*SFR* 000000A0H.2 DATA     BIT       GP22
*SFR* 000000A0H.3 DATA     BIT       GP23
*SFR* 000000A0H.4 DATA     BIT       GP24
*SFR* 000000A0H.5 DATA     BIT       GP25
*SFR* 000000A0H.6 DATA     BIT       GP26
*SFR* 000000A0H.7 DATA     BIT       GP27
*SFR* 000000B0H   DATA     BIT       GP30
*SFR* 000000B0H.1 DATA     BIT       GP31
*SFR* 000000B0H.2 DATA     BIT       GP32
*SFR* 000000B0H.3 DATA     BIT       GP33
*SFR* 000000B0H.4 DATA     BIT       GP34
*SFR* 000000B0H.5 DATA     BIT       GP35
*SFR* 000000B0H.6 DATA     BIT       GP36
*SFR* 000000B0H.7 DATA     BIT       GP37
      010006BAH   CODE     ---       GPIOInit
*SFR* 000000A8H   DATA     BYTE      IE
*SFR* 00000088H.2 DATA     BIT       IF0
      010008B9H   CODE     ---       InternalFastClockConfig
*SFR* 000000B8H   DATA     BYTE      IP0
*SFR* 000000C0H   DATA     BYTE      IP1
*SFR* 000000C8H   DATA     BYTE      IP2
*SFR* 000000D8H   DATA     BYTE      IP3
*SFR* 00000088H   DATA     BIT       IT00
*SFR* 00000088H.1 DATA     BIT       IT01
*SFR* 00000088H.3 DATA     BIT       IT10
*SFR* 00000088H.4 DATA     BIT       IT11
*SFR* 000000DCH   DATA     WORD      LPF_K
*SFR* 000000DDH   DATA     BYTE      LPF_KH
*SFR* 000000DCH   DATA     BYTE      LPF_KL
*SFR* 000000DEH   DATA     WORD      LPF_X
*SFR* 000000DFH   DATA     BYTE      LPF_XH
*SFR* 000000DEH   DATA     BYTE      LPF_XL
*SFR* 000000E6H   DATA     WORD      LPF_Y
*SFR* 000000E7H   DATA     BYTE      LPF_YH
*SFR* 000000E6H   DATA     BYTE      LPF_YL
      01000943H   CODE     ---       LVDPowerDownDetectConfig
      01000952H   CODE     ---       LVDPowerDownWarnIEConfig
*SFR* 000000DBH   DATA     BYTE      LVSR
      01000003H   CODE     ---       main
*SFR* 000000A8H.5 DATA     BIT       MCDIE
*SFR* 00000088H.6 DATA     BIT       MCDIF
*SFR* 000000C4H   DATA     BYTE      MD_DA0
*SFR* 000000C5H   DATA     BYTE      MD_DA1
*SFR* 000000C6H   DATA     BYTE      MD_DA2
*SFR* 000000C7H   DATA     BYTE      MD_DA3
*SFR* 000000C6H   DATA     WORD      MD_DAH
*SFR* 000000C4H   DATA     WORD      MD_DAL
*SFR* 000000CCH   DATA     BYTE      MD_DB0
LX51 LINKER/LOCATER V4.66.1.0                                                         03/30/2017  09:01:59  PAGE 6


*SFR* 000000CDH   DATA     BYTE      MD_DB1
*SFR* 000000CEH   DATA     BYTE      MD_DB2
*SFR* 000000CFH   DATA     BYTE      MD_DB3
*SFR* 000000CEH   DATA     WORD      MD_DBH
*SFR* 000000CCH   DATA     WORD      MD_DBL
*SFR* 000000C2H   DATA     WORD      MD_MA
*SFR* 000000C3H   DATA     BYTE      MD_MAH
*SFR* 000000C2H   DATA     BYTE      MD_MAL
*SFR* 000000CAH   DATA     WORD      MD_MB
*SFR* 000000CBH   DATA     BYTE      MD_MBH
*SFR* 000000CAH   DATA     BYTE      MD_MBL
*SFR* 000000C1H   DATA     BYTE      MD_MODE
*SFR* 00000098H.6 DATA     BIT       MOD0
*SFR* 00000098H.7 DATA     BIT       MOD1
*SFR* 000000F8H.7 DATA     BIT       MOE
*SFR* 000000F8H.6 DATA     BIT       OIS4
*SFR* 000000F8H   DATA     BIT       OISUH
*SFR* 000000F8H.1 DATA     BIT       OISUL
*SFR* 000000F8H.2 DATA     BIT       OISVH
*SFR* 000000F8H.3 DATA     BIT       OISVL
*SFR* 000000F8H.4 DATA     BIT       OISWH
*SFR* 000000F8H.5 DATA     BIT       OISWL
*SFR* 000000F1H   DATA     BYTE      OSC_CFG
*SFR* 000000D0H.2 DATA     BIT       OV
*SFR* 000000D0H   DATA     BIT       P
*SFR* 00000080H   DATA     BYTE      P0
*SFR* 000000FCH   DATA     BYTE      P0_OE
*SFR* 00000090H   DATA     BYTE      P1
*SFR* 000000FDH   DATA     BYTE      P1_OE
*SFR* 000000D1H   DATA     BYTE      P1IE
*SFR* 000000D2H   DATA     BYTE      P1IF
*SFR* 000000A0H   DATA     BYTE      P2
*SFR* 000000FEH   DATA     BYTE      P2_OE
*SFR* 000000D3H   DATA     BYTE      P2IE
*SFR* 000000D4H   DATA     BYTE      P2IF
*SFR* 000000B0H   DATA     BYTE      P3
*SFR* 000000FFH   DATA     BYTE      P3_OE
*SFR* 000000C0H.4 DATA     BIT       PADC0
*SFR* 000000C0H.5 DATA     BIT       PADC1
*SFR* 000000C0H.6 DATA     BIT       PCMP0
*SFR* 000000C0H.7 DATA     BIT       PCMP1
*SFR* 00000087H   DATA     BYTE      PCON
*SFR* 000000B8H.6 DATA     BIT       PFOC0
*SFR* 000000B8H.7 DATA     BIT       PFOC1
*SFR* 000000D8H.2 DATA     BIT       PI2C0
*SFR* 000000D8H.3 DATA     BIT       PI2C1
*SFR* 000000EAH   DATA     WORD      PI_EK
*SFR* 000000EBH   DATA     BYTE      PI_EKH
*SFR* 000000EAH   DATA     BYTE      PI_EKL
*SFR* 000000F2H   DATA     WORD      PI_KI
*SFR* 000000F3H   DATA     BYTE      PI_KIH
*SFR* 000000F2H   DATA     BYTE      PI_KIL
*SFR* 000000EEH   DATA     WORD      PI_KP
*SFR* 000000EFH   DATA     BYTE      PI_KPH
*SFR* 000000EEH   DATA     BYTE      PI_KPL
*SFR* 000000ECH   DATA     WORD      PI_UK
*SFR* 000000EDH   DATA     BYTE      PI_UKH
*SFR* 000000ECH   DATA     BYTE      PI_UKL
*SFR* 000000F4H   DATA     WORD      PI_UKMAX
*SFR* 000000F5H   DATA     BYTE      PI_UKMAXH
*SFR* 000000F4H   DATA     BYTE      PI_UKMAXL
*SFR* 000000F6H   DATA     WORD      PI_UKMIN
*SFR* 000000F7H   DATA     BYTE      PI_UKMINH
*SFR* 000000F6H   DATA     BYTE      PI_UKMINL
*SFR* 000000F9H   DATA     BYTE      PL_CR
LX51 LINKER/LOCATER V4.66.1.0                                                         03/30/2017  09:01:59  PAGE 7


*SFR* 000000B8H   DATA     BIT       PLVW0
*SFR* 000000B8H.1 DATA     BIT       PLVW1
*SFR* 000000D8H.6 DATA     BIT       PMCD0
*SFR* 000000D8H.7 DATA     BIT       PMCD1
*SFR* 000000C8H   DATA     BIT       PRTC0
*SFR* 000000C8H.1 DATA     BIT       PRTC1
*SFR* 00000085H   DATA     BYTE      PSCTL
*SFR* 000000D8H.4 DATA     BIT       PSPI0
*SFR* 000000D8H.5 DATA     BIT       PSPI1
*SFR* 000000D0H   DATA     BYTE      PSW
*SFR* 000000C0H   DATA     BIT       PTIM00
*SFR* 000000C0H.1 DATA     BIT       PTIM01
*SFR* 000000C0H.2 DATA     BIT       PTIM10
*SFR* 000000C0H.3 DATA     BIT       PTIM11
*SFR* 000000C8H.2 DATA     BIT       PTIM230
*SFR* 000000C8H.3 DATA     BIT       PTIM231
*SFR* 000000C8H.4 DATA     BIT       PTIM450
*SFR* 000000C8H.5 DATA     BIT       PTIM451
*SFR* 000000C8H.6 DATA     BIT       PTSD0
*SFR* 000000C8H.7 DATA     BIT       PTSD1
*SFR* 000000D8H   DATA     BIT       PUART0
*SFR* 000000D8H.1 DATA     BIT       PUART1
*SFR* 000000B8H.2 DATA     BIT       PX00
*SFR* 000000B8H.3 DATA     BIT       PX01
*SFR* 000000B8H.4 DATA     BIT       PX10
*SFR* 000000B8H.5 DATA     BIT       PX11
*SFR* 00000098H.2 DATA     BIT       RB8
*SFR* 00000098H.4 DATA     BIT       REN
*SFR* 00000098H   DATA     BIT       RI
*SFR* 000000D0H.3 DATA     BIT       RS0
*SFR* 000000D0H.4 DATA     BIT       RS1
*SFR* 000000C9H   DATA     BYTE      RSTSRC
*SFR* 000000A8H.6 DATA     BIT       RTCIE
*SFR* 00000098H.5 DATA     BIT       SM2
*SFR* 00000081H   DATA     BYTE      SP
*SFR* 000000A8H.3 DATA     BIT       SPIIE
*SFR* 000000E4H   DATA     WORD      SV_ANGLE
*SFR* 000000E5H   DATA     BYTE      SV_ANGLEH
*SFR* 000000E4H   DATA     BYTE      SV_ANGLEL
*SFR* 000000E1H   DATA     BYTE      SV_CR
*SFR* 000000E2H   DATA     WORD      SV_US
*SFR* 000000E3H   DATA     BYTE      SV_USH
*SFR* 000000E2H   DATA     BYTE      SV_USL
      01003FFBH   CODE     ---       SysTable
      01000934H   CODE     ---       SystemFastClockConfig
      010008D4H   CODE     ---       SystemFastClockMCDConfig
      010008EDH   CODE     ---       SystemFastClockSPD2Config
      01000906H   CODE     ---       SystemInit
*SFR* 00000098H.3 DATA     BIT       TB8
*SFR* 00000088H   DATA     BYTE      TCON
*SFR* 00000098H.1 DATA     BIT       TI
*SFR* 000000B6H   DATA     WORD      TIM0_CCR1
*SFR* 000000B7H   DATA     BYTE      TIM0_CCR1H
*SFR* 000000B6H   DATA     BYTE      TIM0_CCR1L
*SFR* 000000BAH   DATA     WORD      TIM0_CCR2
*SFR* 000000BBH   DATA     BYTE      TIM0_CCR2H
*SFR* 000000BAH   DATA     BYTE      TIM0_CCR2L
*SFR* 000000BCH   DATA     WORD      TIM0_CCR3
*SFR* 000000BDH   DATA     BYTE      TIM0_CCR3H
*SFR* 000000BCH   DATA     BYTE      TIM0_CCR3L
*SFR* 000000BEH   DATA     WORD      TIM0_CCR4
*SFR* 000000BFH   DATA     BYTE      TIM0_CCR4H
*SFR* 000000BEH   DATA     BYTE      TIM0_CCR4L
*SFR* 000000B9H   DATA     BYTE      TIM0_IER
      010002A4H   CODE     ---       TIM0_Init
LX51 LINKER/LOCATER V4.66.1.0                                                         03/30/2017  09:01:59  PAGE 8


      01000859H   CODE     ---       TIM0_ISR
*SFR* 000000B1H   DATA     BYTE      TIM0_SR1
*SFR* 000000B4H   DATA     WORD      TIM2_ADTR
*SFR* 000000B5H   DATA     BYTE      TIM2_ADTRH
*SFR* 000000B4H   DATA     BYTE      TIM2_ADTRL
*SFR* 000000AEH   DATA     WORD      TIM2_ARR
*SFR* 000000AFH   DATA     BYTE      TIM2_ARRH
*SFR* 000000AEH   DATA     BYTE      TIM2_ARRL
*SFR* 000000B2H   DATA     WORD      TIM2_CMTR
*SFR* 000000B3H   DATA     BYTE      TIM2_CMTRH
*SFR* 000000B2H   DATA     BYTE      TIM2_CMTRL
*SFR* 000000AAH   DATA     WORD      TIM2_CNTR
*SFR* 000000ABH   DATA     BYTE      TIM2_CNTRH
*SFR* 000000AAH   DATA     BYTE      TIM2_CNTRL
*SFR* 000000A1H   DATA     BYTE      TIM2_CR0
*SFR* 000000A9H   DATA     BYTE      TIM2_CR1
*SFR* 000000ACH   DATA     WORD      TIM2_DR
*SFR* 000000ADH   DATA     BYTE      TIM2_DRH
*SFR* 000000ACH   DATA     BYTE      TIM2_DRL
*SFR* 000000A6H   DATA     WORD      TIM3_ARR
*SFR* 000000A7H   DATA     BYTE      TIM3_ARRH
*SFR* 000000A6H   DATA     BYTE      TIM3_ARRL
*SFR* 000000A2H   DATA     WORD      TIM3_CNTR
*SFR* 000000A3H   DATA     BYTE      TIM3_CNTRH
*SFR* 000000A2H   DATA     BYTE      TIM3_CNTRL
*SFR* 0000009CH   DATA     BYTE      TIM3_CR0
*SFR* 0000009DH   DATA     BYTE      TIM3_CR1
*SFR* 000000A4H   DATA     WORD      TIM3_DR
*SFR* 000000A5H   DATA     BYTE      TIM3_DRH
*SFR* 000000A4H   DATA     BYTE      TIM3_DRL
*SFR* 00000096H   DATA     WORD      TIM4_ARR
*SFR* 00000097H   DATA     BYTE      TIM4_ARRH
*SFR* 00000096H   DATA     BYTE      TIM4_ARRL
*SFR* 00000092H   DATA     WORD      TIM4_CNTR
*SFR* 00000093H   DATA     BYTE      TIM4_CNTRH
*SFR* 00000092H   DATA     BYTE      TIM4_CNTRL
*SFR* 0000009EH   DATA     BYTE      TIM4_CR0
*SFR* 0000009FH   DATA     BYTE      TIM4_CR1
*SFR* 00000094H   DATA     WORD      TIM4_DR
*SFR* 00000095H   DATA     BYTE      TIM4_DRH
*SFR* 00000094H   DATA     BYTE      TIM4_DRL
*SFR* 0000008EH   DATA     WORD      TIM5_ARR
*SFR* 0000008FH   DATA     BYTE      TIM5_ARRH
*SFR* 0000008EH   DATA     BYTE      TIM5_ARRL
*SFR* 0000008AH   DATA     WORD      TIM5_CNTR
*SFR* 0000008BH   DATA     BYTE      TIM5_CNTRH
*SFR* 0000008AH   DATA     BYTE      TIM5_CNTRL
*SFR* 00000089H   DATA     BYTE      TIM5_CR0
*SFR* 00000091H   DATA     BYTE      TIM5_CR1
*SFR* 0000008CH   DATA     WORD      TIM5_DR
*SFR* 0000008DH   DATA     BYTE      TIM5_DRH
*SFR* 0000008CH   DATA     BYTE      TIM5_DRL
*SFR* 000000A8H.1 DATA     BIT       TSDIE
*SFR* 00000088H.5 DATA     BIT       TSDIF
*SFR* 0000009AH   DATA     WORD      UT_BAUD
*SFR* 0000009BH   DATA     BYTE      UT_BAUDH
*SFR* 0000009AH   DATA     BYTE      UT_BAUDL
*SFR* 00000098H   DATA     BYTE      UT_CR
*SFR* 00000099H   DATA     BYTE      UT_DR
      0100089BH   CODE     ---       VHALFConfig
      0100096DH   CODE     ---       WatchDogRefresh
      01000961H   CODE     ---       WDT_INTI



LX51 LINKER/LOCATER V4.66.1.0                                                         03/30/2017  09:01:59  PAGE 9


SYMBOL TABLE OF MODULE:  ADC (MAIN)

      VALUE       REP       CLASS    TYPE      SYMBOL NAME
      ====================================================
      ---         MODULE    ---      ---       MAIN
      01003FFBH   PUBLIC    CODE     ---       SysTable
      01000003H   PUBLIC    CODE     ---       main
      000000E2H   SFRSYM    DATA     BYTE      SV_USL
      000000ABH   SFRSYM    DATA     BYTE      TIM2_CNTRH
      000000B0H.4 SFRSYM    DATA     BIT       GP34
      000000A0H.5 SFRSYM    DATA     BIT       GP25
      00000090H.6 SFRSYM    DATA     BIT       GP16
      00000080H.7 SFRSYM    DATA     BIT       GP07
      00000088H.1 SFRSYM    DATA     BIT       IT01
      00000088H.3 SFRSYM    DATA     BIT       IT10
      000000F6H   SFRSYM    DATA     WORD      PI_UKMIN
      000000C2H   SFRSYM    DATA     WORD      MD_MA
      000000A3H   SFRSYM    DATA     BYTE      TIM3_CNTRH
      000000B0H.5 SFRSYM    DATA     BIT       GP35
      000000A0H.6 SFRSYM    DATA     BIT       GP26
      00000090H.7 SFRSYM    DATA     BIT       GP17
      00000080H   SFRSYM    DATA     BYTE      P0
      00000088H.4 SFRSYM    DATA     BIT       IT11
      000000CAH   SFRSYM    DATA     WORD      MD_MB
      00000093H   SFRSYM    DATA     BYTE      TIM4_CNTRH
      000000B0H.6 SFRSYM    DATA     BIT       GP36
      000000A0H.7 SFRSYM    DATA     BIT       GP27
      00000090H   SFRSYM    DATA     BYTE      P1
      000000D9H   SFRSYM    DATA     BYTE      EVT_FILT
      000000F4H   SFRSYM    DATA     WORD      PI_UKMAX
      0000008BH   SFRSYM    DATA     BYTE      TIM5_CNTRH
      000000B2H   SFRSYM    DATA     BYTE      TIM2_CMTRL
      000000B0H.7 SFRSYM    DATA     BIT       GP37
      000000A0H   SFRSYM    DATA     BYTE      P2
      000000AAH   SFRSYM    DATA     BYTE      TIM2_CNTRL
      000000B0H   SFRSYM    DATA     BYTE      P3
      000000A2H   SFRSYM    DATA     BYTE      TIM3_CNTRL
      000000D0H.6 SFRSYM    DATA     BIT       AC
      00000092H   SFRSYM    DATA     BYTE      TIM4_CNTRL
      0000008AH   SFRSYM    DATA     BYTE      TIM5_CNTRL
      000000B6H   SFRSYM    DATA     WORD      TIM0_CCR1
      000000A8H.7 SFRSYM    DATA     BIT       EA
      000000D5H   SFRSYM    DATA     BYTE      CMP_CR0
      000000BAH   SFRSYM    DATA     WORD      TIM0_CCR2
      000000D6H   SFRSYM    DATA     BYTE      CMP_CR1
      000000BCH   SFRSYM    DATA     WORD      TIM0_CCR3
      00000085H   SFRSYM    DATA     BYTE      PSCTL
      000000DAH   SFRSYM    DATA     BYTE      CMP_CR2
      000000BEH   SFRSYM    DATA     WORD      TIM0_CCR4
      000000B8H.2 SFRSYM    DATA     BIT       PX00
      000000EAH   SFRSYM    DATA     WORD      PI_EK
      000000F8H   SFRSYM    DATA     BIT       OISUH
      000000B8H.3 SFRSYM    DATA     BIT       PX01
      000000B8H.4 SFRSYM    DATA     BIT       PX10
      000000F8H.2 SFRSYM    DATA     BIT       OISVH
      000000B8H.5 SFRSYM    DATA     BIT       PX11
      000000F8H.4 SFRSYM    DATA     BIT       OISWH
      000000DCH   SFRSYM    DATA     WORD      LPF_K
      000000F2H   SFRSYM    DATA     WORD      PI_KI
      000000F8H.1 SFRSYM    DATA     BIT       OISUL
      000000A8H   SFRSYM    DATA     BYTE      IE
      000000F8H.3 SFRSYM    DATA     BIT       OISVL
      000000F8H.5 SFRSYM    DATA     BIT       OISWL
      000000D1H   SFRSYM    DATA     BYTE      P1IE
      00000098H.6 SFRSYM    DATA     BIT       MOD0
LX51 LINKER/LOCATER V4.66.1.0                                                         03/30/2017  09:01:59  PAGE 10


      000000D3H   SFRSYM    DATA     BYTE      P2IE
      000000D2H   SFRSYM    DATA     BYTE      P1IF
      000000F9H   SFRSYM    DATA     BYTE      PL_CR
      00000098H.7 SFRSYM    DATA     BIT       MOD1
      000000D4H   SFRSYM    DATA     BYTE      P2IF
      000000ACH   SFRSYM    DATA     WORD      TIM2_DR
      00000082H   SFRSYM    DATA     WORD      DP
      000000EEH   SFRSYM    DATA     WORD      PI_KP
      000000A4H   SFRSYM    DATA     WORD      TIM3_DR
      00000094H   SFRSYM    DATA     WORD      TIM4_DR
      0000008CH   SFRSYM    DATA     WORD      TIM5_DR
      000000F1H   SFRSYM    DATA     BYTE      OSC_CFG
      000000C1H   SFRSYM    DATA     BYTE      MD_MODE
      000000ECH   SFRSYM    DATA     WORD      PI_UK
      000000DEH   SFRSYM    DATA     WORD      LPF_X
      00000098H   SFRSYM    DATA     BIT       RI
      000000E6H   SFRSYM    DATA     WORD      LPF_Y
      000000C0H   SFRSYM    DATA     BIT       PTIM00
      000000D0H.7 SFRSYM    DATA     BIT       CY
      00000098H.1 SFRSYM    DATA     BIT       TI
      000000C0H.1 SFRSYM    DATA     BIT       PTIM01
      000000C0H.2 SFRSYM    DATA     BIT       PTIM10
      000000C0H.3 SFRSYM    DATA     BIT       PTIM11
      000000E1H   SFRSYM    DATA     BYTE      SV_CR
      00000098H   SFRSYM    DATA     BYTE      UT_CR
      00000099H   SFRSYM    DATA     BYTE      UT_DR
      000000F8H.6 SFRSYM    DATA     BIT       OIS4
      00000081H   SFRSYM    DATA     BYTE      SP
      000000D0H.2 SFRSYM    DATA     BIT       OV
      000000C4H   SFRSYM    DATA     BYTE      MD_DA0
      0000009AH   SFRSYM    DATA     WORD      UT_BAUD
      000000CCH   SFRSYM    DATA     BYTE      MD_DB0
      000000C5H   SFRSYM    DATA     BYTE      MD_DA1
      000000CDH   SFRSYM    DATA     BYTE      MD_DB1
      000000C6H   SFRSYM    DATA     BYTE      MD_DA2
      000000CEH   SFRSYM    DATA     BYTE      MD_DB2
      000000C7H   SFRSYM    DATA     BYTE      MD_DA3
      000000B4H   SFRSYM    DATA     WORD      TIM2_ADTR
      000000CFH   SFRSYM    DATA     BYTE      MD_DB3
      000000AFH   SFRSYM    DATA     BYTE      TIM2_ARRH
      000000A7H   SFRSYM    DATA     BYTE      TIM3_ARRH
      00000097H   SFRSYM    DATA     BYTE      TIM4_ARRH
      0000008FH   SFRSYM    DATA     BYTE      TIM5_ARRH
      000000AEH   SFRSYM    DATA     BYTE      TIM2_ARRL
      000000A6H   SFRSYM    DATA     BYTE      TIM3_ARRL
      00000087H   SFRSYM    DATA     BYTE      PCON
      000000E2H   SFRSYM    DATA     WORD      SV_US
      00000096H   SFRSYM    DATA     BYTE      TIM4_ARRL
      0000008EH   SFRSYM    DATA     BYTE      TIM5_ARRL
      000000B2H   SFRSYM    DATA     WORD      TIM2_CMTR
      00000088H   SFRSYM    DATA     BYTE      TCON
      000000AAH   SFRSYM    DATA     WORD      TIM2_CNTR
      000000A2H   SFRSYM    DATA     WORD      TIM3_CNTR
      00000092H   SFRSYM    DATA     WORD      TIM4_CNTR
      0000008AH   SFRSYM    DATA     WORD      TIM5_CNTR
      00000086H   SFRSYM    DATA     BYTE      CFGKEY
      000000E5H   SFRSYM    DATA     BYTE      SV_ANGLEH
      000000D8H   SFRSYM    DATA     BIT       PUART0
      000000E4H   SFRSYM    DATA     BYTE      SV_ANGLEL
      000000C6H   SFRSYM    DATA     WORD      MD_DAH
      000000D8H.1 SFRSYM    DATA     BIT       PUART1
      000000D8H.2 SFRSYM    DATA     BIT       PI2C0
      00000088H.2 SFRSYM    DATA     BIT       IF0
      000000CEH   SFRSYM    DATA     WORD      MD_DBH
      000000D8H.3 SFRSYM    DATA     BIT       PI2C1
LX51 LINKER/LOCATER V4.66.1.0                                                         03/30/2017  09:01:59  PAGE 11


      000000F0H   SFRSYM    DATA     BYTE      B
      000000C4H   SFRSYM    DATA     WORD      MD_DAL
      000000A1H   SFRSYM    DATA     BYTE      TIM2_CR0
      000000CCH   SFRSYM    DATA     WORD      MD_DBL
      0000009CH   SFRSYM    DATA     BYTE      TIM3_CR0
      000000A9H   SFRSYM    DATA     BYTE      TIM2_CR1
      0000009EH   SFRSYM    DATA     BYTE      TIM4_CR0
      0000009DH   SFRSYM    DATA     BYTE      TIM3_CR1
      00000089H   SFRSYM    DATA     BYTE      TIM5_CR0
      0000009FH   SFRSYM    DATA     BYTE      TIM4_CR1
      000000F8H   SFRSYM    DATA     BYTE      DRV_OUT
      00000091H   SFRSYM    DATA     BYTE      TIM5_CR1
      000000E0H   SFRSYM    DATA     BYTE      ACC
      000000F7H   SFRSYM    DATA     BYTE      PI_UKMINH
      000000C3H   SFRSYM    DATA     BYTE      MD_MAH
      000000A8H.4 SFRSYM    DATA     BIT       ES0
      000000DBH   SFRSYM    DATA     BYTE      LVSR
      000000CBH   SFRSYM    DATA     BYTE      MD_MBH
      000000C0H.4 SFRSYM    DATA     BIT       PADC0
      000000B8H   SFRSYM    DATA     BYTE      IP0
      000000F5H   SFRSYM    DATA     BYTE      PI_UKMAXH
      000000C0H.5 SFRSYM    DATA     BIT       PADC1
      000000C0H   SFRSYM    DATA     BYTE      IP1
      000000C8H   SFRSYM    DATA     BYTE      IP2
      000000F6H   SFRSYM    DATA     BYTE      PI_UKMINL
      000000C2H   SFRSYM    DATA     BYTE      MD_MAL
      00000098H.2 SFRSYM    DATA     BIT       RB8
      000000D8H   SFRSYM    DATA     BYTE      IP3
      000000CAH   SFRSYM    DATA     BYTE      MD_MBL
      000000A8H   SFRSYM    DATA     BIT       EX0
      000000F4H   SFRSYM    DATA     BYTE      PI_UKMAXL
      00000098H.3 SFRSYM    DATA     BIT       TB8
      000000B7H   SFRSYM    DATA     BYTE      TIM0_CCR1H
      000000A8H.2 SFRSYM    DATA     BIT       EX1
      000000BBH   SFRSYM    DATA     BYTE      TIM0_CCR2H
      000000D0H   SFRSYM    DATA     BIT       P
      000000BDH   SFRSYM    DATA     BYTE      TIM0_CCR3H
      000000BFH   SFRSYM    DATA     BYTE      TIM0_CCR4H
      000000C8H.2 SFRSYM    DATA     BIT       PTIM230
      000000EBH   SFRSYM    DATA     BYTE      PI_EKH
      00000098H.5 SFRSYM    DATA     BIT       SM2
      000000B6H   SFRSYM    DATA     BYTE      TIM0_CCR1L
      000000B1H   SFRSYM    DATA     BYTE      TIM0_SR1
      000000C8H.3 SFRSYM    DATA     BIT       PTIM231
      000000BAH   SFRSYM    DATA     BYTE      TIM0_CCR2L
      000000BCH   SFRSYM    DATA     BYTE      TIM0_CCR3L
      000000BEH   SFRSYM    DATA     BYTE      TIM0_CCR4L
      000000D8H.6 SFRSYM    DATA     BIT       PMCD0
      000000C8H.4 SFRSYM    DATA     BIT       PTIM450
      000000D0H.3 SFRSYM    DATA     BIT       RS0
      000000DDH   SFRSYM    DATA     BYTE      LPF_KH
      000000F3H   SFRSYM    DATA     BYTE      PI_KIH
      000000EAH   SFRSYM    DATA     BYTE      PI_EKL
      000000E8H   SFRSYM    DATA     BYTE      FOC_SET0
      000000D8H.7 SFRSYM    DATA     BIT       PMCD1
      000000C8H.5 SFRSYM    DATA     BIT       PTIM451
      000000D0H.4 SFRSYM    DATA     BIT       RS1
      000000E9H   SFRSYM    DATA     BYTE      FOC_SET1
      000000B8H.6 SFRSYM    DATA     BIT       PFOC0
      000000DCH   SFRSYM    DATA     BYTE      LPF_KL
      000000F2H   SFRSYM    DATA     BYTE      PI_KIL
      000000B8H.7 SFRSYM    DATA     BIT       PFOC1
      000000ADH   SFRSYM    DATA     BYTE      TIM2_DRH
      000000B9H   SFRSYM    DATA     BYTE      TIM0_IER
      00000083H   SFRSYM    DATA     BYTE      DPH
LX51 LINKER/LOCATER V4.66.1.0                                                         03/30/2017  09:01:59  PAGE 12


      000000EFH   SFRSYM    DATA     BYTE      PI_KPH
      000000A5H   SFRSYM    DATA     BYTE      TIM3_DRH
      00000095H   SFRSYM    DATA     BYTE      TIM4_DRH
      0000008DH   SFRSYM    DATA     BYTE      TIM5_DRH
      000000ACH   SFRSYM    DATA     BYTE      TIM2_DRL
      00000082H   SFRSYM    DATA     BYTE      DPL
      000000EEH   SFRSYM    DATA     BYTE      PI_KPL
      000000A4H   SFRSYM    DATA     BYTE      TIM3_DRL
      000000F8H.7 SFRSYM    DATA     BIT       MOE
      000000C0H.6 SFRSYM    DATA     BIT       PCMP0
      000000EDH   SFRSYM    DATA     BYTE      PI_UKH
      00000094H   SFRSYM    DATA     BYTE      TIM4_DRL
      000000C0H.7 SFRSYM    DATA     BIT       PCMP1
      000000DFH   SFRSYM    DATA     BYTE      LPF_XH
      0000008CH   SFRSYM    DATA     BYTE      TIM5_DRL
      000000AEH   SFRSYM    DATA     WORD      TIM2_ARR
      000000A8H.5 SFRSYM    DATA     BIT       MCDIE
      000000C9H   SFRSYM    DATA     BYTE      RSTSRC
      000000E7H   SFRSYM    DATA     BYTE      LPF_YH
      000000A6H   SFRSYM    DATA     WORD      TIM3_ARR
      00000088H.6 SFRSYM    DATA     BIT       MCDIF
      00000098H.4 SFRSYM    DATA     BIT       REN
      00000096H   SFRSYM    DATA     WORD      TIM4_ARR
      000000ECH   SFRSYM    DATA     BYTE      PI_UKL
      000000D7H   SFRSYM    DATA     BYTE      CMP_SR
      0000008EH   SFRSYM    DATA     WORD      TIM5_ARR
      000000DEH   SFRSYM    DATA     BYTE      LPF_XL
      000000E6H   SFRSYM    DATA     BYTE      LPF_YL
      000000C8H   SFRSYM    DATA     BIT       PRTC0
      000000C8H.1 SFRSYM    DATA     BIT       PRTC1
      000000E8H.7 SFRSYM    DATA     BIT       FOCEN
      000000C8H.6 SFRSYM    DATA     BIT       PTSD0
      000000D8H.4 SFRSYM    DATA     BIT       PSPI0
      000000C8H.7 SFRSYM    DATA     BIT       PTSD1
      000000D8H.5 SFRSYM    DATA     BIT       PSPI1
      0000009BH   SFRSYM    DATA     BYTE      UT_BAUDH
      000000E4H   SFRSYM    DATA     WORD      SV_ANGLE
      000000B5H   SFRSYM    DATA     BYTE      TIM2_ADTRH
      0000009AH   SFRSYM    DATA     BYTE      UT_BAUDL
      000000FCH   SFRSYM    DATA     BYTE      P0_OE
      000000FDH   SFRSYM    DATA     BYTE      P1_OE
      000000D0H.5 SFRSYM    DATA     BIT       F0
      000000B4H   SFRSYM    DATA     BYTE      TIM2_ADTRL
      000000FEH   SFRSYM    DATA     BYTE      P2_OE
      000000D0H.1 SFRSYM    DATA     BIT       F1
      00000080H   SFRSYM    DATA     BIT       GP00
      000000FFH   SFRSYM    DATA     BYTE      P3_OE
      00000090H   SFRSYM    DATA     BIT       GP10
      00000080H.1 SFRSYM    DATA     BIT       GP01
      000000A8H.6 SFRSYM    DATA     BIT       RTCIE
      000000A0H   SFRSYM    DATA     BIT       GP20
      00000090H.1 SFRSYM    DATA     BIT       GP11
      00000080H.2 SFRSYM    DATA     BIT       GP02
      000000E3H   SFRSYM    DATA     BYTE      SV_USH
      000000B0H   SFRSYM    DATA     BIT       GP30
      000000A0H.1 SFRSYM    DATA     BIT       GP21
      00000090H.2 SFRSYM    DATA     BIT       GP12
      00000080H.3 SFRSYM    DATA     BIT       GP03
      000000B8H   SFRSYM    DATA     BIT       PLVW0
      000000A8H.1 SFRSYM    DATA     BIT       TSDIE
      000000D0H   SFRSYM    DATA     BYTE      PSW
      000000B0H.1 SFRSYM    DATA     BIT       GP31
      000000A0H.2 SFRSYM    DATA     BIT       GP22
      00000090H.3 SFRSYM    DATA     BIT       GP13
      00000080H.4 SFRSYM    DATA     BIT       GP04
LX51 LINKER/LOCATER V4.66.1.0                                                         03/30/2017  09:01:59  PAGE 13


      000000B8H.1 SFRSYM    DATA     BIT       PLVW1
      000000A8H.3 SFRSYM    DATA     BIT       SPIIE
      00000088H.5 SFRSYM    DATA     BIT       TSDIF
      000000B0H.2 SFRSYM    DATA     BIT       GP32
      000000A0H.3 SFRSYM    DATA     BIT       GP23
      00000090H.4 SFRSYM    DATA     BIT       GP14
      00000080H.5 SFRSYM    DATA     BIT       GP05
      00000084H   SFRSYM    DATA     BYTE      FLKEY
      000000B3H   SFRSYM    DATA     BYTE      TIM2_CMTRH
      000000B0H.3 SFRSYM    DATA     BIT       GP33
      000000A0H.4 SFRSYM    DATA     BIT       GP24
      00000090H.5 SFRSYM    DATA     BIT       GP15
      00000080H.6 SFRSYM    DATA     BIT       GP06
      00000088H   SFRSYM    DATA     BIT       IT00

      01000003H   BLOCK     CODE     ---       LVL=0
      01000003H   LINE      CODE     ---       #24
      01000003H   LINE      CODE     ---       #25
      01000003H   LINE      CODE     ---       #27
      01000006H   LINE      CODE     ---       #30
      01000009H   LINE      CODE     ---       #33
      0100000CH   LINE      CODE     ---       #36
      0100000FH   LINE      CODE     ---       #43
      01000018H   LINE      CODE     ---       #46
      01000018H   LINE      CODE     ---       #47
      01000018H   LINE      CODE     ---       #50
      0100001BH   LINE      CODE     ---       #52
      0100001DH   LINE      CODE     ---       #54
      01000020H   LINE      CODE     ---       #55
      ---         BLOCKEND  ---      ---       LVL=0

      ---         MODULE    ---      ---       INTERRUPT
      010003F5H   PUBLIC    CODE     ---       ADC_ISR
      01000859H   PUBLIC    CODE     ---       TIM0_ISR
      000000E2H   SFRSYM    DATA     BYTE      SV_USL
      000000ABH   SFRSYM    DATA     BYTE      TIM2_CNTRH
      000000B0H.4 SFRSYM    DATA     BIT       GP34
      000000A0H.5 SFRSYM    DATA     BIT       GP25
      00000090H.6 SFRSYM    DATA     BIT       GP16
      00000080H.7 SFRSYM    DATA     BIT       GP07
      00000088H.1 SFRSYM    DATA     BIT       IT01
      00000088H.3 SFRSYM    DATA     BIT       IT10
      000000F6H   SFRSYM    DATA     WORD      PI_UKMIN
      000000C2H   SFRSYM    DATA     WORD      MD_MA
      000000A3H   SFRSYM    DATA     BYTE      TIM3_CNTRH
      000000B0H.5 SFRSYM    DATA     BIT       GP35
      000000A0H.6 SFRSYM    DATA     BIT       GP26
      00000090H.7 SFRSYM    DATA     BIT       GP17
      00000080H   SFRSYM    DATA     BYTE      P0
      00000088H.4 SFRSYM    DATA     BIT       IT11
      000000CAH   SFRSYM    DATA     WORD      MD_MB
      00000093H   SFRSYM    DATA     BYTE      TIM4_CNTRH
      000000B0H.6 SFRSYM    DATA     BIT       GP36
      000000A0H.7 SFRSYM    DATA     BIT       GP27
      00000090H   SFRSYM    DATA     BYTE      P1
      000000D9H   SFRSYM    DATA     BYTE      EVT_FILT
      000000F4H   SFRSYM    DATA     WORD      PI_UKMAX
      0000008BH   SFRSYM    DATA     BYTE      TIM5_CNTRH
      000000B2H   SFRSYM    DATA     BYTE      TIM2_CMTRL
      000000B0H.7 SFRSYM    DATA     BIT       GP37
      000000A0H   SFRSYM    DATA     BYTE      P2
      000000AAH   SFRSYM    DATA     BYTE      TIM2_CNTRL
      000000B0H   SFRSYM    DATA     BYTE      P3
      000000A2H   SFRSYM    DATA     BYTE      TIM3_CNTRL
      000000D0H.6 SFRSYM    DATA     BIT       AC
LX51 LINKER/LOCATER V4.66.1.0                                                         03/30/2017  09:01:59  PAGE 14


      00000092H   SFRSYM    DATA     BYTE      TIM4_CNTRL
      0000008AH   SFRSYM    DATA     BYTE      TIM5_CNTRL
      000000B6H   SFRSYM    DATA     WORD      TIM0_CCR1
      000000A8H.7 SFRSYM    DATA     BIT       EA
      000000D5H   SFRSYM    DATA     BYTE      CMP_CR0
      000000BAH   SFRSYM    DATA     WORD      TIM0_CCR2
      000000D6H   SFRSYM    DATA     BYTE      CMP_CR1
      000000BCH   SFRSYM    DATA     WORD      TIM0_CCR3
      00000085H   SFRSYM    DATA     BYTE      PSCTL
      000000DAH   SFRSYM    DATA     BYTE      CMP_CR2
      000000BEH   SFRSYM    DATA     WORD      TIM0_CCR4
      000000B8H.2 SFRSYM    DATA     BIT       PX00
      000000EAH   SFRSYM    DATA     WORD      PI_EK
      000000F8H   SFRSYM    DATA     BIT       OISUH
      000000B8H.3 SFRSYM    DATA     BIT       PX01
      000000B8H.4 SFRSYM    DATA     BIT       PX10
      000000F8H.2 SFRSYM    DATA     BIT       OISVH
      000000B8H.5 SFRSYM    DATA     BIT       PX11
      000000F8H.4 SFRSYM    DATA     BIT       OISWH
      000000DCH   SFRSYM    DATA     WORD      LPF_K
      000000F2H   SFRSYM    DATA     WORD      PI_KI
      000000F8H.1 SFRSYM    DATA     BIT       OISUL
      000000A8H   SFRSYM    DATA     BYTE      IE
      000000F8H.3 SFRSYM    DATA     BIT       OISVL
      000000F8H.5 SFRSYM    DATA     BIT       OISWL
      000000D1H   SFRSYM    DATA     BYTE      P1IE
      00000098H.6 SFRSYM    DATA     BIT       MOD0
      000000D3H   SFRSYM    DATA     BYTE      P2IE
      000000D2H   SFRSYM    DATA     BYTE      P1IF
      000000F9H   SFRSYM    DATA     BYTE      PL_CR
      00000098H.7 SFRSYM    DATA     BIT       MOD1
      000000D4H   SFRSYM    DATA     BYTE      P2IF
      000000ACH   SFRSYM    DATA     WORD      TIM2_DR
      00000082H   SFRSYM    DATA     WORD      DP
      000000EEH   SFRSYM    DATA     WORD      PI_KP
      000000A4H   SFRSYM    DATA     WORD      TIM3_DR
      00000094H   SFRSYM    DATA     WORD      TIM4_DR
      0000008CH   SFRSYM    DATA     WORD      TIM5_DR
      000000F1H   SFRSYM    DATA     BYTE      OSC_CFG
      000000C1H   SFRSYM    DATA     BYTE      MD_MODE
      000000ECH   SFRSYM    DATA     WORD      PI_UK
      000000DEH   SFRSYM    DATA     WORD      LPF_X
      00000098H   SFRSYM    DATA     BIT       RI
      000000E6H   SFRSYM    DATA     WORD      LPF_Y
      000000C0H   SFRSYM    DATA     BIT       PTIM00
      000000D0H.7 SFRSYM    DATA     BIT       CY
      00000098H.1 SFRSYM    DATA     BIT       TI
      000000C0H.1 SFRSYM    DATA     BIT       PTIM01
      000000C0H.2 SFRSYM    DATA     BIT       PTIM10
      000000C0H.3 SFRSYM    DATA     BIT       PTIM11
      000000E1H   SFRSYM    DATA     BYTE      SV_CR
      00000098H   SFRSYM    DATA     BYTE      UT_CR
      00000099H   SFRSYM    DATA     BYTE      UT_DR
      000000F8H.6 SFRSYM    DATA     BIT       OIS4
      00000081H   SFRSYM    DATA     BYTE      SP
      000000D0H.2 SFRSYM    DATA     BIT       OV
      000000C4H   SFRSYM    DATA     BYTE      MD_DA0
      0000009AH   SFRSYM    DATA     WORD      UT_BAUD
      000000CCH   SFRSYM    DATA     BYTE      MD_DB0
      000000C5H   SFRSYM    DATA     BYTE      MD_DA1
      000000CDH   SFRSYM    DATA     BYTE      MD_DB1
      000000C6H   SFRSYM    DATA     BYTE      MD_DA2
      000000CEH   SFRSYM    DATA     BYTE      MD_DB2
      000000C7H   SFRSYM    DATA     BYTE      MD_DA3
      000000B4H   SFRSYM    DATA     WORD      TIM2_ADTR
LX51 LINKER/LOCATER V4.66.1.0                                                         03/30/2017  09:01:59  PAGE 15


      000000CFH   SFRSYM    DATA     BYTE      MD_DB3
      000000AFH   SFRSYM    DATA     BYTE      TIM2_ARRH
      000000A7H   SFRSYM    DATA     BYTE      TIM3_ARRH
      00000097H   SFRSYM    DATA     BYTE      TIM4_ARRH
      0000008FH   SFRSYM    DATA     BYTE      TIM5_ARRH
      000000AEH   SFRSYM    DATA     BYTE      TIM2_ARRL
      000000A6H   SFRSYM    DATA     BYTE      TIM3_ARRL
      00000087H   SFRSYM    DATA     BYTE      PCON
      000000E2H   SFRSYM    DATA     WORD      SV_US
      00000096H   SFRSYM    DATA     BYTE      TIM4_ARRL
      0000008EH   SFRSYM    DATA     BYTE      TIM5_ARRL
      000000B2H   SFRSYM    DATA     WORD      TIM2_CMTR
      00000088H   SFRSYM    DATA     BYTE      TCON
      000000AAH   SFRSYM    DATA     WORD      TIM2_CNTR
      000000A2H   SFRSYM    DATA     WORD      TIM3_CNTR
      00000092H   SFRSYM    DATA     WORD      TIM4_CNTR
      0000008AH   SFRSYM    DATA     WORD      TIM5_CNTR
      00000086H   SFRSYM    DATA     BYTE      CFGKEY
      000000E5H   SFRSYM    DATA     BYTE      SV_ANGLEH
      000000D8H   SFRSYM    DATA     BIT       PUART0
      000000E4H   SFRSYM    DATA     BYTE      SV_ANGLEL
      000000C6H   SFRSYM    DATA     WORD      MD_DAH
      000000D8H.1 SFRSYM    DATA     BIT       PUART1
      000000D8H.2 SFRSYM    DATA     BIT       PI2C0
      00000088H.2 SFRSYM    DATA     BIT       IF0
      000000CEH   SFRSYM    DATA     WORD      MD_DBH
      000000D8H.3 SFRSYM    DATA     BIT       PI2C1
      000000F0H   SFRSYM    DATA     BYTE      B
      000000C4H   SFRSYM    DATA     WORD      MD_DAL
      000000A1H   SFRSYM    DATA     BYTE      TIM2_CR0
      000000CCH   SFRSYM    DATA     WORD      MD_DBL
      0000009CH   SFRSYM    DATA     BYTE      TIM3_CR0
      000000A9H   SFRSYM    DATA     BYTE      TIM2_CR1
      0000009EH   SFRSYM    DATA     BYTE      TIM4_CR0
      0000009DH   SFRSYM    DATA     BYTE      TIM3_CR1
      00000089H   SFRSYM    DATA     BYTE      TIM5_CR0
      0000009FH   SFRSYM    DATA     BYTE      TIM4_CR1
      000000F8H   SFRSYM    DATA     BYTE      DRV_OUT
      00000091H   SFRSYM    DATA     BYTE      TIM5_CR1
      000000E0H   SFRSYM    DATA     BYTE      ACC
      000000F7H   SFRSYM    DATA     BYTE      PI_UKMINH
      000000C3H   SFRSYM    DATA     BYTE      MD_MAH
      000000A8H.4 SFRSYM    DATA     BIT       ES0
      000000DBH   SFRSYM    DATA     BYTE      LVSR
      000000CBH   SFRSYM    DATA     BYTE      MD_MBH
      000000C0H.4 SFRSYM    DATA     BIT       PADC0
      000000B8H   SFRSYM    DATA     BYTE      IP0
      000000F5H   SFRSYM    DATA     BYTE      PI_UKMAXH
      000000C0H.5 SFRSYM    DATA     BIT       PADC1
      000000C0H   SFRSYM    DATA     BYTE      IP1
      000000C8H   SFRSYM    DATA     BYTE      IP2
      000000F6H   SFRSYM    DATA     BYTE      PI_UKMINL
      000000C2H   SFRSYM    DATA     BYTE      MD_MAL
      00000098H.2 SFRSYM    DATA     BIT       RB8
      000000D8H   SFRSYM    DATA     BYTE      IP3
      000000CAH   SFRSYM    DATA     BYTE      MD_MBL
      000000A8H   SFRSYM    DATA     BIT       EX0
      000000F4H   SFRSYM    DATA     BYTE      PI_UKMAXL
      00000098H.3 SFRSYM    DATA     BIT       TB8
      000000B7H   SFRSYM    DATA     BYTE      TIM0_CCR1H
      000000A8H.2 SFRSYM    DATA     BIT       EX1
      000000BBH   SFRSYM    DATA     BYTE      TIM0_CCR2H
      000000D0H   SFRSYM    DATA     BIT       P
      000000BDH   SFRSYM    DATA     BYTE      TIM0_CCR3H
      000000BFH   SFRSYM    DATA     BYTE      TIM0_CCR4H
LX51 LINKER/LOCATER V4.66.1.0                                                         03/30/2017  09:01:59  PAGE 16


      000000C8H.2 SFRSYM    DATA     BIT       PTIM230
      000000EBH   SFRSYM    DATA     BYTE      PI_EKH
      00000098H.5 SFRSYM    DATA     BIT       SM2
      000000B6H   SFRSYM    DATA     BYTE      TIM0_CCR1L
      000000B1H   SFRSYM    DATA     BYTE      TIM0_SR1
      000000C8H.3 SFRSYM    DATA     BIT       PTIM231
      000000BAH   SFRSYM    DATA     BYTE      TIM0_CCR2L
      000000BCH   SFRSYM    DATA     BYTE      TIM0_CCR3L
      000000BEH   SFRSYM    DATA     BYTE      TIM0_CCR4L
      000000D8H.6 SFRSYM    DATA     BIT       PMCD0
      000000C8H.4 SFRSYM    DATA     BIT       PTIM450
      000000D0H.3 SFRSYM    DATA     BIT       RS0
      000000DDH   SFRSYM    DATA     BYTE      LPF_KH
      000000F3H   SFRSYM    DATA     BYTE      PI_KIH
      000000EAH   SFRSYM    DATA     BYTE      PI_EKL
      000000E8H   SFRSYM    DATA     BYTE      FOC_SET0
      000000D8H.7 SFRSYM    DATA     BIT       PMCD1
      000000C8H.5 SFRSYM    DATA     BIT       PTIM451
      000000D0H.4 SFRSYM    DATA     BIT       RS1
      000000E9H   SFRSYM    DATA     BYTE      FOC_SET1
      000000B8H.6 SFRSYM    DATA     BIT       PFOC0
      000000DCH   SFRSYM    DATA     BYTE      LPF_KL
      000000F2H   SFRSYM    DATA     BYTE      PI_KIL
      000000B8H.7 SFRSYM    DATA     BIT       PFOC1
      000000ADH   SFRSYM    DATA     BYTE      TIM2_DRH
      000000B9H   SFRSYM    DATA     BYTE      TIM0_IER
      00000083H   SFRSYM    DATA     BYTE      DPH
      000000EFH   SFRSYM    DATA     BYTE      PI_KPH
      000000A5H   SFRSYM    DATA     BYTE      TIM3_DRH
      00000095H   SFRSYM    DATA     BYTE      TIM4_DRH
      0000008DH   SFRSYM    DATA     BYTE      TIM5_DRH
      000000ACH   SFRSYM    DATA     BYTE      TIM2_DRL
      00000082H   SFRSYM    DATA     BYTE      DPL
      000000EEH   SFRSYM    DATA     BYTE      PI_KPL
      000000A4H   SFRSYM    DATA     BYTE      TIM3_DRL
      000000F8H.7 SFRSYM    DATA     BIT       MOE
      000000C0H.6 SFRSYM    DATA     BIT       PCMP0
      000000EDH   SFRSYM    DATA     BYTE      PI_UKH
      00000094H   SFRSYM    DATA     BYTE      TIM4_DRL
      000000C0H.7 SFRSYM    DATA     BIT       PCMP1
      000000DFH   SFRSYM    DATA     BYTE      LPF_XH
      0000008CH   SFRSYM    DATA     BYTE      TIM5_DRL
      000000AEH   SFRSYM    DATA     WORD      TIM2_ARR
      000000A8H.5 SFRSYM    DATA     BIT       MCDIE
      000000C9H   SFRSYM    DATA     BYTE      RSTSRC
      000000E7H   SFRSYM    DATA     BYTE      LPF_YH
      000000A6H   SFRSYM    DATA     WORD      TIM3_ARR
      00000088H.6 SFRSYM    DATA     BIT       MCDIF
      00000098H.4 SFRSYM    DATA     BIT       REN
      00000096H   SFRSYM    DATA     WORD      TIM4_ARR
      000000ECH   SFRSYM    DATA     BYTE      PI_UKL
      000000D7H   SFRSYM    DATA     BYTE      CMP_SR
      0000008EH   SFRSYM    DATA     WORD      TIM5_ARR
      000000DEH   SFRSYM    DATA     BYTE      LPF_XL
      000000E6H   SFRSYM    DATA     BYTE      LPF_YL
      000000C8H   SFRSYM    DATA     BIT       PRTC0
      000000C8H.1 SFRSYM    DATA     BIT       PRTC1
      000000E8H.7 SFRSYM    DATA     BIT       FOCEN
      000000C8H.6 SFRSYM    DATA     BIT       PTSD0
      000000D8H.4 SFRSYM    DATA     BIT       PSPI0
      000000C8H.7 SFRSYM    DATA     BIT       PTSD1
      000000D8H.5 SFRSYM    DATA     BIT       PSPI1
      0000009BH   SFRSYM    DATA     BYTE      UT_BAUDH
      000000E4H   SFRSYM    DATA     WORD      SV_ANGLE
      000000B5H   SFRSYM    DATA     BYTE      TIM2_ADTRH
LX51 LINKER/LOCATER V4.66.1.0                                                         03/30/2017  09:01:59  PAGE 17


      0000009AH   SFRSYM    DATA     BYTE      UT_BAUDL
      000000FCH   SFRSYM    DATA     BYTE      P0_OE
      000000FDH   SFRSYM    DATA     BYTE      P1_OE
      000000D0H.5 SFRSYM    DATA     BIT       F0
      000000B4H   SFRSYM    DATA     BYTE      TIM2_ADTRL
      000000FEH   SFRSYM    DATA     BYTE      P2_OE
      000000D0H.1 SFRSYM    DATA     BIT       F1
      00000080H   SFRSYM    DATA     BIT       GP00
      000000FFH   SFRSYM    DATA     BYTE      P3_OE
      00000090H   SFRSYM    DATA     BIT       GP10
      00000080H.1 SFRSYM    DATA     BIT       GP01
      000000A8H.6 SFRSYM    DATA     BIT       RTCIE
      000000A0H   SFRSYM    DATA     BIT       GP20
      00000090H.1 SFRSYM    DATA     BIT       GP11
      00000080H.2 SFRSYM    DATA     BIT       GP02
      000000E3H   SFRSYM    DATA     BYTE      SV_USH
      000000B0H   SFRSYM    DATA     BIT       GP30
      000000A0H.1 SFRSYM    DATA     BIT       GP21
      00000090H.2 SFRSYM    DATA     BIT       GP12
      00000080H.3 SFRSYM    DATA     BIT       GP03
      000000B8H   SFRSYM    DATA     BIT       PLVW0
      000000A8H.1 SFRSYM    DATA     BIT       TSDIE
      000000D0H   SFRSYM    DATA     BYTE      PSW
      000000B0H.1 SFRSYM    DATA     BIT       GP31
      000000A0H.2 SFRSYM    DATA     BIT       GP22
      00000090H.3 SFRSYM    DATA     BIT       GP13
      00000080H.4 SFRSYM    DATA     BIT       GP04
      000000B8H.1 SFRSYM    DATA     BIT       PLVW1
      000000A8H.3 SFRSYM    DATA     BIT       SPIIE
      00000088H.5 SFRSYM    DATA     BIT       TSDIF
      000000B0H.2 SFRSYM    DATA     BIT       GP32
      000000A0H.3 SFRSYM    DATA     BIT       GP23
      00000090H.4 SFRSYM    DATA     BIT       GP14
      00000080H.5 SFRSYM    DATA     BIT       GP05
      00000084H   SFRSYM    DATA     BYTE      FLKEY
      000000B3H   SFRSYM    DATA     BYTE      TIM2_CMTRH
      000000B0H.3 SFRSYM    DATA     BIT       GP33
      000000A0H.4 SFRSYM    DATA     BIT       GP24
      00000090H.5 SFRSYM    DATA     BIT       GP15
      00000080H.6 SFRSYM    DATA     BIT       GP06
      00000088H   SFRSYM    DATA     BIT       IT00

      01000859H   BLOCK     CODE     ---       LVL=0
      01000859H   LINE      CODE     ---       #25
      0100085FH   LINE      CODE     ---       #27
      01000864H   LINE      CODE     ---       #28
      01000864H   LINE      CODE     ---       #30
      0100086BH   LINE      CODE     ---       #31
      0100086EH   LINE      CODE     ---       #32
      0100086EH   LINE      CODE     ---       #34
      01000873H   LINE      CODE     ---       #35
      01000873H   LINE      CODE     ---       #36
      01000876H   LINE      CODE     ---       #37
      01000876H   LINE      CODE     ---       #39
      ---         BLOCKEND  ---      ---       LVL=0

      010003F5H   BLOCK     CODE     ---       LVL=0
      01000412H   BLOCK     CODE     NEAR LAB  LVL=1
      00000008H   SYMBOL    DATA     WORD      ADCData_VoltageBUS
      0000000AH   SYMBOL    DATA     WORD      ADCData_CurrentBUS
      0000000CH   SYMBOL    DATA     WORD      ADCData_VoltageSREF
      ---         BLOCKEND  ---      ---       LVL=1
      010003F5H   LINE      CODE     ---       #49
      01000412H   LINE      CODE     ---       #55
      0100041CH   LINE      CODE     ---       #56
LX51 LINKER/LOCATER V4.66.1.0                                                         03/30/2017  09:01:59  PAGE 18


      0100041CH   LINE      CODE     ---       #59
      01000430H   LINE      CODE     ---       #60
      01000444H   LINE      CODE     ---       #61
      01000458H   LINE      CODE     ---       #66
      01000473H   LINE      CODE     ---       #67
      0100048EH   LINE      CODE     ---       #68
      010004A9H   LINE      CODE     ---       #70
      010004B0H   LINE      CODE     ---       #71
      010004B0H   LINE      CODE     ---       #74
      010004B7H   LINE      CODE     ---       #75
      010004B7H   LINE      CODE     ---       #76
      010004BBH   LINE      CODE     ---       #77
      010004BBH   LINE      CODE     ---       #78
      ---         BLOCKEND  ---      ---       LVL=0

      ---         MODULE    ---      ---       LPF
      0100087DH   PUBLIC    CODE     ---       _LPF
      000000E2H   SFRSYM    DATA     BYTE      SV_USL
      000000ABH   SFRSYM    DATA     BYTE      TIM2_CNTRH
      000000B0H.4 SFRSYM    DATA     BIT       GP34
      000000A0H.5 SFRSYM    DATA     BIT       GP25
      00000090H.6 SFRSYM    DATA     BIT       GP16
      00000080H.7 SFRSYM    DATA     BIT       GP07
      00000088H.1 SFRSYM    DATA     BIT       IT01
      00000088H.3 SFRSYM    DATA     BIT       IT10
      000000F6H   SFRSYM    DATA     WORD      PI_UKMIN
      000000C2H   SFRSYM    DATA     WORD      MD_MA
      000000A3H   SFRSYM    DATA     BYTE      TIM3_CNTRH
      000000B0H.5 SFRSYM    DATA     BIT       GP35
      000000A0H.6 SFRSYM    DATA     BIT       GP26
      00000090H.7 SFRSYM    DATA     BIT       GP17
      00000080H   SFRSYM    DATA     BYTE      P0
      00000088H.4 SFRSYM    DATA     BIT       IT11
      000000CAH   SFRSYM    DATA     WORD      MD_MB
      00000093H   SFRSYM    DATA     BYTE      TIM4_CNTRH
      000000B0H.6 SFRSYM    DATA     BIT       GP36
      000000A0H.7 SFRSYM    DATA     BIT       GP27
      00000090H   SFRSYM    DATA     BYTE      P1
      000000D9H   SFRSYM    DATA     BYTE      EVT_FILT
      000000F4H   SFRSYM    DATA     WORD      PI_UKMAX
      0000008BH   SFRSYM    DATA     BYTE      TIM5_CNTRH
      000000B2H   SFRSYM    DATA     BYTE      TIM2_CMTRL
      000000B0H.7 SFRSYM    DATA     BIT       GP37
      000000A0H   SFRSYM    DATA     BYTE      P2
      000000AAH   SFRSYM    DATA     BYTE      TIM2_CNTRL
      000000B0H   SFRSYM    DATA     BYTE      P3
      000000A2H   SFRSYM    DATA     BYTE      TIM3_CNTRL
      000000D0H.6 SFRSYM    DATA     BIT       AC
      00000092H   SFRSYM    DATA     BYTE      TIM4_CNTRL
      0000008AH   SFRSYM    DATA     BYTE      TIM5_CNTRL
      000000B6H   SFRSYM    DATA     WORD      TIM0_CCR1
      000000A8H.7 SFRSYM    DATA     BIT       EA
      000000D5H   SFRSYM    DATA     BYTE      CMP_CR0
      000000BAH   SFRSYM    DATA     WORD      TIM0_CCR2
      000000D6H   SFRSYM    DATA     BYTE      CMP_CR1
      000000BCH   SFRSYM    DATA     WORD      TIM0_CCR3
      00000085H   SFRSYM    DATA     BYTE      PSCTL
      000000DAH   SFRSYM    DATA     BYTE      CMP_CR2
      000000BEH   SFRSYM    DATA     WORD      TIM0_CCR4
      000000B8H.2 SFRSYM    DATA     BIT       PX00
      000000EAH   SFRSYM    DATA     WORD      PI_EK
      000000F8H   SFRSYM    DATA     BIT       OISUH
      000000B8H.3 SFRSYM    DATA     BIT       PX01
      000000B8H.4 SFRSYM    DATA     BIT       PX10
      000000F8H.2 SFRSYM    DATA     BIT       OISVH
LX51 LINKER/LOCATER V4.66.1.0                                                         03/30/2017  09:01:59  PAGE 19


      000000B8H.5 SFRSYM    DATA     BIT       PX11
      000000F8H.4 SFRSYM    DATA     BIT       OISWH
      000000DCH   SFRSYM    DATA     WORD      LPF_K
      000000F2H   SFRSYM    DATA     WORD      PI_KI
      000000F8H.1 SFRSYM    DATA     BIT       OISUL
      000000A8H   SFRSYM    DATA     BYTE      IE
      000000F8H.3 SFRSYM    DATA     BIT       OISVL
      000000F8H.5 SFRSYM    DATA     BIT       OISWL
      000000D1H   SFRSYM    DATA     BYTE      P1IE
      00000098H.6 SFRSYM    DATA     BIT       MOD0
      000000D3H   SFRSYM    DATA     BYTE      P2IE
      000000D2H   SFRSYM    DATA     BYTE      P1IF
      000000F9H   SFRSYM    DATA     BYTE      PL_CR
      00000098H.7 SFRSYM    DATA     BIT       MOD1
      000000D4H   SFRSYM    DATA     BYTE      P2IF
      000000ACH   SFRSYM    DATA     WORD      TIM2_DR
      00000082H   SFRSYM    DATA     WORD      DP
      000000EEH   SFRSYM    DATA     WORD      PI_KP
      000000A4H   SFRSYM    DATA     WORD      TIM3_DR
      00000094H   SFRSYM    DATA     WORD      TIM4_DR
      0000008CH   SFRSYM    DATA     WORD      TIM5_DR
      000000F1H   SFRSYM    DATA     BYTE      OSC_CFG
      000000C1H   SFRSYM    DATA     BYTE      MD_MODE
      000000ECH   SFRSYM    DATA     WORD      PI_UK
      000000DEH   SFRSYM    DATA     WORD      LPF_X
      00000098H   SFRSYM    DATA     BIT       RI
      000000E6H   SFRSYM    DATA     WORD      LPF_Y
      000000C0H   SFRSYM    DATA     BIT       PTIM00
      000000D0H.7 SFRSYM    DATA     BIT       CY
      00000098H.1 SFRSYM    DATA     BIT       TI
      000000C0H.1 SFRSYM    DATA     BIT       PTIM01
      000000C0H.2 SFRSYM    DATA     BIT       PTIM10
      000000C0H.3 SFRSYM    DATA     BIT       PTIM11
      000000E1H   SFRSYM    DATA     BYTE      SV_CR
      00000098H   SFRSYM    DATA     BYTE      UT_CR
      00000099H   SFRSYM    DATA     BYTE      UT_DR
      000000F8H.6 SFRSYM    DATA     BIT       OIS4
      00000081H   SFRSYM    DATA     BYTE      SP
      000000D0H.2 SFRSYM    DATA     BIT       OV
      000000C4H   SFRSYM    DATA     BYTE      MD_DA0
      0000009AH   SFRSYM    DATA     WORD      UT_BAUD
      000000CCH   SFRSYM    DATA     BYTE      MD_DB0
      000000C5H   SFRSYM    DATA     BYTE      MD_DA1
      000000CDH   SFRSYM    DATA     BYTE      MD_DB1
      000000C6H   SFRSYM    DATA     BYTE      MD_DA2
      000000CEH   SFRSYM    DATA     BYTE      MD_DB2
      000000C7H   SFRSYM    DATA     BYTE      MD_DA3
      000000B4H   SFRSYM    DATA     WORD      TIM2_ADTR
      000000CFH   SFRSYM    DATA     BYTE      MD_DB3
      000000AFH   SFRSYM    DATA     BYTE      TIM2_ARRH
      000000A7H   SFRSYM    DATA     BYTE      TIM3_ARRH
      00000097H   SFRSYM    DATA     BYTE      TIM4_ARRH
      0000008FH   SFRSYM    DATA     BYTE      TIM5_ARRH
      000000AEH   SFRSYM    DATA     BYTE      TIM2_ARRL
      000000A6H   SFRSYM    DATA     BYTE      TIM3_ARRL
      00000087H   SFRSYM    DATA     BYTE      PCON
      000000E2H   SFRSYM    DATA     WORD      SV_US
      00000096H   SFRSYM    DATA     BYTE      TIM4_ARRL
      0000008EH   SFRSYM    DATA     BYTE      TIM5_ARRL
      000000B2H   SFRSYM    DATA     WORD      TIM2_CMTR
      00000088H   SFRSYM    DATA     BYTE      TCON
      000000AAH   SFRSYM    DATA     WORD      TIM2_CNTR
      000000A2H   SFRSYM    DATA     WORD      TIM3_CNTR
      00000092H   SFRSYM    DATA     WORD      TIM4_CNTR
      0000008AH   SFRSYM    DATA     WORD      TIM5_CNTR
LX51 LINKER/LOCATER V4.66.1.0                                                         03/30/2017  09:01:59  PAGE 20


      00000086H   SFRSYM    DATA     BYTE      CFGKEY
      000000E5H   SFRSYM    DATA     BYTE      SV_ANGLEH
      000000D8H   SFRSYM    DATA     BIT       PUART0
      000000E4H   SFRSYM    DATA     BYTE      SV_ANGLEL
      000000C6H   SFRSYM    DATA     WORD      MD_DAH
      000000D8H.1 SFRSYM    DATA     BIT       PUART1
      000000D8H.2 SFRSYM    DATA     BIT       PI2C0
      00000088H.2 SFRSYM    DATA     BIT       IF0
      000000CEH   SFRSYM    DATA     WORD      MD_DBH
      000000D8H.3 SFRSYM    DATA     BIT       PI2C1
      000000F0H   SFRSYM    DATA     BYTE      B
      000000C4H   SFRSYM    DATA     WORD      MD_DAL
      000000A1H   SFRSYM    DATA     BYTE      TIM2_CR0
      000000CCH   SFRSYM    DATA     WORD      MD_DBL
      0000009CH   SFRSYM    DATA     BYTE      TIM3_CR0
      000000A9H   SFRSYM    DATA     BYTE      TIM2_CR1
      0000009EH   SFRSYM    DATA     BYTE      TIM4_CR0
      0000009DH   SFRSYM    DATA     BYTE      TIM3_CR1
      00000089H   SFRSYM    DATA     BYTE      TIM5_CR0
      0000009FH   SFRSYM    DATA     BYTE      TIM4_CR1
      000000F8H   SFRSYM    DATA     BYTE      DRV_OUT
      00000091H   SFRSYM    DATA     BYTE      TIM5_CR1
      000000E0H   SFRSYM    DATA     BYTE      ACC
      000000F7H   SFRSYM    DATA     BYTE      PI_UKMINH
      000000C3H   SFRSYM    DATA     BYTE      MD_MAH
      000000A8H.4 SFRSYM    DATA     BIT       ES0
      000000DBH   SFRSYM    DATA     BYTE      LVSR
      000000CBH   SFRSYM    DATA     BYTE      MD_MBH
      000000C0H.4 SFRSYM    DATA     BIT       PADC0
      000000B8H   SFRSYM    DATA     BYTE      IP0
      000000F5H   SFRSYM    DATA     BYTE      PI_UKMAXH
      000000C0H.5 SFRSYM    DATA     BIT       PADC1
      000000C0H   SFRSYM    DATA     BYTE      IP1
      000000C8H   SFRSYM    DATA     BYTE      IP2
      000000F6H   SFRSYM    DATA     BYTE      PI_UKMINL
      000000C2H   SFRSYM    DATA     BYTE      MD_MAL
      00000098H.2 SFRSYM    DATA     BIT       RB8
      000000D8H   SFRSYM    DATA     BYTE      IP3
      000000CAH   SFRSYM    DATA     BYTE      MD_MBL
      000000A8H   SFRSYM    DATA     BIT       EX0
      000000F4H   SFRSYM    DATA     BYTE      PI_UKMAXL
      00000098H.3 SFRSYM    DATA     BIT       TB8
      000000B7H   SFRSYM    DATA     BYTE      TIM0_CCR1H
      000000A8H.2 SFRSYM    DATA     BIT       EX1
      000000BBH   SFRSYM    DATA     BYTE      TIM0_CCR2H
      000000D0H   SFRSYM    DATA     BIT       P
      000000BDH   SFRSYM    DATA     BYTE      TIM0_CCR3H
      000000BFH   SFRSYM    DATA     BYTE      TIM0_CCR4H
      000000C8H.2 SFRSYM    DATA     BIT       PTIM230
      000000EBH   SFRSYM    DATA     BYTE      PI_EKH
      00000098H.5 SFRSYM    DATA     BIT       SM2
      000000B6H   SFRSYM    DATA     BYTE      TIM0_CCR1L
      000000B1H   SFRSYM    DATA     BYTE      TIM0_SR1
      000000C8H.3 SFRSYM    DATA     BIT       PTIM231
      000000BAH   SFRSYM    DATA     BYTE      TIM0_CCR2L
      000000BCH   SFRSYM    DATA     BYTE      TIM0_CCR3L
      000000BEH   SFRSYM    DATA     BYTE      TIM0_CCR4L
      000000D8H.6 SFRSYM    DATA     BIT       PMCD0
      000000C8H.4 SFRSYM    DATA     BIT       PTIM450
      000000D0H.3 SFRSYM    DATA     BIT       RS0
      000000DDH   SFRSYM    DATA     BYTE      LPF_KH
      000000F3H   SFRSYM    DATA     BYTE      PI_KIH
      000000EAH   SFRSYM    DATA     BYTE      PI_EKL
      000000E8H   SFRSYM    DATA     BYTE      FOC_SET0
      000000D8H.7 SFRSYM    DATA     BIT       PMCD1
LX51 LINKER/LOCATER V4.66.1.0                                                         03/30/2017  09:01:59  PAGE 21


      000000C8H.5 SFRSYM    DATA     BIT       PTIM451
      000000D0H.4 SFRSYM    DATA     BIT       RS1
      000000E9H   SFRSYM    DATA     BYTE      FOC_SET1
      000000B8H.6 SFRSYM    DATA     BIT       PFOC0
      000000DCH   SFRSYM    DATA     BYTE      LPF_KL
      000000F2H   SFRSYM    DATA     BYTE      PI_KIL
      000000B8H.7 SFRSYM    DATA     BIT       PFOC1
      000000ADH   SFRSYM    DATA     BYTE      TIM2_DRH
      000000B9H   SFRSYM    DATA     BYTE      TIM0_IER
      00000083H   SFRSYM    DATA     BYTE      DPH
      000000EFH   SFRSYM    DATA     BYTE      PI_KPH
      000000A5H   SFRSYM    DATA     BYTE      TIM3_DRH
      00000095H   SFRSYM    DATA     BYTE      TIM4_DRH
      0000008DH   SFRSYM    DATA     BYTE      TIM5_DRH
      000000ACH   SFRSYM    DATA     BYTE      TIM2_DRL
      00000082H   SFRSYM    DATA     BYTE      DPL
      000000EEH   SFRSYM    DATA     BYTE      PI_KPL
      000000A4H   SFRSYM    DATA     BYTE      TIM3_DRL
      000000F8H.7 SFRSYM    DATA     BIT       MOE
      000000C0H.6 SFRSYM    DATA     BIT       PCMP0
      000000EDH   SFRSYM    DATA     BYTE      PI_UKH
      00000094H   SFRSYM    DATA     BYTE      TIM4_DRL
      000000C0H.7 SFRSYM    DATA     BIT       PCMP1
      000000DFH   SFRSYM    DATA     BYTE      LPF_XH
      0000008CH   SFRSYM    DATA     BYTE      TIM5_DRL
      000000AEH   SFRSYM    DATA     WORD      TIM2_ARR
      000000A8H.5 SFRSYM    DATA     BIT       MCDIE
      000000C9H   SFRSYM    DATA     BYTE      RSTSRC
      000000E7H   SFRSYM    DATA     BYTE      LPF_YH
      000000A6H   SFRSYM    DATA     WORD      TIM3_ARR
      00000088H.6 SFRSYM    DATA     BIT       MCDIF
      00000098H.4 SFRSYM    DATA     BIT       REN
      00000096H   SFRSYM    DATA     WORD      TIM4_ARR
      000000ECH   SFRSYM    DATA     BYTE      PI_UKL
      000000D7H   SFRSYM    DATA     BYTE      CMP_SR
      0000008EH   SFRSYM    DATA     WORD      TIM5_ARR
      000000DEH   SFRSYM    DATA     BYTE      LPF_XL
      000000E6H   SFRSYM    DATA     BYTE      LPF_YL
      000000C8H   SFRSYM    DATA     BIT       PRTC0
      000000C8H.1 SFRSYM    DATA     BIT       PRTC1
      000000E8H.7 SFRSYM    DATA     BIT       FOCEN
      000000C8H.6 SFRSYM    DATA     BIT       PTSD0
      000000D8H.4 SFRSYM    DATA     BIT       PSPI0
      000000C8H.7 SFRSYM    DATA     BIT       PTSD1
      000000D8H.5 SFRSYM    DATA     BIT       PSPI1
      0000009BH   SFRSYM    DATA     BYTE      UT_BAUDH
      000000E4H   SFRSYM    DATA     WORD      SV_ANGLE
      000000B5H   SFRSYM    DATA     BYTE      TIM2_ADTRH
      0000009AH   SFRSYM    DATA     BYTE      UT_BAUDL
      000000FCH   SFRSYM    DATA     BYTE      P0_OE
      000000FDH   SFRSYM    DATA     BYTE      P1_OE
      000000D0H.5 SFRSYM    DATA     BIT       F0
      000000B4H   SFRSYM    DATA     BYTE      TIM2_ADTRL
      000000FEH   SFRSYM    DATA     BYTE      P2_OE
      000000D0H.1 SFRSYM    DATA     BIT       F1
      00000080H   SFRSYM    DATA     BIT       GP00
      000000FFH   SFRSYM    DATA     BYTE      P3_OE
      00000090H   SFRSYM    DATA     BIT       GP10
      00000080H.1 SFRSYM    DATA     BIT       GP01
      000000A8H.6 SFRSYM    DATA     BIT       RTCIE
      000000A0H   SFRSYM    DATA     BIT       GP20
      00000090H.1 SFRSYM    DATA     BIT       GP11
      00000080H.2 SFRSYM    DATA     BIT       GP02
      000000E3H   SFRSYM    DATA     BYTE      SV_USH
      000000B0H   SFRSYM    DATA     BIT       GP30
LX51 LINKER/LOCATER V4.66.1.0                                                         03/30/2017  09:01:59  PAGE 22


      000000A0H.1 SFRSYM    DATA     BIT       GP21
      00000090H.2 SFRSYM    DATA     BIT       GP12
      00000080H.3 SFRSYM    DATA     BIT       GP03
      000000B8H   SFRSYM    DATA     BIT       PLVW0
      000000A8H.1 SFRSYM    DATA     BIT       TSDIE
      000000D0H   SFRSYM    DATA     BYTE      PSW
      000000B0H.1 SFRSYM    DATA     BIT       GP31
      000000A0H.2 SFRSYM    DATA     BIT       GP22
      00000090H.3 SFRSYM    DATA     BIT       GP13
      00000080H.4 SFRSYM    DATA     BIT       GP04
      000000B8H.1 SFRSYM    DATA     BIT       PLVW1
      000000A8H.3 SFRSYM    DATA     BIT       SPIIE
      00000088H.5 SFRSYM    DATA     BIT       TSDIF
      000000B0H.2 SFRSYM    DATA     BIT       GP32
      000000A0H.3 SFRSYM    DATA     BIT       GP23
      00000090H.4 SFRSYM    DATA     BIT       GP14
      00000080H.5 SFRSYM    DATA     BIT       GP05
      00000084H   SFRSYM    DATA     BYTE      FLKEY
      000000B3H   SFRSYM    DATA     BYTE      TIM2_CMTRH
      000000B0H.3 SFRSYM    DATA     BIT       GP33
      000000A0H.4 SFRSYM    DATA     BIT       GP24
      00000090H.5 SFRSYM    DATA     BIT       GP15
      00000080H.6 SFRSYM    DATA     BIT       GP06
      00000088H   SFRSYM    DATA     BIT       IT00

      0100087DH   BLOCK     CODE     ---       LVL=0
      00000006H   SYMBOL    DATA     WORD      Xn1
      00000004H   SYMBOL    DATA     WORD      Xn0
      00000002H   SYMBOL    DATA     WORD      K
      0100087DH   LINE      CODE     ---       #26
      0100087DH   LINE      CODE     ---       #27
      0100087DH   LINE      CODE     ---       #28
      01000881H   LINE      CODE     ---       #29
      01000885H   LINE      CODE     ---       #30
      01000889H   LINE      CODE     ---       #31
      0100088CH   LINE      CODE     ---       #32
      01000891H   LINE      CODE     ---       #33
      01000896H   LINE      CODE     ---       #34
      0100089AH   LINE      CODE     ---       #35
      ---         BLOCKEND  ---      ---       LVL=0

      ---         MODULE    ---      ---       SYSTEMINIT
      01000906H   PUBLIC    CODE     ---       SystemInit
      000000E2H   SFRSYM    DATA     BYTE      SV_USL
      000000ABH   SFRSYM    DATA     BYTE      TIM2_CNTRH
      000000B0H.4 SFRSYM    DATA     BIT       GP34
      000000A0H.5 SFRSYM    DATA     BIT       GP25
      00000090H.6 SFRSYM    DATA     BIT       GP16
      00000080H.7 SFRSYM    DATA     BIT       GP07
      00000088H.1 SFRSYM    DATA     BIT       IT01
      00000088H.3 SFRSYM    DATA     BIT       IT10
      000000F6H   SFRSYM    DATA     WORD      PI_UKMIN
      000000C2H   SFRSYM    DATA     WORD      MD_MA
      000000A3H   SFRSYM    DATA     BYTE      TIM3_CNTRH
      000000B0H.5 SFRSYM    DATA     BIT       GP35
      000000A0H.6 SFRSYM    DATA     BIT       GP26
      00000090H.7 SFRSYM    DATA     BIT       GP17
      00000080H   SFRSYM    DATA     BYTE      P0
      00000088H.4 SFRSYM    DATA     BIT       IT11
      000000CAH   SFRSYM    DATA     WORD      MD_MB
      00000093H   SFRSYM    DATA     BYTE      TIM4_CNTRH
      000000B0H.6 SFRSYM    DATA     BIT       GP36
      000000A0H.7 SFRSYM    DATA     BIT       GP27
      00000090H   SFRSYM    DATA     BYTE      P1
      000000D9H   SFRSYM    DATA     BYTE      EVT_FILT
LX51 LINKER/LOCATER V4.66.1.0                                                         03/30/2017  09:01:59  PAGE 23


      000000F4H   SFRSYM    DATA     WORD      PI_UKMAX
      0000008BH   SFRSYM    DATA     BYTE      TIM5_CNTRH
      000000B2H   SFRSYM    DATA     BYTE      TIM2_CMTRL
      000000B0H.7 SFRSYM    DATA     BIT       GP37
      000000A0H   SFRSYM    DATA     BYTE      P2
      000000AAH   SFRSYM    DATA     BYTE      TIM2_CNTRL
      000000B0H   SFRSYM    DATA     BYTE      P3
      000000A2H   SFRSYM    DATA     BYTE      TIM3_CNTRL
      000000D0H.6 SFRSYM    DATA     BIT       AC
      00000092H   SFRSYM    DATA     BYTE      TIM4_CNTRL
      0000008AH   SFRSYM    DATA     BYTE      TIM5_CNTRL
      000000B6H   SFRSYM    DATA     WORD      TIM0_CCR1
      000000A8H.7 SFRSYM    DATA     BIT       EA
      000000D5H   SFRSYM    DATA     BYTE      CMP_CR0
      000000BAH   SFRSYM    DATA     WORD      TIM0_CCR2
      000000D6H   SFRSYM    DATA     BYTE      CMP_CR1
      000000BCH   SFRSYM    DATA     WORD      TIM0_CCR3
      00000085H   SFRSYM    DATA     BYTE      PSCTL
      000000DAH   SFRSYM    DATA     BYTE      CMP_CR2
      000000BEH   SFRSYM    DATA     WORD      TIM0_CCR4
      000000B8H.2 SFRSYM    DATA     BIT       PX00
      000000EAH   SFRSYM    DATA     WORD      PI_EK
      000000F8H   SFRSYM    DATA     BIT       OISUH
      000000B8H.3 SFRSYM    DATA     BIT       PX01
      000000B8H.4 SFRSYM    DATA     BIT       PX10
      000000F8H.2 SFRSYM    DATA     BIT       OISVH
      000000B8H.5 SFRSYM    DATA     BIT       PX11
      000000F8H.4 SFRSYM    DATA     BIT       OISWH
      000000DCH   SFRSYM    DATA     WORD      LPF_K
      000000F2H   SFRSYM    DATA     WORD      PI_KI
      000000F8H.1 SFRSYM    DATA     BIT       OISUL
      000000A8H   SFRSYM    DATA     BYTE      IE
      000000F8H.3 SFRSYM    DATA     BIT       OISVL
      000000F8H.5 SFRSYM    DATA     BIT       OISWL
      000000D1H   SFRSYM    DATA     BYTE      P1IE
      00000098H.6 SFRSYM    DATA     BIT       MOD0
      000000D3H   SFRSYM    DATA     BYTE      P2IE
      000000D2H   SFRSYM    DATA     BYTE      P1IF
      000000F9H   SFRSYM    DATA     BYTE      PL_CR
      00000098H.7 SFRSYM    DATA     BIT       MOD1
      000000D4H   SFRSYM    DATA     BYTE      P2IF
      000000ACH   SFRSYM    DATA     WORD      TIM2_DR
      00000082H   SFRSYM    DATA     WORD      DP
      000000EEH   SFRSYM    DATA     WORD      PI_KP
      000000A4H   SFRSYM    DATA     WORD      TIM3_DR
      00000094H   SFRSYM    DATA     WORD      TIM4_DR
      0000008CH   SFRSYM    DATA     WORD      TIM5_DR
      000000F1H   SFRSYM    DATA     BYTE      OSC_CFG
      000000C1H   SFRSYM    DATA     BYTE      MD_MODE
      000000ECH   SFRSYM    DATA     WORD      PI_UK
      000000DEH   SFRSYM    DATA     WORD      LPF_X
      00000098H   SFRSYM    DATA     BIT       RI
      000000E6H   SFRSYM    DATA     WORD      LPF_Y
      000000C0H   SFRSYM    DATA     BIT       PTIM00
      000000D0H.7 SFRSYM    DATA     BIT       CY
      00000098H.1 SFRSYM    DATA     BIT       TI
      000000C0H.1 SFRSYM    DATA     BIT       PTIM01
      000000C0H.2 SFRSYM    DATA     BIT       PTIM10
      000000C0H.3 SFRSYM    DATA     BIT       PTIM11
      000000E1H   SFRSYM    DATA     BYTE      SV_CR
      00000098H   SFRSYM    DATA     BYTE      UT_CR
      00000099H   SFRSYM    DATA     BYTE      UT_DR
      000000F8H.6 SFRSYM    DATA     BIT       OIS4
      00000081H   SFRSYM    DATA     BYTE      SP
      000000D0H.2 SFRSYM    DATA     BIT       OV
LX51 LINKER/LOCATER V4.66.1.0                                                         03/30/2017  09:01:59  PAGE 24


      000000C4H   SFRSYM    DATA     BYTE      MD_DA0
      0000009AH   SFRSYM    DATA     WORD      UT_BAUD
      000000CCH   SFRSYM    DATA     BYTE      MD_DB0
      000000C5H   SFRSYM    DATA     BYTE      MD_DA1
      000000CDH   SFRSYM    DATA     BYTE      MD_DB1
      000000C6H   SFRSYM    DATA     BYTE      MD_DA2
      000000CEH   SFRSYM    DATA     BYTE      MD_DB2
      000000C7H   SFRSYM    DATA     BYTE      MD_DA3
      000000B4H   SFRSYM    DATA     WORD      TIM2_ADTR
      000000CFH   SFRSYM    DATA     BYTE      MD_DB3
      000000AFH   SFRSYM    DATA     BYTE      TIM2_ARRH
      000000A7H   SFRSYM    DATA     BYTE      TIM3_ARRH
      00000097H   SFRSYM    DATA     BYTE      TIM4_ARRH
      0000008FH   SFRSYM    DATA     BYTE      TIM5_ARRH
      000000AEH   SFRSYM    DATA     BYTE      TIM2_ARRL
      000000A6H   SFRSYM    DATA     BYTE      TIM3_ARRL
      00000087H   SFRSYM    DATA     BYTE      PCON
      000000E2H   SFRSYM    DATA     WORD      SV_US
      00000096H   SFRSYM    DATA     BYTE      TIM4_ARRL
      0000008EH   SFRSYM    DATA     BYTE      TIM5_ARRL
      000000B2H   SFRSYM    DATA     WORD      TIM2_CMTR
      00000088H   SFRSYM    DATA     BYTE      TCON
      000000AAH   SFRSYM    DATA     WORD      TIM2_CNTR
      000000A2H   SFRSYM    DATA     WORD      TIM3_CNTR
      00000092H   SFRSYM    DATA     WORD      TIM4_CNTR
      0000008AH   SFRSYM    DATA     WORD      TIM5_CNTR
      00000086H   SFRSYM    DATA     BYTE      CFGKEY
      000000E5H   SFRSYM    DATA     BYTE      SV_ANGLEH
      000000D8H   SFRSYM    DATA     BIT       PUART0
      000000E4H   SFRSYM    DATA     BYTE      SV_ANGLEL
      000000C6H   SFRSYM    DATA     WORD      MD_DAH
      000000D8H.1 SFRSYM    DATA     BIT       PUART1
      000000D8H.2 SFRSYM    DATA     BIT       PI2C0
      00000088H.2 SFRSYM    DATA     BIT       IF0
      000000CEH   SFRSYM    DATA     WORD      MD_DBH
      000000D8H.3 SFRSYM    DATA     BIT       PI2C1
      000000F0H   SFRSYM    DATA     BYTE      B
      000000C4H   SFRSYM    DATA     WORD      MD_DAL
      000000A1H   SFRSYM    DATA     BYTE      TIM2_CR0
      000000CCH   SFRSYM    DATA     WORD      MD_DBL
      0000009CH   SFRSYM    DATA     BYTE      TIM3_CR0
      000000A9H   SFRSYM    DATA     BYTE      TIM2_CR1
      0000009EH   SFRSYM    DATA     BYTE      TIM4_CR0
      0000009DH   SFRSYM    DATA     BYTE      TIM3_CR1
      00000089H   SFRSYM    DATA     BYTE      TIM5_CR0
      0000009FH   SFRSYM    DATA     BYTE      TIM4_CR1
      000000F8H   SFRSYM    DATA     BYTE      DRV_OUT
      00000091H   SFRSYM    DATA     BYTE      TIM5_CR1
      000000E0H   SFRSYM    DATA     BYTE      ACC
      000000F7H   SFRSYM    DATA     BYTE      PI_UKMINH
      000000C3H   SFRSYM    DATA     BYTE      MD_MAH
      000000A8H.4 SFRSYM    DATA     BIT       ES0
      000000DBH   SFRSYM    DATA     BYTE      LVSR
      000000CBH   SFRSYM    DATA     BYTE      MD_MBH
      000000C0H.4 SFRSYM    DATA     BIT       PADC0
      000000B8H   SFRSYM    DATA     BYTE      IP0
      000000F5H   SFRSYM    DATA     BYTE      PI_UKMAXH
      000000C0H.5 SFRSYM    DATA     BIT       PADC1
      000000C0H   SFRSYM    DATA     BYTE      IP1
      000000C8H   SFRSYM    DATA     BYTE      IP2
      000000F6H   SFRSYM    DATA     BYTE      PI_UKMINL
      000000C2H   SFRSYM    DATA     BYTE      MD_MAL
      00000098H.2 SFRSYM    DATA     BIT       RB8
      000000D8H   SFRSYM    DATA     BYTE      IP3
      000000CAH   SFRSYM    DATA     BYTE      MD_MBL
LX51 LINKER/LOCATER V4.66.1.0                                                         03/30/2017  09:01:59  PAGE 25


      000000A8H   SFRSYM    DATA     BIT       EX0
      000000F4H   SFRSYM    DATA     BYTE      PI_UKMAXL
      00000098H.3 SFRSYM    DATA     BIT       TB8
      000000B7H   SFRSYM    DATA     BYTE      TIM0_CCR1H
      000000A8H.2 SFRSYM    DATA     BIT       EX1
      000000BBH   SFRSYM    DATA     BYTE      TIM0_CCR2H
      000000D0H   SFRSYM    DATA     BIT       P
      000000BDH   SFRSYM    DATA     BYTE      TIM0_CCR3H
      000000BFH   SFRSYM    DATA     BYTE      TIM0_CCR4H
      000000C8H.2 SFRSYM    DATA     BIT       PTIM230
      000000EBH   SFRSYM    DATA     BYTE      PI_EKH
      00000098H.5 SFRSYM    DATA     BIT       SM2
      000000B6H   SFRSYM    DATA     BYTE      TIM0_CCR1L
      000000B1H   SFRSYM    DATA     BYTE      TIM0_SR1
      000000C8H.3 SFRSYM    DATA     BIT       PTIM231
      000000BAH   SFRSYM    DATA     BYTE      TIM0_CCR2L
      000000BCH   SFRSYM    DATA     BYTE      TIM0_CCR3L
      000000BEH   SFRSYM    DATA     BYTE      TIM0_CCR4L
      000000D8H.6 SFRSYM    DATA     BIT       PMCD0
      000000C8H.4 SFRSYM    DATA     BIT       PTIM450
      000000D0H.3 SFRSYM    DATA     BIT       RS0
      000000DDH   SFRSYM    DATA     BYTE      LPF_KH
      000000F3H   SFRSYM    DATA     BYTE      PI_KIH
      000000EAH   SFRSYM    DATA     BYTE      PI_EKL
      000000E8H   SFRSYM    DATA     BYTE      FOC_SET0
      000000D8H.7 SFRSYM    DATA     BIT       PMCD1
      000000C8H.5 SFRSYM    DATA     BIT       PTIM451
      000000D0H.4 SFRSYM    DATA     BIT       RS1
      000000E9H   SFRSYM    DATA     BYTE      FOC_SET1
      000000B8H.6 SFRSYM    DATA     BIT       PFOC0
      000000DCH   SFRSYM    DATA     BYTE      LPF_KL
      000000F2H   SFRSYM    DATA     BYTE      PI_KIL
      000000B8H.7 SFRSYM    DATA     BIT       PFOC1
      000000ADH   SFRSYM    DATA     BYTE      TIM2_DRH
      000000B9H   SFRSYM    DATA     BYTE      TIM0_IER
      00000083H   SFRSYM    DATA     BYTE      DPH
      000000EFH   SFRSYM    DATA     BYTE      PI_KPH
      000000A5H   SFRSYM    DATA     BYTE      TIM3_DRH
      00000095H   SFRSYM    DATA     BYTE      TIM4_DRH
      0000008DH   SFRSYM    DATA     BYTE      TIM5_DRH
      000000ACH   SFRSYM    DATA     BYTE      TIM2_DRL
      00000082H   SFRSYM    DATA     BYTE      DPL
      000000EEH   SFRSYM    DATA     BYTE      PI_KPL
      000000A4H   SFRSYM    DATA     BYTE      TIM3_DRL
      000000F8H.7 SFRSYM    DATA     BIT       MOE
      000000C0H.6 SFRSYM    DATA     BIT       PCMP0
      000000EDH   SFRSYM    DATA     BYTE      PI_UKH
      00000094H   SFRSYM    DATA     BYTE      TIM4_DRL
      000000C0H.7 SFRSYM    DATA     BIT       PCMP1
      000000DFH   SFRSYM    DATA     BYTE      LPF_XH
      0000008CH   SFRSYM    DATA     BYTE      TIM5_DRL
      000000AEH   SFRSYM    DATA     WORD      TIM2_ARR
      000000A8H.5 SFRSYM    DATA     BIT       MCDIE
      000000C9H   SFRSYM    DATA     BYTE      RSTSRC
      000000E7H   SFRSYM    DATA     BYTE      LPF_YH
      000000A6H   SFRSYM    DATA     WORD      TIM3_ARR
      00000088H.6 SFRSYM    DATA     BIT       MCDIF
      00000098H.4 SFRSYM    DATA     BIT       REN
      00000096H   SFRSYM    DATA     WORD      TIM4_ARR
      000000ECH   SFRSYM    DATA     BYTE      PI_UKL
      000000D7H   SFRSYM    DATA     BYTE      CMP_SR
      0000008EH   SFRSYM    DATA     WORD      TIM5_ARR
      000000DEH   SFRSYM    DATA     BYTE      LPF_XL
      000000E6H   SFRSYM    DATA     BYTE      LPF_YL
      000000C8H   SFRSYM    DATA     BIT       PRTC0
LX51 LINKER/LOCATER V4.66.1.0                                                         03/30/2017  09:01:59  PAGE 26


      000000C8H.1 SFRSYM    DATA     BIT       PRTC1
      000000E8H.7 SFRSYM    DATA     BIT       FOCEN
      000000C8H.6 SFRSYM    DATA     BIT       PTSD0
      000000D8H.4 SFRSYM    DATA     BIT       PSPI0
      000000C8H.7 SFRSYM    DATA     BIT       PTSD1
      000000D8H.5 SFRSYM    DATA     BIT       PSPI1
      0000009BH   SFRSYM    DATA     BYTE      UT_BAUDH
      000000E4H   SFRSYM    DATA     WORD      SV_ANGLE
      000000B5H   SFRSYM    DATA     BYTE      TIM2_ADTRH
      0000009AH   SFRSYM    DATA     BYTE      UT_BAUDL
      000000FCH   SFRSYM    DATA     BYTE      P0_OE
      000000FDH   SFRSYM    DATA     BYTE      P1_OE
      000000D0H.5 SFRSYM    DATA     BIT       F0
      000000B4H   SFRSYM    DATA     BYTE      TIM2_ADTRL
      000000FEH   SFRSYM    DATA     BYTE      P2_OE
      000000D0H.1 SFRSYM    DATA     BIT       F1
      00000080H   SFRSYM    DATA     BIT       GP00
      000000FFH   SFRSYM    DATA     BYTE      P3_OE
      00000090H   SFRSYM    DATA     BIT       GP10
      00000080H.1 SFRSYM    DATA     BIT       GP01
      000000A8H.6 SFRSYM    DATA     BIT       RTCIE
      000000A0H   SFRSYM    DATA     BIT       GP20
      00000090H.1 SFRSYM    DATA     BIT       GP11
      00000080H.2 SFRSYM    DATA     BIT       GP02
      000000E3H   SFRSYM    DATA     BYTE      SV_USH
      000000B0H   SFRSYM    DATA     BIT       GP30
      000000A0H.1 SFRSYM    DATA     BIT       GP21
      00000090H.2 SFRSYM    DATA     BIT       GP12
      00000080H.3 SFRSYM    DATA     BIT       GP03
      000000B8H   SFRSYM    DATA     BIT       PLVW0
      000000A8H.1 SFRSYM    DATA     BIT       TSDIE
      000000D0H   SFRSYM    DATA     BYTE      PSW
      000000B0H.1 SFRSYM    DATA     BIT       GP31
      000000A0H.2 SFRSYM    DATA     BIT       GP22
      00000090H.3 SFRSYM    DATA     BIT       GP13
      00000080H.4 SFRSYM    DATA     BIT       GP04
      000000B8H.1 SFRSYM    DATA     BIT       PLVW1
      000000A8H.3 SFRSYM    DATA     BIT       SPIIE
      00000088H.5 SFRSYM    DATA     BIT       TSDIF
      000000B0H.2 SFRSYM    DATA     BIT       GP32
      000000A0H.3 SFRSYM    DATA     BIT       GP23
      00000090H.4 SFRSYM    DATA     BIT       GP14
      00000080H.5 SFRSYM    DATA     BIT       GP05
      00000084H   SFRSYM    DATA     BYTE      FLKEY
      000000B3H   SFRSYM    DATA     BYTE      TIM2_CMTRH
      000000B0H.3 SFRSYM    DATA     BIT       GP33
      000000A0H.4 SFRSYM    DATA     BIT       GP24
      00000090H.5 SFRSYM    DATA     BIT       GP15
      00000080H.6 SFRSYM    DATA     BIT       GP06
      00000088H   SFRSYM    DATA     BIT       IT00

      01000906H   BLOCK     CODE     ---       LVL=0
      01000906H   LINE      CODE     ---       #23
      01000906H   LINE      CODE     ---       #24
      01000906H   LINE      CODE     ---       #32
      0100090BH   LINE      CODE     ---       #33
      01000910H   LINE      CODE     ---       #39
      01000917H   LINE      CODE     ---       #40
      ---         BLOCKEND  ---      ---       LVL=0

      ---         MODULE    ---      ---       TIMERINIT
      010002A4H   PUBLIC    CODE     ---       TIM0_Init
      000000E2H   SFRSYM    DATA     BYTE      SV_USL
      000000ABH   SFRSYM    DATA     BYTE      TIM2_CNTRH
      000000B0H.4 SFRSYM    DATA     BIT       GP34
LX51 LINKER/LOCATER V4.66.1.0                                                         03/30/2017  09:01:59  PAGE 27


      000000A0H.5 SFRSYM    DATA     BIT       GP25
      00000090H.6 SFRSYM    DATA     BIT       GP16
      00000080H.7 SFRSYM    DATA     BIT       GP07
      00000088H.1 SFRSYM    DATA     BIT       IT01
      00000088H.3 SFRSYM    DATA     BIT       IT10
      000000F6H   SFRSYM    DATA     WORD      PI_UKMIN
      000000C2H   SFRSYM    DATA     WORD      MD_MA
      000000A3H   SFRSYM    DATA     BYTE      TIM3_CNTRH
      000000B0H.5 SFRSYM    DATA     BIT       GP35
      000000A0H.6 SFRSYM    DATA     BIT       GP26
      00000090H.7 SFRSYM    DATA     BIT       GP17
      00000080H   SFRSYM    DATA     BYTE      P0
      00000088H.4 SFRSYM    DATA     BIT       IT11
      000000CAH   SFRSYM    DATA     WORD      MD_MB
      00000093H   SFRSYM    DATA     BYTE      TIM4_CNTRH
      000000B0H.6 SFRSYM    DATA     BIT       GP36
      000000A0H.7 SFRSYM    DATA     BIT       GP27
      00000090H   SFRSYM    DATA     BYTE      P1
      000000D9H   SFRSYM    DATA     BYTE      EVT_FILT
      000000F4H   SFRSYM    DATA     WORD      PI_UKMAX
      0000008BH   SFRSYM    DATA     BYTE      TIM5_CNTRH
      000000B2H   SFRSYM    DATA     BYTE      TIM2_CMTRL
      000000B0H.7 SFRSYM    DATA     BIT       GP37
      000000A0H   SFRSYM    DATA     BYTE      P2
      000000AAH   SFRSYM    DATA     BYTE      TIM2_CNTRL
      000000B0H   SFRSYM    DATA     BYTE      P3
      000000A2H   SFRSYM    DATA     BYTE      TIM3_CNTRL
      000000D0H.6 SFRSYM    DATA     BIT       AC
      00000092H   SFRSYM    DATA     BYTE      TIM4_CNTRL
      0000008AH   SFRSYM    DATA     BYTE      TIM5_CNTRL
      000000B6H   SFRSYM    DATA     WORD      TIM0_CCR1
      000000A8H.7 SFRSYM    DATA     BIT       EA
      000000D5H   SFRSYM    DATA     BYTE      CMP_CR0
      000000BAH   SFRSYM    DATA     WORD      TIM0_CCR2
      000000D6H   SFRSYM    DATA     BYTE      CMP_CR1
      000000BCH   SFRSYM    DATA     WORD      TIM0_CCR3
      00000085H   SFRSYM    DATA     BYTE      PSCTL
      000000DAH   SFRSYM    DATA     BYTE      CMP_CR2
      000000BEH   SFRSYM    DATA     WORD      TIM0_CCR4
      000000B8H.2 SFRSYM    DATA     BIT       PX00
      000000EAH   SFRSYM    DATA     WORD      PI_EK
      000000F8H   SFRSYM    DATA     BIT       OISUH
      000000B8H.3 SFRSYM    DATA     BIT       PX01
      000000B8H.4 SFRSYM    DATA     BIT       PX10
      000000F8H.2 SFRSYM    DATA     BIT       OISVH
      000000B8H.5 SFRSYM    DATA     BIT       PX11
      000000F8H.4 SFRSYM    DATA     BIT       OISWH
      000000DCH   SFRSYM    DATA     WORD      LPF_K
      000000F2H   SFRSYM    DATA     WORD      PI_KI
      000000F8H.1 SFRSYM    DATA     BIT       OISUL
      000000A8H   SFRSYM    DATA     BYTE      IE
      000000F8H.3 SFRSYM    DATA     BIT       OISVL
      000000F8H.5 SFRSYM    DATA     BIT       OISWL
      000000D1H   SFRSYM    DATA     BYTE      P1IE
      00000098H.6 SFRSYM    DATA     BIT       MOD0
      000000D3H   SFRSYM    DATA     BYTE      P2IE
      000000D2H   SFRSYM    DATA     BYTE      P1IF
      000000F9H   SFRSYM    DATA     BYTE      PL_CR
      00000098H.7 SFRSYM    DATA     BIT       MOD1
      000000D4H   SFRSYM    DATA     BYTE      P2IF
      000000ACH   SFRSYM    DATA     WORD      TIM2_DR
      00000082H   SFRSYM    DATA     WORD      DP
      000000EEH   SFRSYM    DATA     WORD      PI_KP
      000000A4H   SFRSYM    DATA     WORD      TIM3_DR
      00000094H   SFRSYM    DATA     WORD      TIM4_DR
LX51 LINKER/LOCATER V4.66.1.0                                                         03/30/2017  09:01:59  PAGE 28


      0000008CH   SFRSYM    DATA     WORD      TIM5_DR
      000000F1H   SFRSYM    DATA     BYTE      OSC_CFG
      000000C1H   SFRSYM    DATA     BYTE      MD_MODE
      000000ECH   SFRSYM    DATA     WORD      PI_UK
      000000DEH   SFRSYM    DATA     WORD      LPF_X
      00000098H   SFRSYM    DATA     BIT       RI
      000000E6H   SFRSYM    DATA     WORD      LPF_Y
      000000C0H   SFRSYM    DATA     BIT       PTIM00
      000000D0H.7 SFRSYM    DATA     BIT       CY
      00000098H.1 SFRSYM    DATA     BIT       TI
      000000C0H.1 SFRSYM    DATA     BIT       PTIM01
      000000C0H.2 SFRSYM    DATA     BIT       PTIM10
      000000C0H.3 SFRSYM    DATA     BIT       PTIM11
      000000E1H   SFRSYM    DATA     BYTE      SV_CR
      00000098H   SFRSYM    DATA     BYTE      UT_CR
      00000099H   SFRSYM    DATA     BYTE      UT_DR
      000000F8H.6 SFRSYM    DATA     BIT       OIS4
      00000081H   SFRSYM    DATA     BYTE      SP
      000000D0H.2 SFRSYM    DATA     BIT       OV
      000000C4H   SFRSYM    DATA     BYTE      MD_DA0
      0000009AH   SFRSYM    DATA     WORD      UT_BAUD
      000000CCH   SFRSYM    DATA     BYTE      MD_DB0
      000000C5H   SFRSYM    DATA     BYTE      MD_DA1
      000000CDH   SFRSYM    DATA     BYTE      MD_DB1
      000000C6H   SFRSYM    DATA     BYTE      MD_DA2
      000000CEH   SFRSYM    DATA     BYTE      MD_DB2
      000000C7H   SFRSYM    DATA     BYTE      MD_DA3
      000000B4H   SFRSYM    DATA     WORD      TIM2_ADTR
      000000CFH   SFRSYM    DATA     BYTE      MD_DB3
      000000AFH   SFRSYM    DATA     BYTE      TIM2_ARRH
      000000A7H   SFRSYM    DATA     BYTE      TIM3_ARRH
      00000097H   SFRSYM    DATA     BYTE      TIM4_ARRH
      0000008FH   SFRSYM    DATA     BYTE      TIM5_ARRH
      000000AEH   SFRSYM    DATA     BYTE      TIM2_ARRL
      000000A6H   SFRSYM    DATA     BYTE      TIM3_ARRL
      00000087H   SFRSYM    DATA     BYTE      PCON
      000000E2H   SFRSYM    DATA     WORD      SV_US
      00000096H   SFRSYM    DATA     BYTE      TIM4_ARRL
      0000008EH   SFRSYM    DATA     BYTE      TIM5_ARRL
      000000B2H   SFRSYM    DATA     WORD      TIM2_CMTR
      00000088H   SFRSYM    DATA     BYTE      TCON
      000000AAH   SFRSYM    DATA     WORD      TIM2_CNTR
      000000A2H   SFRSYM    DATA     WORD      TIM3_CNTR
      00000092H   SFRSYM    DATA     WORD      TIM4_CNTR
      0000008AH   SFRSYM    DATA     WORD      TIM5_CNTR
      00000086H   SFRSYM    DATA     BYTE      CFGKEY
      000000E5H   SFRSYM    DATA     BYTE      SV_ANGLEH
      000000D8H   SFRSYM    DATA     BIT       PUART0
      000000E4H   SFRSYM    DATA     BYTE      SV_ANGLEL
      000000C6H   SFRSYM    DATA     WORD      MD_DAH
      000000D8H.1 SFRSYM    DATA     BIT       PUART1
      000000D8H.2 SFRSYM    DATA     BIT       PI2C0
      00000088H.2 SFRSYM    DATA     BIT       IF0
      000000CEH   SFRSYM    DATA     WORD      MD_DBH
      000000D8H.3 SFRSYM    DATA     BIT       PI2C1
      000000F0H   SFRSYM    DATA     BYTE      B
      000000C4H   SFRSYM    DATA     WORD      MD_DAL
      000000A1H   SFRSYM    DATA     BYTE      TIM2_CR0
      000000CCH   SFRSYM    DATA     WORD      MD_DBL
      0000009CH   SFRSYM    DATA     BYTE      TIM3_CR0
      000000A9H   SFRSYM    DATA     BYTE      TIM2_CR1
      0000009EH   SFRSYM    DATA     BYTE      TIM4_CR0
      0000009DH   SFRSYM    DATA     BYTE      TIM3_CR1
      00000089H   SFRSYM    DATA     BYTE      TIM5_CR0
      0000009FH   SFRSYM    DATA     BYTE      TIM4_CR1
LX51 LINKER/LOCATER V4.66.1.0                                                         03/30/2017  09:01:59  PAGE 29


      000000F8H   SFRSYM    DATA     BYTE      DRV_OUT
      00000091H   SFRSYM    DATA     BYTE      TIM5_CR1
      000000E0H   SFRSYM    DATA     BYTE      ACC
      000000F7H   SFRSYM    DATA     BYTE      PI_UKMINH
      000000C3H   SFRSYM    DATA     BYTE      MD_MAH
      000000A8H.4 SFRSYM    DATA     BIT       ES0
      000000DBH   SFRSYM    DATA     BYTE      LVSR
      000000CBH   SFRSYM    DATA     BYTE      MD_MBH
      000000C0H.4 SFRSYM    DATA     BIT       PADC0
      000000B8H   SFRSYM    DATA     BYTE      IP0
      000000F5H   SFRSYM    DATA     BYTE      PI_UKMAXH
      000000C0H.5 SFRSYM    DATA     BIT       PADC1
      000000C0H   SFRSYM    DATA     BYTE      IP1
      000000C8H   SFRSYM    DATA     BYTE      IP2
      000000F6H   SFRSYM    DATA     BYTE      PI_UKMINL
      000000C2H   SFRSYM    DATA     BYTE      MD_MAL
      00000098H.2 SFRSYM    DATA     BIT       RB8
      000000D8H   SFRSYM    DATA     BYTE      IP3
      000000CAH   SFRSYM    DATA     BYTE      MD_MBL
      000000A8H   SFRSYM    DATA     BIT       EX0
      000000F4H   SFRSYM    DATA     BYTE      PI_UKMAXL
      00000098H.3 SFRSYM    DATA     BIT       TB8
      000000B7H   SFRSYM    DATA     BYTE      TIM0_CCR1H
      000000A8H.2 SFRSYM    DATA     BIT       EX1
      000000BBH   SFRSYM    DATA     BYTE      TIM0_CCR2H
      000000D0H   SFRSYM    DATA     BIT       P
      000000BDH   SFRSYM    DATA     BYTE      TIM0_CCR3H
      000000BFH   SFRSYM    DATA     BYTE      TIM0_CCR4H
      000000C8H.2 SFRSYM    DATA     BIT       PTIM230
      000000EBH   SFRSYM    DATA     BYTE      PI_EKH
      00000098H.5 SFRSYM    DATA     BIT       SM2
      000000B6H   SFRSYM    DATA     BYTE      TIM0_CCR1L
      000000B1H   SFRSYM    DATA     BYTE      TIM0_SR1
      000000C8H.3 SFRSYM    DATA     BIT       PTIM231
      000000BAH   SFRSYM    DATA     BYTE      TIM0_CCR2L
      000000BCH   SFRSYM    DATA     BYTE      TIM0_CCR3L
      000000BEH   SFRSYM    DATA     BYTE      TIM0_CCR4L
      000000D8H.6 SFRSYM    DATA     BIT       PMCD0
      000000C8H.4 SFRSYM    DATA     BIT       PTIM450
      000000D0H.3 SFRSYM    DATA     BIT       RS0
      000000DDH   SFRSYM    DATA     BYTE      LPF_KH
      000000F3H   SFRSYM    DATA     BYTE      PI_KIH
      000000EAH   SFRSYM    DATA     BYTE      PI_EKL
      000000E8H   SFRSYM    DATA     BYTE      FOC_SET0
      000000D8H.7 SFRSYM    DATA     BIT       PMCD1
      000000C8H.5 SFRSYM    DATA     BIT       PTIM451
      000000D0H.4 SFRSYM    DATA     BIT       RS1
      000000E9H   SFRSYM    DATA     BYTE      FOC_SET1
      000000B8H.6 SFRSYM    DATA     BIT       PFOC0
      000000DCH   SFRSYM    DATA     BYTE      LPF_KL
      000000F2H   SFRSYM    DATA     BYTE      PI_KIL
      000000B8H.7 SFRSYM    DATA     BIT       PFOC1
      000000ADH   SFRSYM    DATA     BYTE      TIM2_DRH
      000000B9H   SFRSYM    DATA     BYTE      TIM0_IER
      00000083H   SFRSYM    DATA     BYTE      DPH
      000000EFH   SFRSYM    DATA     BYTE      PI_KPH
      000000A5H   SFRSYM    DATA     BYTE      TIM3_DRH
      00000095H   SFRSYM    DATA     BYTE      TIM4_DRH
      0000008DH   SFRSYM    DATA     BYTE      TIM5_DRH
      000000ACH   SFRSYM    DATA     BYTE      TIM2_DRL
      00000082H   SFRSYM    DATA     BYTE      DPL
      000000EEH   SFRSYM    DATA     BYTE      PI_KPL
      000000A4H   SFRSYM    DATA     BYTE      TIM3_DRL
      000000F8H.7 SFRSYM    DATA     BIT       MOE
      000000C0H.6 SFRSYM    DATA     BIT       PCMP0
LX51 LINKER/LOCATER V4.66.1.0                                                         03/30/2017  09:01:59  PAGE 30


      000000EDH   SFRSYM    DATA     BYTE      PI_UKH
      00000094H   SFRSYM    DATA     BYTE      TIM4_DRL
      000000C0H.7 SFRSYM    DATA     BIT       PCMP1
      000000DFH   SFRSYM    DATA     BYTE      LPF_XH
      0000008CH   SFRSYM    DATA     BYTE      TIM5_DRL
      000000AEH   SFRSYM    DATA     WORD      TIM2_ARR
      000000A8H.5 SFRSYM    DATA     BIT       MCDIE
      000000C9H   SFRSYM    DATA     BYTE      RSTSRC
      000000E7H   SFRSYM    DATA     BYTE      LPF_YH
      000000A6H   SFRSYM    DATA     WORD      TIM3_ARR
      00000088H.6 SFRSYM    DATA     BIT       MCDIF
      00000098H.4 SFRSYM    DATA     BIT       REN
      00000096H   SFRSYM    DATA     WORD      TIM4_ARR
      000000ECH   SFRSYM    DATA     BYTE      PI_UKL
      000000D7H   SFRSYM    DATA     BYTE      CMP_SR
      0000008EH   SFRSYM    DATA     WORD      TIM5_ARR
      000000DEH   SFRSYM    DATA     BYTE      LPF_XL
      000000E6H   SFRSYM    DATA     BYTE      LPF_YL
      000000C8H   SFRSYM    DATA     BIT       PRTC0
      000000C8H.1 SFRSYM    DATA     BIT       PRTC1
      000000E8H.7 SFRSYM    DATA     BIT       FOCEN
      000000C8H.6 SFRSYM    DATA     BIT       PTSD0
      000000D8H.4 SFRSYM    DATA     BIT       PSPI0
      000000C8H.7 SFRSYM    DATA     BIT       PTSD1
      000000D8H.5 SFRSYM    DATA     BIT       PSPI1
      0000009BH   SFRSYM    DATA     BYTE      UT_BAUDH
      000000E4H   SFRSYM    DATA     WORD      SV_ANGLE
      000000B5H   SFRSYM    DATA     BYTE      TIM2_ADTRH
      0000009AH   SFRSYM    DATA     BYTE      UT_BAUDL
      000000FCH   SFRSYM    DATA     BYTE      P0_OE
      000000FDH   SFRSYM    DATA     BYTE      P1_OE
      000000D0H.5 SFRSYM    DATA     BIT       F0
      000000B4H   SFRSYM    DATA     BYTE      TIM2_ADTRL
      000000FEH   SFRSYM    DATA     BYTE      P2_OE
      000000D0H.1 SFRSYM    DATA     BIT       F1
      00000080H   SFRSYM    DATA     BIT       GP00
      000000FFH   SFRSYM    DATA     BYTE      P3_OE
      00000090H   SFRSYM    DATA     BIT       GP10
      00000080H.1 SFRSYM    DATA     BIT       GP01
      000000A8H.6 SFRSYM    DATA     BIT       RTCIE
      000000A0H   SFRSYM    DATA     BIT       GP20
      00000090H.1 SFRSYM    DATA     BIT       GP11
      00000080H.2 SFRSYM    DATA     BIT       GP02
      000000E3H   SFRSYM    DATA     BYTE      SV_USH
      000000B0H   SFRSYM    DATA     BIT       GP30
      000000A0H.1 SFRSYM    DATA     BIT       GP21
      00000090H.2 SFRSYM    DATA     BIT       GP12
      00000080H.3 SFRSYM    DATA     BIT       GP03
      000000B8H   SFRSYM    DATA     BIT       PLVW0
      000000A8H.1 SFRSYM    DATA     BIT       TSDIE
      000000D0H   SFRSYM    DATA     BYTE      PSW
      000000B0H.1 SFRSYM    DATA     BIT       GP31
      000000A0H.2 SFRSYM    DATA     BIT       GP22
      00000090H.3 SFRSYM    DATA     BIT       GP13
      00000080H.4 SFRSYM    DATA     BIT       GP04
      000000B8H.1 SFRSYM    DATA     BIT       PLVW1
      000000A8H.3 SFRSYM    DATA     BIT       SPIIE
      00000088H.5 SFRSYM    DATA     BIT       TSDIF
      000000B0H.2 SFRSYM    DATA     BIT       GP32
      000000A0H.3 SFRSYM    DATA     BIT       GP23
      00000090H.4 SFRSYM    DATA     BIT       GP14
      00000080H.5 SFRSYM    DATA     BIT       GP05
      00000084H   SFRSYM    DATA     BYTE      FLKEY
      000000B3H   SFRSYM    DATA     BYTE      TIM2_CMTRH
      000000B0H.3 SFRSYM    DATA     BIT       GP33
LX51 LINKER/LOCATER V4.66.1.0                                                         03/30/2017  09:01:59  PAGE 31


      000000A0H.4 SFRSYM    DATA     BIT       GP24
      00000090H.5 SFRSYM    DATA     BIT       GP15
      00000080H.6 SFRSYM    DATA     BIT       GP06
      00000088H   SFRSYM    DATA     BIT       IT00

      010002A4H   BLOCK     CODE     ---       LVL=0
      010002A4H   LINE      CODE     ---       #29
      010002A4H   LINE      CODE     ---       #30
      010002A4H   LINE      CODE     ---       #31
      010002ABH   LINE      CODE     ---       #41
      010002AFH   LINE      CODE     ---       #42
      010002B3H   LINE      CODE     ---       #43
      010002B7H   LINE      CODE     ---       #46
      010002BBH   LINE      CODE     ---       #49
      010002BFH   LINE      CODE     ---       #52
      010002C5H   LINE      CODE     ---       #53
      010002CAH   LINE      CODE     ---       #54
      010002D4H   LINE      CODE     ---       #55
      010002DCH   LINE      CODE     ---       #69
      010002E3H   LINE      CODE     ---       #72
      010002EAH   LINE      CODE     ---       #73
      010002EEH   LINE      CODE     ---       #74
      010002F2H   LINE      CODE     ---       #75
      010002F6H   LINE      CODE     ---       #76
      010002FDH   LINE      CODE     ---       #77
      01000301H   LINE      CODE     ---       #78
      01000305H   LINE      CODE     ---       #79
      01000309H   LINE      CODE     ---       #82
      01000310H   LINE      CODE     ---       #83
      01000314H   LINE      CODE     ---       #84
      01000318H   LINE      CODE     ---       #85
      0100031CH   LINE      CODE     ---       #86
      01000323H   LINE      CODE     ---       #87
      01000327H   LINE      CODE     ---       #88
      0100032BH   LINE      CODE     ---       #89
      0100032FH   LINE      CODE     ---       #92
      01000336H   LINE      CODE     ---       #93
      0100033AH   LINE      CODE     ---       #94
      0100033EH   LINE      CODE     ---       #95
      01000342H   LINE      CODE     ---       #96
      01000349H   LINE      CODE     ---       #97
      0100034DH   LINE      CODE     ---       #98
      01000351H   LINE      CODE     ---       #99
      01000355H   LINE      CODE     ---       #102
      0100035CH   LINE      CODE     ---       #103
      01000360H   LINE      CODE     ---       #104
      01000364H   LINE      CODE     ---       #105
      01000368H   LINE      CODE     ---       #106
      0100036FH   LINE      CODE     ---       #107
      01000373H   LINE      CODE     ---       #111
      01000379H   LINE      CODE     ---       #114
      0100037FH   LINE      CODE     ---       #115
      01000385H   LINE      CODE     ---       #116
      0100038BH   LINE      CODE     ---       #117
      01000391H   LINE      CODE     ---       #120
      01000398H   LINE      CODE     ---       #121
      0100039CH   LINE      CODE     ---       #122
      0100039FH   LINE      CODE     ---       #130
      010003A6H   LINE      CODE     ---       #131
      010003AAH   LINE      CODE     ---       #134
      010003ADH   LINE      CODE     ---       #135
      010003B0H   LINE      CODE     ---       #136
      010003B3H   LINE      CODE     ---       #137
      010003B6H   LINE      CODE     ---       #138
      010003B9H   LINE      CODE     ---       #139
LX51 LINKER/LOCATER V4.66.1.0                                                         03/30/2017  09:01:59  PAGE 32


      010003BCH   LINE      CODE     ---       #142
      010003BFH   LINE      CODE     ---       #143
      010003C2H   LINE      CODE     ---       #144
      010003C5H   LINE      CODE     ---       #145
      010003C8H   LINE      CODE     ---       #146
      010003CBH   LINE      CODE     ---       #147
      010003CEH   LINE      CODE     ---       #148
      010003D0H   LINE      CODE     ---       #149
      010003D2H   LINE      CODE     ---       #150
      010003D4H   LINE      CODE     ---       #153
      010003D9H   LINE      CODE     ---       #154
      010003DDH   LINE      CODE     ---       #155
      010003E1H   LINE      CODE     ---       #156
      010003E5H   LINE      CODE     ---       #157
      010003E9H   LINE      CODE     ---       #158
      010003EDH   LINE      CODE     ---       #160
      010003F4H   LINE      CODE     ---       #162
      ---         BLOCKEND  ---      ---       LVL=0

      ---         MODULE    ---      ---       ADCINIT
      02000000H   PUBLIC    XDATA    ---       ADCData
      0100065DH   PUBLIC    CODE     ---       ADCGetConversionValue
      010004D6H   PUBLIC    CODE     ---       ADCDataInit
      010005F0H   PUBLIC    CODE     ---       ADC_Init
      000000E2H   SFRSYM    DATA     BYTE      SV_USL
      000000ABH   SFRSYM    DATA     BYTE      TIM2_CNTRH
      000000B0H.4 SFRSYM    DATA     BIT       GP34
      000000A0H.5 SFRSYM    DATA     BIT       GP25
      00000090H.6 SFRSYM    DATA     BIT       GP16
      00000080H.7 SFRSYM    DATA     BIT       GP07
      00000088H.1 SFRSYM    DATA     BIT       IT01
      00000088H.3 SFRSYM    DATA     BIT       IT10
      000000F6H   SFRSYM    DATA     WORD      PI_UKMIN
      000000C2H   SFRSYM    DATA     WORD      MD_MA
      000000A3H   SFRSYM    DATA     BYTE      TIM3_CNTRH
      000000B0H.5 SFRSYM    DATA     BIT       GP35
      000000A0H.6 SFRSYM    DATA     BIT       GP26
      00000090H.7 SFRSYM    DATA     BIT       GP17
      00000080H   SFRSYM    DATA     BYTE      P0
      00000088H.4 SFRSYM    DATA     BIT       IT11
      000000CAH   SFRSYM    DATA     WORD      MD_MB
      00000093H   SFRSYM    DATA     BYTE      TIM4_CNTRH
      000000B0H.6 SFRSYM    DATA     BIT       GP36
      000000A0H.7 SFRSYM    DATA     BIT       GP27
      00000090H   SFRSYM    DATA     BYTE      P1
      000000D9H   SFRSYM    DATA     BYTE      EVT_FILT
      000000F4H   SFRSYM    DATA     WORD      PI_UKMAX
      0000008BH   SFRSYM    DATA     BYTE      TIM5_CNTRH
      000000B2H   SFRSYM    DATA     BYTE      TIM2_CMTRL
      000000B0H.7 SFRSYM    DATA     BIT       GP37
      000000A0H   SFRSYM    DATA     BYTE      P2
      000000AAH   SFRSYM    DATA     BYTE      TIM2_CNTRL
      000000B0H   SFRSYM    DATA     BYTE      P3
      000000A2H   SFRSYM    DATA     BYTE      TIM3_CNTRL
      000000D0H.6 SFRSYM    DATA     BIT       AC
      00000092H   SFRSYM    DATA     BYTE      TIM4_CNTRL
      0000008AH   SFRSYM    DATA     BYTE      TIM5_CNTRL
      000000B6H   SFRSYM    DATA     WORD      TIM0_CCR1
      000000A8H.7 SFRSYM    DATA     BIT       EA
      000000D5H   SFRSYM    DATA     BYTE      CMP_CR0
      000000BAH   SFRSYM    DATA     WORD      TIM0_CCR2
      000000D6H   SFRSYM    DATA     BYTE      CMP_CR1
      000000BCH   SFRSYM    DATA     WORD      TIM0_CCR3
      00000085H   SFRSYM    DATA     BYTE      PSCTL
      000000DAH   SFRSYM    DATA     BYTE      CMP_CR2
LX51 LINKER/LOCATER V4.66.1.0                                                         03/30/2017  09:01:59  PAGE 33


      000000BEH   SFRSYM    DATA     WORD      TIM0_CCR4
      000000B8H.2 SFRSYM    DATA     BIT       PX00
      000000EAH   SFRSYM    DATA     WORD      PI_EK
      000000F8H   SFRSYM    DATA     BIT       OISUH
      000000B8H.3 SFRSYM    DATA     BIT       PX01
      000000B8H.4 SFRSYM    DATA     BIT       PX10
      000000F8H.2 SFRSYM    DATA     BIT       OISVH
      000000B8H.5 SFRSYM    DATA     BIT       PX11
      000000F8H.4 SFRSYM    DATA     BIT       OISWH
      000000DCH   SFRSYM    DATA     WORD      LPF_K
      000000F2H   SFRSYM    DATA     WORD      PI_KI
      000000F8H.1 SFRSYM    DATA     BIT       OISUL
      000000A8H   SFRSYM    DATA     BYTE      IE
      000000F8H.3 SFRSYM    DATA     BIT       OISVL
      000000F8H.5 SFRSYM    DATA     BIT       OISWL
      000000D1H   SFRSYM    DATA     BYTE      P1IE
      00000098H.6 SFRSYM    DATA     BIT       MOD0
      000000D3H   SFRSYM    DATA     BYTE      P2IE
      000000D2H   SFRSYM    DATA     BYTE      P1IF
      000000F9H   SFRSYM    DATA     BYTE      PL_CR
      00000098H.7 SFRSYM    DATA     BIT       MOD1
      000000D4H   SFRSYM    DATA     BYTE      P2IF
      000000ACH   SFRSYM    DATA     WORD      TIM2_DR
      00000082H   SFRSYM    DATA     WORD      DP
      000000EEH   SFRSYM    DATA     WORD      PI_KP
      000000A4H   SFRSYM    DATA     WORD      TIM3_DR
      00000094H   SFRSYM    DATA     WORD      TIM4_DR
      0000008CH   SFRSYM    DATA     WORD      TIM5_DR
      000000F1H   SFRSYM    DATA     BYTE      OSC_CFG
      000000C1H   SFRSYM    DATA     BYTE      MD_MODE
      000000ECH   SFRSYM    DATA     WORD      PI_UK
      000000DEH   SFRSYM    DATA     WORD      LPF_X
      00000098H   SFRSYM    DATA     BIT       RI
      000000E6H   SFRSYM    DATA     WORD      LPF_Y
      000000C0H   SFRSYM    DATA     BIT       PTIM00
      000000D0H.7 SFRSYM    DATA     BIT       CY
      00000098H.1 SFRSYM    DATA     BIT       TI
      000000C0H.1 SFRSYM    DATA     BIT       PTIM01
      000000C0H.2 SFRSYM    DATA     BIT       PTIM10
      000000C0H.3 SFRSYM    DATA     BIT       PTIM11
      000000E1H   SFRSYM    DATA     BYTE      SV_CR
      00000098H   SFRSYM    DATA     BYTE      UT_CR
      00000099H   SFRSYM    DATA     BYTE      UT_DR
      000000F8H.6 SFRSYM    DATA     BIT       OIS4
      00000081H   SFRSYM    DATA     BYTE      SP
      000000D0H.2 SFRSYM    DATA     BIT       OV
      000000C4H   SFRSYM    DATA     BYTE      MD_DA0
      0000009AH   SFRSYM    DATA     WORD      UT_BAUD
      000000CCH   SFRSYM    DATA     BYTE      MD_DB0
      000000C5H   SFRSYM    DATA     BYTE      MD_DA1
      000000CDH   SFRSYM    DATA     BYTE      MD_DB1
      000000C6H   SFRSYM    DATA     BYTE      MD_DA2
      000000CEH   SFRSYM    DATA     BYTE      MD_DB2
      000000C7H   SFRSYM    DATA     BYTE      MD_DA3
      000000B4H   SFRSYM    DATA     WORD      TIM2_ADTR
      000000CFH   SFRSYM    DATA     BYTE      MD_DB3
      000000AFH   SFRSYM    DATA     BYTE      TIM2_ARRH
      000000A7H   SFRSYM    DATA     BYTE      TIM3_ARRH
      00000097H   SFRSYM    DATA     BYTE      TIM4_ARRH
      0000008FH   SFRSYM    DATA     BYTE      TIM5_ARRH
      000000AEH   SFRSYM    DATA     BYTE      TIM2_ARRL
      000000A6H   SFRSYM    DATA     BYTE      TIM3_ARRL
      00000087H   SFRSYM    DATA     BYTE      PCON
      000000E2H   SFRSYM    DATA     WORD      SV_US
      00000096H   SFRSYM    DATA     BYTE      TIM4_ARRL
LX51 LINKER/LOCATER V4.66.1.0                                                         03/30/2017  09:01:59  PAGE 34


      0000008EH   SFRSYM    DATA     BYTE      TIM5_ARRL
      000000B2H   SFRSYM    DATA     WORD      TIM2_CMTR
      00000088H   SFRSYM    DATA     BYTE      TCON
      000000AAH   SFRSYM    DATA     WORD      TIM2_CNTR
      000000A2H   SFRSYM    DATA     WORD      TIM3_CNTR
      00000092H   SFRSYM    DATA     WORD      TIM4_CNTR
      0000008AH   SFRSYM    DATA     WORD      TIM5_CNTR
      00000086H   SFRSYM    DATA     BYTE      CFGKEY
      000000E5H   SFRSYM    DATA     BYTE      SV_ANGLEH
      000000D8H   SFRSYM    DATA     BIT       PUART0
      000000E4H   SFRSYM    DATA     BYTE      SV_ANGLEL
      000000C6H   SFRSYM    DATA     WORD      MD_DAH
      000000D8H.1 SFRSYM    DATA     BIT       PUART1
      000000D8H.2 SFRSYM    DATA     BIT       PI2C0
      00000088H.2 SFRSYM    DATA     BIT       IF0
      000000CEH   SFRSYM    DATA     WORD      MD_DBH
      000000D8H.3 SFRSYM    DATA     BIT       PI2C1
      000000F0H   SFRSYM    DATA     BYTE      B
      000000C4H   SFRSYM    DATA     WORD      MD_DAL
      000000A1H   SFRSYM    DATA     BYTE      TIM2_CR0
      000000CCH   SFRSYM    DATA     WORD      MD_DBL
      0000009CH   SFRSYM    DATA     BYTE      TIM3_CR0
      000000A9H   SFRSYM    DATA     BYTE      TIM2_CR1
      0000009EH   SFRSYM    DATA     BYTE      TIM4_CR0
      0000009DH   SFRSYM    DATA     BYTE      TIM3_CR1
      00000089H   SFRSYM    DATA     BYTE      TIM5_CR0
      0000009FH   SFRSYM    DATA     BYTE      TIM4_CR1
      000000F8H   SFRSYM    DATA     BYTE      DRV_OUT
      00000091H   SFRSYM    DATA     BYTE      TIM5_CR1
      000000E0H   SFRSYM    DATA     BYTE      ACC
      000000F7H   SFRSYM    DATA     BYTE      PI_UKMINH
      000000C3H   SFRSYM    DATA     BYTE      MD_MAH
      000000A8H.4 SFRSYM    DATA     BIT       ES0
      000000DBH   SFRSYM    DATA     BYTE      LVSR
      000000CBH   SFRSYM    DATA     BYTE      MD_MBH
      000000C0H.4 SFRSYM    DATA     BIT       PADC0
      000000B8H   SFRSYM    DATA     BYTE      IP0
      000000F5H   SFRSYM    DATA     BYTE      PI_UKMAXH
      000000C0H.5 SFRSYM    DATA     BIT       PADC1
      000000C0H   SFRSYM    DATA     BYTE      IP1
      000000C8H   SFRSYM    DATA     BYTE      IP2
      000000F6H   SFRSYM    DATA     BYTE      PI_UKMINL
      000000C2H   SFRSYM    DATA     BYTE      MD_MAL
      00000098H.2 SFRSYM    DATA     BIT       RB8
      000000D8H   SFRSYM    DATA     BYTE      IP3
      000000CAH   SFRSYM    DATA     BYTE      MD_MBL
      000000A8H   SFRSYM    DATA     BIT       EX0
      000000F4H   SFRSYM    DATA     BYTE      PI_UKMAXL
      00000098H.3 SFRSYM    DATA     BIT       TB8
      000000B7H   SFRSYM    DATA     BYTE      TIM0_CCR1H
      000000A8H.2 SFRSYM    DATA     BIT       EX1
      000000BBH   SFRSYM    DATA     BYTE      TIM0_CCR2H
      000000D0H   SFRSYM    DATA     BIT       P
      000000BDH   SFRSYM    DATA     BYTE      TIM0_CCR3H
      000000BFH   SFRSYM    DATA     BYTE      TIM0_CCR4H
      000000C8H.2 SFRSYM    DATA     BIT       PTIM230
      000000EBH   SFRSYM    DATA     BYTE      PI_EKH
      00000098H.5 SFRSYM    DATA     BIT       SM2
      000000B6H   SFRSYM    DATA     BYTE      TIM0_CCR1L
      000000B1H   SFRSYM    DATA     BYTE      TIM0_SR1
      000000C8H.3 SFRSYM    DATA     BIT       PTIM231
      000000BAH   SFRSYM    DATA     BYTE      TIM0_CCR2L
      000000BCH   SFRSYM    DATA     BYTE      TIM0_CCR3L
      000000BEH   SFRSYM    DATA     BYTE      TIM0_CCR4L
      000000D8H.6 SFRSYM    DATA     BIT       PMCD0
LX51 LINKER/LOCATER V4.66.1.0                                                         03/30/2017  09:01:59  PAGE 35


      000000C8H.4 SFRSYM    DATA     BIT       PTIM450
      000000D0H.3 SFRSYM    DATA     BIT       RS0
      000000DDH   SFRSYM    DATA     BYTE      LPF_KH
      000000F3H   SFRSYM    DATA     BYTE      PI_KIH
      000000EAH   SFRSYM    DATA     BYTE      PI_EKL
      000000E8H   SFRSYM    DATA     BYTE      FOC_SET0
      000000D8H.7 SFRSYM    DATA     BIT       PMCD1
      000000C8H.5 SFRSYM    DATA     BIT       PTIM451
      000000D0H.4 SFRSYM    DATA     BIT       RS1
      000000E9H   SFRSYM    DATA     BYTE      FOC_SET1
      000000B8H.6 SFRSYM    DATA     BIT       PFOC0
      000000DCH   SFRSYM    DATA     BYTE      LPF_KL
      000000F2H   SFRSYM    DATA     BYTE      PI_KIL
      000000B8H.7 SFRSYM    DATA     BIT       PFOC1
      000000ADH   SFRSYM    DATA     BYTE      TIM2_DRH
      000000B9H   SFRSYM    DATA     BYTE      TIM0_IER
      00000083H   SFRSYM    DATA     BYTE      DPH
      000000EFH   SFRSYM    DATA     BYTE      PI_KPH
      000000A5H   SFRSYM    DATA     BYTE      TIM3_DRH
      00000095H   SFRSYM    DATA     BYTE      TIM4_DRH
      0000008DH   SFRSYM    DATA     BYTE      TIM5_DRH
      000000ACH   SFRSYM    DATA     BYTE      TIM2_DRL
      00000082H   SFRSYM    DATA     BYTE      DPL
      000000EEH   SFRSYM    DATA     BYTE      PI_KPL
      000000A4H   SFRSYM    DATA     BYTE      TIM3_DRL
      000000F8H.7 SFRSYM    DATA     BIT       MOE
      000000C0H.6 SFRSYM    DATA     BIT       PCMP0
      000000EDH   SFRSYM    DATA     BYTE      PI_UKH
      00000094H   SFRSYM    DATA     BYTE      TIM4_DRL
      000000C0H.7 SFRSYM    DATA     BIT       PCMP1
      000000DFH   SFRSYM    DATA     BYTE      LPF_XH
      0000008CH   SFRSYM    DATA     BYTE      TIM5_DRL
      000000AEH   SFRSYM    DATA     WORD      TIM2_ARR
      000000A8H.5 SFRSYM    DATA     BIT       MCDIE
      000000C9H   SFRSYM    DATA     BYTE      RSTSRC
      000000E7H   SFRSYM    DATA     BYTE      LPF_YH
      000000A6H   SFRSYM    DATA     WORD      TIM3_ARR
      00000088H.6 SFRSYM    DATA     BIT       MCDIF
      00000098H.4 SFRSYM    DATA     BIT       REN
      00000096H   SFRSYM    DATA     WORD      TIM4_ARR
      000000ECH   SFRSYM    DATA     BYTE      PI_UKL
      000000D7H   SFRSYM    DATA     BYTE      CMP_SR
      0000008EH   SFRSYM    DATA     WORD      TIM5_ARR
      000000DEH   SFRSYM    DATA     BYTE      LPF_XL
      000000E6H   SFRSYM    DATA     BYTE      LPF_YL
      000000C8H   SFRSYM    DATA     BIT       PRTC0
      000000C8H.1 SFRSYM    DATA     BIT       PRTC1
      000000E8H.7 SFRSYM    DATA     BIT       FOCEN
      000000C8H.6 SFRSYM    DATA     BIT       PTSD0
      000000D8H.4 SFRSYM    DATA     BIT       PSPI0
      000000C8H.7 SFRSYM    DATA     BIT       PTSD1
      000000D8H.5 SFRSYM    DATA     BIT       PSPI1
      0000009BH   SFRSYM    DATA     BYTE      UT_BAUDH
      000000E4H   SFRSYM    DATA     WORD      SV_ANGLE
      000000B5H   SFRSYM    DATA     BYTE      TIM2_ADTRH
      0000009AH   SFRSYM    DATA     BYTE      UT_BAUDL
      000000FCH   SFRSYM    DATA     BYTE      P0_OE
      000000FDH   SFRSYM    DATA     BYTE      P1_OE
      000000D0H.5 SFRSYM    DATA     BIT       F0
      000000B4H   SFRSYM    DATA     BYTE      TIM2_ADTRL
      000000FEH   SFRSYM    DATA     BYTE      P2_OE
      000000D0H.1 SFRSYM    DATA     BIT       F1
      00000080H   SFRSYM    DATA     BIT       GP00
      000000FFH   SFRSYM    DATA     BYTE      P3_OE
      00000090H   SFRSYM    DATA     BIT       GP10
LX51 LINKER/LOCATER V4.66.1.0                                                         03/30/2017  09:01:59  PAGE 36


      00000080H.1 SFRSYM    DATA     BIT       GP01
      000000A8H.6 SFRSYM    DATA     BIT       RTCIE
      000000A0H   SFRSYM    DATA     BIT       GP20
      00000090H.1 SFRSYM    DATA     BIT       GP11
      00000080H.2 SFRSYM    DATA     BIT       GP02
      000000E3H   SFRSYM    DATA     BYTE      SV_USH
      000000B0H   SFRSYM    DATA     BIT       GP30
      000000A0H.1 SFRSYM    DATA     BIT       GP21
      00000090H.2 SFRSYM    DATA     BIT       GP12
      00000080H.3 SFRSYM    DATA     BIT       GP03
      000000B8H   SFRSYM    DATA     BIT       PLVW0
      000000A8H.1 SFRSYM    DATA     BIT       TSDIE
      000000D0H   SFRSYM    DATA     BYTE      PSW
      000000B0H.1 SFRSYM    DATA     BIT       GP31
      000000A0H.2 SFRSYM    DATA     BIT       GP22
      00000090H.3 SFRSYM    DATA     BIT       GP13
      00000080H.4 SFRSYM    DATA     BIT       GP04
      000000B8H.1 SFRSYM    DATA     BIT       PLVW1
      000000A8H.3 SFRSYM    DATA     BIT       SPIIE
      00000088H.5 SFRSYM    DATA     BIT       TSDIF
      000000B0H.2 SFRSYM    DATA     BIT       GP32
      000000A0H.3 SFRSYM    DATA     BIT       GP23
      00000090H.4 SFRSYM    DATA     BIT       GP14
      00000080H.5 SFRSYM    DATA     BIT       GP05
      00000084H   SFRSYM    DATA     BYTE      FLKEY
      000000B3H   SFRSYM    DATA     BYTE      TIM2_CMTRH
      000000B0H.3 SFRSYM    DATA     BIT       GP33
      000000A0H.4 SFRSYM    DATA     BIT       GP24
      00000090H.5 SFRSYM    DATA     BIT       GP15
      00000080H.6 SFRSYM    DATA     BIT       GP06
      00000088H   SFRSYM    DATA     BIT       IT00

      010005F0H   BLOCK     CODE     ---       LVL=0
      010005F0H   LINE      CODE     ---       #26
      010005F0H   LINE      CODE     ---       #27
      010005F0H   LINE      CODE     ---       #34
      010005F7H   LINE      CODE     ---       #35
      010005FBH   LINE      CODE     ---       #36
      01000602H   LINE      CODE     ---       #46
      01000606H   LINE      CODE     ---       #47
      0100060AH   LINE      CODE     ---       #54
      01000611H   LINE      CODE     ---       #55
      01000618H   LINE      CODE     ---       #57
      0100061FH   LINE      CODE     ---       #58
      01000626H   LINE      CODE     ---       #60
      0100062DH   LINE      CODE     ---       #61
      01000634H   LINE      CODE     ---       #65
      0100063AH   LINE      CODE     ---       #66
      0100063EH   LINE      CODE     ---       #74
      01000645H   LINE      CODE     ---       #75
      01000649H   LINE      CODE     ---       #76
      01000650H   LINE      CODE     ---       #77
      01000654H   LINE      CODE     ---       #78
      01000656H   LINE      CODE     ---       #79
      01000658H   LINE      CODE     ---       #80
      0100065AH   LINE      CODE     ---       #83
      ---         BLOCKEND  ---      ---       LVL=0

      010004D6H   BLOCK     CODE     ---       LVL=0
      010004D6H   LINE      CODE     ---       #92
      010004D6H   LINE      CODE     ---       #93
      010004D6H   LINE      CODE     ---       #95
      010004DDH   LINE      CODE     ---       #96
      010004E1H   LINE      CODE     ---       #97
      010004E5H   LINE      CODE     ---       #98
LX51 LINKER/LOCATER V4.66.1.0                                                         03/30/2017  09:01:59  PAGE 37


      010004E9H   LINE      CODE     ---       #99
      010004EDH   LINE      CODE     ---       #100
      010004F1H   LINE      CODE     ---       #101
      010004F5H   LINE      CODE     ---       #102
      010004F9H   LINE      CODE     ---       #103
      010004FDH   LINE      CODE     ---       #104
      01000501H   LINE      CODE     ---       #105
      01000509H   LINE      CODE     ---       #106
      01000513H   LINE      CODE     ---       #107
      0100051DH   LINE      CODE     ---       #108
      01000527H   LINE      CODE     ---       #109
      01000531H   LINE      CODE     ---       #110
      0100053BH   LINE      CODE     ---       #111
      01000545H   LINE      CODE     ---       #112
      0100054FH   LINE      CODE     ---       #113
      01000559H   LINE      CODE     ---       #114
      01000563H   LINE      CODE     ---       #116
      ---         BLOCKEND  ---      ---       LVL=0

      0100065DH   BLOCK     CODE     ---       LVL=0
      0100065DH   LINE      CODE     ---       #124
      0100065DH   LINE      CODE     ---       #125
      0100065DH   LINE      CODE     ---       #126
      0100067CH   LINE      CODE     ---       #127
      0100069BH   LINE      CODE     ---       #128
      ---         BLOCKEND  ---      ---       LVL=0

      ---         MODULE    ---      ---       WDTINIT
      0100096DH   PUBLIC    CODE     ---       WatchDogRefresh
      00000020H.2 PUBLIC    BIT      BIT       ?_WatchDogConfig?BIT
      01000712H   PUBLIC    CODE     ---       _WatchDogConfig
      01000961H   PUBLIC    CODE     ---       WDT_INTI
      000000E2H   SFRSYM    DATA     BYTE      SV_USL
      000000ABH   SFRSYM    DATA     BYTE      TIM2_CNTRH
      000000B0H.4 SFRSYM    DATA     BIT       GP34
      000000A0H.5 SFRSYM    DATA     BIT       GP25
      00000090H.6 SFRSYM    DATA     BIT       GP16
      00000080H.7 SFRSYM    DATA     BIT       GP07
      00000088H.1 SFRSYM    DATA     BIT       IT01
      00000088H.3 SFRSYM    DATA     BIT       IT10
      000000F6H   SFRSYM    DATA     WORD      PI_UKMIN
      000000C2H   SFRSYM    DATA     WORD      MD_MA
      000000A3H   SFRSYM    DATA     BYTE      TIM3_CNTRH
      000000B0H.5 SFRSYM    DATA     BIT       GP35
      000000A0H.6 SFRSYM    DATA     BIT       GP26
      00000090H.7 SFRSYM    DATA     BIT       GP17
      00000080H   SFRSYM    DATA     BYTE      P0
      00000088H.4 SFRSYM    DATA     BIT       IT11
      000000CAH   SFRSYM    DATA     WORD      MD_MB
      00000093H   SFRSYM    DATA     BYTE      TIM4_CNTRH
      000000B0H.6 SFRSYM    DATA     BIT       GP36
      000000A0H.7 SFRSYM    DATA     BIT       GP27
      00000090H   SFRSYM    DATA     BYTE      P1
      000000D9H   SFRSYM    DATA     BYTE      EVT_FILT
      000000F4H   SFRSYM    DATA     WORD      PI_UKMAX
      0000008BH   SFRSYM    DATA     BYTE      TIM5_CNTRH
      000000B2H   SFRSYM    DATA     BYTE      TIM2_CMTRL
      000000B0H.7 SFRSYM    DATA     BIT       GP37
      000000A0H   SFRSYM    DATA     BYTE      P2
      000000AAH   SFRSYM    DATA     BYTE      TIM2_CNTRL
      000000B0H   SFRSYM    DATA     BYTE      P3
      000000A2H   SFRSYM    DATA     BYTE      TIM3_CNTRL
      000000D0H.6 SFRSYM    DATA     BIT       AC
      00000092H   SFRSYM    DATA     BYTE      TIM4_CNTRL
      0000008AH   SFRSYM    DATA     BYTE      TIM5_CNTRL
LX51 LINKER/LOCATER V4.66.1.0                                                         03/30/2017  09:01:59  PAGE 38


      000000B6H   SFRSYM    DATA     WORD      TIM0_CCR1
      000000A8H.7 SFRSYM    DATA     BIT       EA
      000000D5H   SFRSYM    DATA     BYTE      CMP_CR0
      000000BAH   SFRSYM    DATA     WORD      TIM0_CCR2
      000000D6H   SFRSYM    DATA     BYTE      CMP_CR1
      000000BCH   SFRSYM    DATA     WORD      TIM0_CCR3
      00000085H   SFRSYM    DATA     BYTE      PSCTL
      000000DAH   SFRSYM    DATA     BYTE      CMP_CR2
      000000BEH   SFRSYM    DATA     WORD      TIM0_CCR4
      000000B8H.2 SFRSYM    DATA     BIT       PX00
      000000EAH   SFRSYM    DATA     WORD      PI_EK
      000000F8H   SFRSYM    DATA     BIT       OISUH
      000000B8H.3 SFRSYM    DATA     BIT       PX01
      000000B8H.4 SFRSYM    DATA     BIT       PX10
      000000F8H.2 SFRSYM    DATA     BIT       OISVH
      000000B8H.5 SFRSYM    DATA     BIT       PX11
      000000F8H.4 SFRSYM    DATA     BIT       OISWH
      000000DCH   SFRSYM    DATA     WORD      LPF_K
      000000F2H   SFRSYM    DATA     WORD      PI_KI
      000000F8H.1 SFRSYM    DATA     BIT       OISUL
      000000A8H   SFRSYM    DATA     BYTE      IE
      000000F8H.3 SFRSYM    DATA     BIT       OISVL
      000000F8H.5 SFRSYM    DATA     BIT       OISWL
      000000D1H   SFRSYM    DATA     BYTE      P1IE
      00000098H.6 SFRSYM    DATA     BIT       MOD0
      000000D3H   SFRSYM    DATA     BYTE      P2IE
      000000D2H   SFRSYM    DATA     BYTE      P1IF
      000000F9H   SFRSYM    DATA     BYTE      PL_CR
      00000098H.7 SFRSYM    DATA     BIT       MOD1
      000000D4H   SFRSYM    DATA     BYTE      P2IF
      000000ACH   SFRSYM    DATA     WORD      TIM2_DR
      00000082H   SFRSYM    DATA     WORD      DP
      000000EEH   SFRSYM    DATA     WORD      PI_KP
      000000A4H   SFRSYM    DATA     WORD      TIM3_DR
      00000094H   SFRSYM    DATA     WORD      TIM4_DR
      0000008CH   SFRSYM    DATA     WORD      TIM5_DR
      000000F1H   SFRSYM    DATA     BYTE      OSC_CFG
      000000C1H   SFRSYM    DATA     BYTE      MD_MODE
      000000ECH   SFRSYM    DATA     WORD      PI_UK
      000000DEH   SFRSYM    DATA     WORD      LPF_X
      00000098H   SFRSYM    DATA     BIT       RI
      000000E6H   SFRSYM    DATA     WORD      LPF_Y
      000000C0H   SFRSYM    DATA     BIT       PTIM00
      000000D0H.7 SFRSYM    DATA     BIT       CY
      00000098H.1 SFRSYM    DATA     BIT       TI
      000000C0H.1 SFRSYM    DATA     BIT       PTIM01
      000000C0H.2 SFRSYM    DATA     BIT       PTIM10
      000000C0H.3 SFRSYM    DATA     BIT       PTIM11
      000000E1H   SFRSYM    DATA     BYTE      SV_CR
      00000098H   SFRSYM    DATA     BYTE      UT_CR
      00000099H   SFRSYM    DATA     BYTE      UT_DR
      000000F8H.6 SFRSYM    DATA     BIT       OIS4
      00000081H   SFRSYM    DATA     BYTE      SP
      000000D0H.2 SFRSYM    DATA     BIT       OV
      000000C4H   SFRSYM    DATA     BYTE      MD_DA0
      0000009AH   SFRSYM    DATA     WORD      UT_BAUD
      000000CCH   SFRSYM    DATA     BYTE      MD_DB0
      000000C5H   SFRSYM    DATA     BYTE      MD_DA1
      000000CDH   SFRSYM    DATA     BYTE      MD_DB1
      000000C6H   SFRSYM    DATA     BYTE      MD_DA2
      000000CEH   SFRSYM    DATA     BYTE      MD_DB2
      000000C7H   SFRSYM    DATA     BYTE      MD_DA3
      000000B4H   SFRSYM    DATA     WORD      TIM2_ADTR
      000000CFH   SFRSYM    DATA     BYTE      MD_DB3
      000000AFH   SFRSYM    DATA     BYTE      TIM2_ARRH
LX51 LINKER/LOCATER V4.66.1.0                                                         03/30/2017  09:01:59  PAGE 39


      000000A7H   SFRSYM    DATA     BYTE      TIM3_ARRH
      00000097H   SFRSYM    DATA     BYTE      TIM4_ARRH
      0000008FH   SFRSYM    DATA     BYTE      TIM5_ARRH
      000000AEH   SFRSYM    DATA     BYTE      TIM2_ARRL
      000000A6H   SFRSYM    DATA     BYTE      TIM3_ARRL
      00000087H   SFRSYM    DATA     BYTE      PCON
      000000E2H   SFRSYM    DATA     WORD      SV_US
      00000096H   SFRSYM    DATA     BYTE      TIM4_ARRL
      0000008EH   SFRSYM    DATA     BYTE      TIM5_ARRL
      000000B2H   SFRSYM    DATA     WORD      TIM2_CMTR
      00000088H   SFRSYM    DATA     BYTE      TCON
      000000AAH   SFRSYM    DATA     WORD      TIM2_CNTR
      000000A2H   SFRSYM    DATA     WORD      TIM3_CNTR
      00000092H   SFRSYM    DATA     WORD      TIM4_CNTR
      0000008AH   SFRSYM    DATA     WORD      TIM5_CNTR
      00000086H   SFRSYM    DATA     BYTE      CFGKEY
      000000E5H   SFRSYM    DATA     BYTE      SV_ANGLEH
      000000D8H   SFRSYM    DATA     BIT       PUART0
      000000E4H   SFRSYM    DATA     BYTE      SV_ANGLEL
      000000C6H   SFRSYM    DATA     WORD      MD_DAH
      000000D8H.1 SFRSYM    DATA     BIT       PUART1
      000000D8H.2 SFRSYM    DATA     BIT       PI2C0
      00000088H.2 SFRSYM    DATA     BIT       IF0
      000000CEH   SFRSYM    DATA     WORD      MD_DBH
      000000D8H.3 SFRSYM    DATA     BIT       PI2C1
      000000F0H   SFRSYM    DATA     BYTE      B
      000000C4H   SFRSYM    DATA     WORD      MD_DAL
      000000A1H   SFRSYM    DATA     BYTE      TIM2_CR0
      000000CCH   SFRSYM    DATA     WORD      MD_DBL
      0000009CH   SFRSYM    DATA     BYTE      TIM3_CR0
      000000A9H   SFRSYM    DATA     BYTE      TIM2_CR1
      0000009EH   SFRSYM    DATA     BYTE      TIM4_CR0
      0000009DH   SFRSYM    DATA     BYTE      TIM3_CR1
      00000089H   SFRSYM    DATA     BYTE      TIM5_CR0
      0000009FH   SFRSYM    DATA     BYTE      TIM4_CR1
      000000F8H   SFRSYM    DATA     BYTE      DRV_OUT
      00000091H   SFRSYM    DATA     BYTE      TIM5_CR1
      000000E0H   SFRSYM    DATA     BYTE      ACC
      000000F7H   SFRSYM    DATA     BYTE      PI_UKMINH
      000000C3H   SFRSYM    DATA     BYTE      MD_MAH
      000000A8H.4 SFRSYM    DATA     BIT       ES0
      000000DBH   SFRSYM    DATA     BYTE      LVSR
      000000CBH   SFRSYM    DATA     BYTE      MD_MBH
      000000C0H.4 SFRSYM    DATA     BIT       PADC0
      000000B8H   SFRSYM    DATA     BYTE      IP0
      000000F5H   SFRSYM    DATA     BYTE      PI_UKMAXH
      000000C0H.5 SFRSYM    DATA     BIT       PADC1
      000000C0H   SFRSYM    DATA     BYTE      IP1
      000000C8H   SFRSYM    DATA     BYTE      IP2
      000000F6H   SFRSYM    DATA     BYTE      PI_UKMINL
      000000C2H   SFRSYM    DATA     BYTE      MD_MAL
      00000098H.2 SFRSYM    DATA     BIT       RB8
      000000D8H   SFRSYM    DATA     BYTE      IP3
      000000CAH   SFRSYM    DATA     BYTE      MD_MBL
      000000A8H   SFRSYM    DATA     BIT       EX0
      000000F4H   SFRSYM    DATA     BYTE      PI_UKMAXL
      00000098H.3 SFRSYM    DATA     BIT       TB8
      000000B7H   SFRSYM    DATA     BYTE      TIM0_CCR1H
      000000A8H.2 SFRSYM    DATA     BIT       EX1
      000000BBH   SFRSYM    DATA     BYTE      TIM0_CCR2H
      000000D0H   SFRSYM    DATA     BIT       P
      000000BDH   SFRSYM    DATA     BYTE      TIM0_CCR3H
      000000BFH   SFRSYM    DATA     BYTE      TIM0_CCR4H
      000000C8H.2 SFRSYM    DATA     BIT       PTIM230
      000000EBH   SFRSYM    DATA     BYTE      PI_EKH
LX51 LINKER/LOCATER V4.66.1.0                                                         03/30/2017  09:01:59  PAGE 40


      00000098H.5 SFRSYM    DATA     BIT       SM2
      000000B6H   SFRSYM    DATA     BYTE      TIM0_CCR1L
      000000B1H   SFRSYM    DATA     BYTE      TIM0_SR1
      000000C8H.3 SFRSYM    DATA     BIT       PTIM231
      000000BAH   SFRSYM    DATA     BYTE      TIM0_CCR2L
      000000BCH   SFRSYM    DATA     BYTE      TIM0_CCR3L
      000000BEH   SFRSYM    DATA     BYTE      TIM0_CCR4L
      000000D8H.6 SFRSYM    DATA     BIT       PMCD0
      000000C8H.4 SFRSYM    DATA     BIT       PTIM450
      000000D0H.3 SFRSYM    DATA     BIT       RS0
      000000DDH   SFRSYM    DATA     BYTE      LPF_KH
      000000F3H   SFRSYM    DATA     BYTE      PI_KIH
      000000EAH   SFRSYM    DATA     BYTE      PI_EKL
      000000E8H   SFRSYM    DATA     BYTE      FOC_SET0
      000000D8H.7 SFRSYM    DATA     BIT       PMCD1
      000000C8H.5 SFRSYM    DATA     BIT       PTIM451
      000000D0H.4 SFRSYM    DATA     BIT       RS1
      000000E9H   SFRSYM    DATA     BYTE      FOC_SET1
      000000B8H.6 SFRSYM    DATA     BIT       PFOC0
      000000DCH   SFRSYM    DATA     BYTE      LPF_KL
      000000F2H   SFRSYM    DATA     BYTE      PI_KIL
      000000B8H.7 SFRSYM    DATA     BIT       PFOC1
      000000ADH   SFRSYM    DATA     BYTE      TIM2_DRH
      000000B9H   SFRSYM    DATA     BYTE      TIM0_IER
      00000083H   SFRSYM    DATA     BYTE      DPH
      000000EFH   SFRSYM    DATA     BYTE      PI_KPH
      000000A5H   SFRSYM    DATA     BYTE      TIM3_DRH
      00000095H   SFRSYM    DATA     BYTE      TIM4_DRH
      0000008DH   SFRSYM    DATA     BYTE      TIM5_DRH
      000000ACH   SFRSYM    DATA     BYTE      TIM2_DRL
      00000082H   SFRSYM    DATA     BYTE      DPL
      000000EEH   SFRSYM    DATA     BYTE      PI_KPL
      000000A4H   SFRSYM    DATA     BYTE      TIM3_DRL
      000000F8H.7 SFRSYM    DATA     BIT       MOE
      000000C0H.6 SFRSYM    DATA     BIT       PCMP0
      000000EDH   SFRSYM    DATA     BYTE      PI_UKH
      00000094H   SFRSYM    DATA     BYTE      TIM4_DRL
      000000C0H.7 SFRSYM    DATA     BIT       PCMP1
      000000DFH   SFRSYM    DATA     BYTE      LPF_XH
      0000008CH   SFRSYM    DATA     BYTE      TIM5_DRL
      000000AEH   SFRSYM    DATA     WORD      TIM2_ARR
      000000A8H.5 SFRSYM    DATA     BIT       MCDIE
      000000C9H   SFRSYM    DATA     BYTE      RSTSRC
      000000E7H   SFRSYM    DATA     BYTE      LPF_YH
      000000A6H   SFRSYM    DATA     WORD      TIM3_ARR
      00000088H.6 SFRSYM    DATA     BIT       MCDIF
      00000098H.4 SFRSYM    DATA     BIT       REN
      00000096H   SFRSYM    DATA     WORD      TIM4_ARR
      000000ECH   SFRSYM    DATA     BYTE      PI_UKL
      000000D7H   SFRSYM    DATA     BYTE      CMP_SR
      0000008EH   SFRSYM    DATA     WORD      TIM5_ARR
      000000DEH   SFRSYM    DATA     BYTE      LPF_XL
      000000E6H   SFRSYM    DATA     BYTE      LPF_YL
      000000C8H   SFRSYM    DATA     BIT       PRTC0
      000000C8H.1 SFRSYM    DATA     BIT       PRTC1
      000000E8H.7 SFRSYM    DATA     BIT       FOCEN
      000000C8H.6 SFRSYM    DATA     BIT       PTSD0
      000000D8H.4 SFRSYM    DATA     BIT       PSPI0
      000000C8H.7 SFRSYM    DATA     BIT       PTSD1
      000000D8H.5 SFRSYM    DATA     BIT       PSPI1
      0000009BH   SFRSYM    DATA     BYTE      UT_BAUDH
      000000E4H   SFRSYM    DATA     WORD      SV_ANGLE
      000000B5H   SFRSYM    DATA     BYTE      TIM2_ADTRH
      0000009AH   SFRSYM    DATA     BYTE      UT_BAUDL
      000000FCH   SFRSYM    DATA     BYTE      P0_OE
LX51 LINKER/LOCATER V4.66.1.0                                                         03/30/2017  09:01:59  PAGE 41


      000000FDH   SFRSYM    DATA     BYTE      P1_OE
      000000D0H.5 SFRSYM    DATA     BIT       F0
      000000B4H   SFRSYM    DATA     BYTE      TIM2_ADTRL
      000000FEH   SFRSYM    DATA     BYTE      P2_OE
      000000D0H.1 SFRSYM    DATA     BIT       F1
      00000080H   SFRSYM    DATA     BIT       GP00
      000000FFH   SFRSYM    DATA     BYTE      P3_OE
      00000090H   SFRSYM    DATA     BIT       GP10
      00000080H.1 SFRSYM    DATA     BIT       GP01
      000000A8H.6 SFRSYM    DATA     BIT       RTCIE
      000000A0H   SFRSYM    DATA     BIT       GP20
      00000090H.1 SFRSYM    DATA     BIT       GP11
      00000080H.2 SFRSYM    DATA     BIT       GP02
      000000E3H   SFRSYM    DATA     BYTE      SV_USH
      000000B0H   SFRSYM    DATA     BIT       GP30
      000000A0H.1 SFRSYM    DATA     BIT       GP21
      00000090H.2 SFRSYM    DATA     BIT       GP12
      00000080H.3 SFRSYM    DATA     BIT       GP03
      000000B8H   SFRSYM    DATA     BIT       PLVW0
      000000A8H.1 SFRSYM    DATA     BIT       TSDIE
      000000D0H   SFRSYM    DATA     BYTE      PSW
      000000B0H.1 SFRSYM    DATA     BIT       GP31
      000000A0H.2 SFRSYM    DATA     BIT       GP22
      00000090H.3 SFRSYM    DATA     BIT       GP13
      00000080H.4 SFRSYM    DATA     BIT       GP04
      000000B8H.1 SFRSYM    DATA     BIT       PLVW1
      000000A8H.3 SFRSYM    DATA     BIT       SPIIE
      00000088H.5 SFRSYM    DATA     BIT       TSDIF
      000000B0H.2 SFRSYM    DATA     BIT       GP32
      000000A0H.3 SFRSYM    DATA     BIT       GP23
      00000090H.4 SFRSYM    DATA     BIT       GP14
      00000080H.5 SFRSYM    DATA     BIT       GP05
      00000084H   SFRSYM    DATA     BYTE      FLKEY
      000000B3H   SFRSYM    DATA     BYTE      TIM2_CMTRH
      000000B0H.3 SFRSYM    DATA     BIT       GP33
      000000A0H.4 SFRSYM    DATA     BIT       GP24
      00000090H.5 SFRSYM    DATA     BIT       GP15
      00000080H.6 SFRSYM    DATA     BIT       GP06
      00000088H   SFRSYM    DATA     BIT       IT00

      01000961H   BLOCK     CODE     ---       LVL=0
      01000961H   LINE      CODE     ---       #29
      01000961H   LINE      CODE     ---       #30
      01000961H   LINE      CODE     ---       #31
      01000968H   LINE      CODE     ---       #32
      0100096CH   LINE      CODE     ---       #33
      ---         BLOCKEND  ---      ---       LVL=0

      01000712H   BLOCK     CODE     ---       LVL=0
      00000006H   SYMBOL    DATA     WORD      Value
      00000020H.2 SYMBOL    BIT      BIT       Status
      01000712H   LINE      CODE     ---       #42
      01000712H   LINE      CODE     ---       #43
      01000712H   LINE      CODE     ---       #44
      01000715H   LINE      CODE     ---       #45
      01000718H   LINE      CODE     ---       #46
      01000727H   LINE      CODE     ---       #47
      01000736H   LINE      CODE     ---       #48
      01000739H   LINE      CODE     ---       #49
      01000755H   LINE      CODE     ---       #50
      0100075CH   LINE      CODE     ---       #51
      01000760H   LINE      CODE     ---       #52
      ---         BLOCKEND  ---      ---       LVL=0

      0100096DH   BLOCK     CODE     ---       LVL=0
LX51 LINKER/LOCATER V4.66.1.0                                                         03/30/2017  09:01:59  PAGE 42


      0100096DH   LINE      CODE     ---       #61
      0100096DH   LINE      CODE     ---       #62
      0100096DH   LINE      CODE     ---       #63
      01000974H   LINE      CODE     ---       #64
      ---         BLOCKEND  ---      ---       LVL=0

      ---         MODULE    ---      ---       GPIOINIT
      010006BAH   PUBLIC    CODE     ---       GPIOInit
      000000E2H   SFRSYM    DATA     BYTE      SV_USL
      000000ABH   SFRSYM    DATA     BYTE      TIM2_CNTRH
      000000B0H.4 SFRSYM    DATA     BIT       GP34
      000000A0H.5 SFRSYM    DATA     BIT       GP25
      00000090H.6 SFRSYM    DATA     BIT       GP16
      00000080H.7 SFRSYM    DATA     BIT       GP07
      00000088H.1 SFRSYM    DATA     BIT       IT01
      00000088H.3 SFRSYM    DATA     BIT       IT10
      000000F6H   SFRSYM    DATA     WORD      PI_UKMIN
      000000C2H   SFRSYM    DATA     WORD      MD_MA
      000000A3H   SFRSYM    DATA     BYTE      TIM3_CNTRH
      000000B0H.5 SFRSYM    DATA     BIT       GP35
      000000A0H.6 SFRSYM    DATA     BIT       GP26
      00000090H.7 SFRSYM    DATA     BIT       GP17
      00000080H   SFRSYM    DATA     BYTE      P0
      00000088H.4 SFRSYM    DATA     BIT       IT11
      000000CAH   SFRSYM    DATA     WORD      MD_MB
      00000093H   SFRSYM    DATA     BYTE      TIM4_CNTRH
      000000B0H.6 SFRSYM    DATA     BIT       GP36
      000000A0H.7 SFRSYM    DATA     BIT       GP27
      00000090H   SFRSYM    DATA     BYTE      P1
      000000D9H   SFRSYM    DATA     BYTE      EVT_FILT
      000000F4H   SFRSYM    DATA     WORD      PI_UKMAX
      0000008BH   SFRSYM    DATA     BYTE      TIM5_CNTRH
      000000B2H   SFRSYM    DATA     BYTE      TIM2_CMTRL
      000000B0H.7 SFRSYM    DATA     BIT       GP37
      000000A0H   SFRSYM    DATA     BYTE      P2
      000000AAH   SFRSYM    DATA     BYTE      TIM2_CNTRL
      000000B0H   SFRSYM    DATA     BYTE      P3
      000000A2H   SFRSYM    DATA     BYTE      TIM3_CNTRL
      000000D0H.6 SFRSYM    DATA     BIT       AC
      00000092H   SFRSYM    DATA     BYTE      TIM4_CNTRL
      0000008AH   SFRSYM    DATA     BYTE      TIM5_CNTRL
      000000B6H   SFRSYM    DATA     WORD      TIM0_CCR1
      000000A8H.7 SFRSYM    DATA     BIT       EA
      000000D5H   SFRSYM    DATA     BYTE      CMP_CR0
      000000BAH   SFRSYM    DATA     WORD      TIM0_CCR2
      000000D6H   SFRSYM    DATA     BYTE      CMP_CR1
      000000BCH   SFRSYM    DATA     WORD      TIM0_CCR3
      00000085H   SFRSYM    DATA     BYTE      PSCTL
      000000DAH   SFRSYM    DATA     BYTE      CMP_CR2
      000000BEH   SFRSYM    DATA     WORD      TIM0_CCR4
      000000B8H.2 SFRSYM    DATA     BIT       PX00
      000000EAH   SFRSYM    DATA     WORD      PI_EK
      000000F8H   SFRSYM    DATA     BIT       OISUH
      000000B8H.3 SFRSYM    DATA     BIT       PX01
      000000B8H.4 SFRSYM    DATA     BIT       PX10
      000000F8H.2 SFRSYM    DATA     BIT       OISVH
      000000B8H.5 SFRSYM    DATA     BIT       PX11
      000000F8H.4 SFRSYM    DATA     BIT       OISWH
      000000DCH   SFRSYM    DATA     WORD      LPF_K
      000000F2H   SFRSYM    DATA     WORD      PI_KI
      000000F8H.1 SFRSYM    DATA     BIT       OISUL
      000000A8H   SFRSYM    DATA     BYTE      IE
      000000F8H.3 SFRSYM    DATA     BIT       OISVL
      000000F8H.5 SFRSYM    DATA     BIT       OISWL
      000000D1H   SFRSYM    DATA     BYTE      P1IE
LX51 LINKER/LOCATER V4.66.1.0                                                         03/30/2017  09:01:59  PAGE 43


      00000098H.6 SFRSYM    DATA     BIT       MOD0
      000000D3H   SFRSYM    DATA     BYTE      P2IE
      000000D2H   SFRSYM    DATA     BYTE      P1IF
      000000F9H   SFRSYM    DATA     BYTE      PL_CR
      00000098H.7 SFRSYM    DATA     BIT       MOD1
      000000D4H   SFRSYM    DATA     BYTE      P2IF
      000000ACH   SFRSYM    DATA     WORD      TIM2_DR
      00000082H   SFRSYM    DATA     WORD      DP
      000000EEH   SFRSYM    DATA     WORD      PI_KP
      000000A4H   SFRSYM    DATA     WORD      TIM3_DR
      00000094H   SFRSYM    DATA     WORD      TIM4_DR
      0000008CH   SFRSYM    DATA     WORD      TIM5_DR
      000000F1H   SFRSYM    DATA     BYTE      OSC_CFG
      000000C1H   SFRSYM    DATA     BYTE      MD_MODE
      000000ECH   SFRSYM    DATA     WORD      PI_UK
      000000DEH   SFRSYM    DATA     WORD      LPF_X
      00000098H   SFRSYM    DATA     BIT       RI
      000000E6H   SFRSYM    DATA     WORD      LPF_Y
      000000C0H   SFRSYM    DATA     BIT       PTIM00
      000000D0H.7 SFRSYM    DATA     BIT       CY
      00000098H.1 SFRSYM    DATA     BIT       TI
      000000C0H.1 SFRSYM    DATA     BIT       PTIM01
      000000C0H.2 SFRSYM    DATA     BIT       PTIM10
      000000C0H.3 SFRSYM    DATA     BIT       PTIM11
      000000E1H   SFRSYM    DATA     BYTE      SV_CR
      00000098H   SFRSYM    DATA     BYTE      UT_CR
      00000099H   SFRSYM    DATA     BYTE      UT_DR
      000000F8H.6 SFRSYM    DATA     BIT       OIS4
      00000081H   SFRSYM    DATA     BYTE      SP
      000000D0H.2 SFRSYM    DATA     BIT       OV
      000000C4H   SFRSYM    DATA     BYTE      MD_DA0
      0000009AH   SFRSYM    DATA     WORD      UT_BAUD
      000000CCH   SFRSYM    DATA     BYTE      MD_DB0
      000000C5H   SFRSYM    DATA     BYTE      MD_DA1
      000000CDH   SFRSYM    DATA     BYTE      MD_DB1
      000000C6H   SFRSYM    DATA     BYTE      MD_DA2
      000000CEH   SFRSYM    DATA     BYTE      MD_DB2
      000000C7H   SFRSYM    DATA     BYTE      MD_DA3
      000000B4H   SFRSYM    DATA     WORD      TIM2_ADTR
      000000CFH   SFRSYM    DATA     BYTE      MD_DB3
      000000AFH   SFRSYM    DATA     BYTE      TIM2_ARRH
      000000A7H   SFRSYM    DATA     BYTE      TIM3_ARRH
      00000097H   SFRSYM    DATA     BYTE      TIM4_ARRH
      0000008FH   SFRSYM    DATA     BYTE      TIM5_ARRH
      000000AEH   SFRSYM    DATA     BYTE      TIM2_ARRL
      000000A6H   SFRSYM    DATA     BYTE      TIM3_ARRL
      00000087H   SFRSYM    DATA     BYTE      PCON
      000000E2H   SFRSYM    DATA     WORD      SV_US
      00000096H   SFRSYM    DATA     BYTE      TIM4_ARRL
      0000008EH   SFRSYM    DATA     BYTE      TIM5_ARRL
      000000B2H   SFRSYM    DATA     WORD      TIM2_CMTR
      00000088H   SFRSYM    DATA     BYTE      TCON
      000000AAH   SFRSYM    DATA     WORD      TIM2_CNTR
      000000A2H   SFRSYM    DATA     WORD      TIM3_CNTR
      00000092H   SFRSYM    DATA     WORD      TIM4_CNTR
      0000008AH   SFRSYM    DATA     WORD      TIM5_CNTR
      00000086H   SFRSYM    DATA     BYTE      CFGKEY
      000000E5H   SFRSYM    DATA     BYTE      SV_ANGLEH
      000000D8H   SFRSYM    DATA     BIT       PUART0
      000000E4H   SFRSYM    DATA     BYTE      SV_ANGLEL
      000000C6H   SFRSYM    DATA     WORD      MD_DAH
      000000D8H.1 SFRSYM    DATA     BIT       PUART1
      000000D8H.2 SFRSYM    DATA     BIT       PI2C0
      00000088H.2 SFRSYM    DATA     BIT       IF0
      000000CEH   SFRSYM    DATA     WORD      MD_DBH
LX51 LINKER/LOCATER V4.66.1.0                                                         03/30/2017  09:01:59  PAGE 44


      000000D8H.3 SFRSYM    DATA     BIT       PI2C1
      000000F0H   SFRSYM    DATA     BYTE      B
      000000C4H   SFRSYM    DATA     WORD      MD_DAL
      000000A1H   SFRSYM    DATA     BYTE      TIM2_CR0
      000000CCH   SFRSYM    DATA     WORD      MD_DBL
      0000009CH   SFRSYM    DATA     BYTE      TIM3_CR0
      000000A9H   SFRSYM    DATA     BYTE      TIM2_CR1
      0000009EH   SFRSYM    DATA     BYTE      TIM4_CR0
      0000009DH   SFRSYM    DATA     BYTE      TIM3_CR1
      00000089H   SFRSYM    DATA     BYTE      TIM5_CR0
      0000009FH   SFRSYM    DATA     BYTE      TIM4_CR1
      000000F8H   SFRSYM    DATA     BYTE      DRV_OUT
      00000091H   SFRSYM    DATA     BYTE      TIM5_CR1
      000000E0H   SFRSYM    DATA     BYTE      ACC
      000000F7H   SFRSYM    DATA     BYTE      PI_UKMINH
      000000C3H   SFRSYM    DATA     BYTE      MD_MAH
      000000A8H.4 SFRSYM    DATA     BIT       ES0
      000000DBH   SFRSYM    DATA     BYTE      LVSR
      000000CBH   SFRSYM    DATA     BYTE      MD_MBH
      000000C0H.4 SFRSYM    DATA     BIT       PADC0
      000000B8H   SFRSYM    DATA     BYTE      IP0
      000000F5H   SFRSYM    DATA     BYTE      PI_UKMAXH
      000000C0H.5 SFRSYM    DATA     BIT       PADC1
      000000C0H   SFRSYM    DATA     BYTE      IP1
      000000C8H   SFRSYM    DATA     BYTE      IP2
      000000F6H   SFRSYM    DATA     BYTE      PI_UKMINL
      000000C2H   SFRSYM    DATA     BYTE      MD_MAL
      00000098H.2 SFRSYM    DATA     BIT       RB8
      000000D8H   SFRSYM    DATA     BYTE      IP3
      000000CAH   SFRSYM    DATA     BYTE      MD_MBL
      000000A8H   SFRSYM    DATA     BIT       EX0
      000000F4H   SFRSYM    DATA     BYTE      PI_UKMAXL
      00000098H.3 SFRSYM    DATA     BIT       TB8
      000000B7H   SFRSYM    DATA     BYTE      TIM0_CCR1H
      000000A8H.2 SFRSYM    DATA     BIT       EX1
      000000BBH   SFRSYM    DATA     BYTE      TIM0_CCR2H
      000000D0H   SFRSYM    DATA     BIT       P
      000000BDH   SFRSYM    DATA     BYTE      TIM0_CCR3H
      000000BFH   SFRSYM    DATA     BYTE      TIM0_CCR4H
      000000C8H.2 SFRSYM    DATA     BIT       PTIM230
      000000EBH   SFRSYM    DATA     BYTE      PI_EKH
      00000098H.5 SFRSYM    DATA     BIT       SM2
      000000B6H   SFRSYM    DATA     BYTE      TIM0_CCR1L
      000000B1H   SFRSYM    DATA     BYTE      TIM0_SR1
      000000C8H.3 SFRSYM    DATA     BIT       PTIM231
      000000BAH   SFRSYM    DATA     BYTE      TIM0_CCR2L
      000000BCH   SFRSYM    DATA     BYTE      TIM0_CCR3L
      000000BEH   SFRSYM    DATA     BYTE      TIM0_CCR4L
      000000D8H.6 SFRSYM    DATA     BIT       PMCD0
      000000C8H.4 SFRSYM    DATA     BIT       PTIM450
      000000D0H.3 SFRSYM    DATA     BIT       RS0
      000000DDH   SFRSYM    DATA     BYTE      LPF_KH
      000000F3H   SFRSYM    DATA     BYTE      PI_KIH
      000000EAH   SFRSYM    DATA     BYTE      PI_EKL
      000000E8H   SFRSYM    DATA     BYTE      FOC_SET0
      000000D8H.7 SFRSYM    DATA     BIT       PMCD1
      000000C8H.5 SFRSYM    DATA     BIT       PTIM451
      000000D0H.4 SFRSYM    DATA     BIT       RS1
      000000E9H   SFRSYM    DATA     BYTE      FOC_SET1
      000000B8H.6 SFRSYM    DATA     BIT       PFOC0
      000000DCH   SFRSYM    DATA     BYTE      LPF_KL
      000000F2H   SFRSYM    DATA     BYTE      PI_KIL
      000000B8H.7 SFRSYM    DATA     BIT       PFOC1
      000000ADH   SFRSYM    DATA     BYTE      TIM2_DRH
      000000B9H   SFRSYM    DATA     BYTE      TIM0_IER
LX51 LINKER/LOCATER V4.66.1.0                                                         03/30/2017  09:01:59  PAGE 45


      00000083H   SFRSYM    DATA     BYTE      DPH
      000000EFH   SFRSYM    DATA     BYTE      PI_KPH
      000000A5H   SFRSYM    DATA     BYTE      TIM3_DRH
      00000095H   SFRSYM    DATA     BYTE      TIM4_DRH
      0000008DH   SFRSYM    DATA     BYTE      TIM5_DRH
      000000ACH   SFRSYM    DATA     BYTE      TIM2_DRL
      00000082H   SFRSYM    DATA     BYTE      DPL
      000000EEH   SFRSYM    DATA     BYTE      PI_KPL
      000000A4H   SFRSYM    DATA     BYTE      TIM3_DRL
      000000F8H.7 SFRSYM    DATA     BIT       MOE
      000000C0H.6 SFRSYM    DATA     BIT       PCMP0
      000000EDH   SFRSYM    DATA     BYTE      PI_UKH
      00000094H   SFRSYM    DATA     BYTE      TIM4_DRL
      000000C0H.7 SFRSYM    DATA     BIT       PCMP1
      000000DFH   SFRSYM    DATA     BYTE      LPF_XH
      0000008CH   SFRSYM    DATA     BYTE      TIM5_DRL
      000000AEH   SFRSYM    DATA     WORD      TIM2_ARR
      000000A8H.5 SFRSYM    DATA     BIT       MCDIE
      000000C9H   SFRSYM    DATA     BYTE      RSTSRC
      000000E7H   SFRSYM    DATA     BYTE      LPF_YH
      000000A6H   SFRSYM    DATA     WORD      TIM3_ARR
      00000088H.6 SFRSYM    DATA     BIT       MCDIF
      00000098H.4 SFRSYM    DATA     BIT       REN
      00000096H   SFRSYM    DATA     WORD      TIM4_ARR
      000000ECH   SFRSYM    DATA     BYTE      PI_UKL
      000000D7H   SFRSYM    DATA     BYTE      CMP_SR
      0000008EH   SFRSYM    DATA     WORD      TIM5_ARR
      000000DEH   SFRSYM    DATA     BYTE      LPF_XL
      000000E6H   SFRSYM    DATA     BYTE      LPF_YL
      000000C8H   SFRSYM    DATA     BIT       PRTC0
      000000C8H.1 SFRSYM    DATA     BIT       PRTC1
      000000E8H.7 SFRSYM    DATA     BIT       FOCEN
      000000C8H.6 SFRSYM    DATA     BIT       PTSD0
      000000D8H.4 SFRSYM    DATA     BIT       PSPI0
      000000C8H.7 SFRSYM    DATA     BIT       PTSD1
      000000D8H.5 SFRSYM    DATA     BIT       PSPI1
      0000009BH   SFRSYM    DATA     BYTE      UT_BAUDH
      000000E4H   SFRSYM    DATA     WORD      SV_ANGLE
      000000B5H   SFRSYM    DATA     BYTE      TIM2_ADTRH
      0000009AH   SFRSYM    DATA     BYTE      UT_BAUDL
      000000FCH   SFRSYM    DATA     BYTE      P0_OE
      000000FDH   SFRSYM    DATA     BYTE      P1_OE
      000000D0H.5 SFRSYM    DATA     BIT       F0
      000000B4H   SFRSYM    DATA     BYTE      TIM2_ADTRL
      000000FEH   SFRSYM    DATA     BYTE      P2_OE
      000000D0H.1 SFRSYM    DATA     BIT       F1
      00000080H   SFRSYM    DATA     BIT       GP00
      000000FFH   SFRSYM    DATA     BYTE      P3_OE
      00000090H   SFRSYM    DATA     BIT       GP10
      00000080H.1 SFRSYM    DATA     BIT       GP01
      000000A8H.6 SFRSYM    DATA     BIT       RTCIE
      000000A0H   SFRSYM    DATA     BIT       GP20
      00000090H.1 SFRSYM    DATA     BIT       GP11
      00000080H.2 SFRSYM    DATA     BIT       GP02
      000000E3H   SFRSYM    DATA     BYTE      SV_USH
      000000B0H   SFRSYM    DATA     BIT       GP30
      000000A0H.1 SFRSYM    DATA     BIT       GP21
      00000090H.2 SFRSYM    DATA     BIT       GP12
      00000080H.3 SFRSYM    DATA     BIT       GP03
      000000B8H   SFRSYM    DATA     BIT       PLVW0
      000000A8H.1 SFRSYM    DATA     BIT       TSDIE
      000000D0H   SFRSYM    DATA     BYTE      PSW
      000000B0H.1 SFRSYM    DATA     BIT       GP31
      000000A0H.2 SFRSYM    DATA     BIT       GP22
      00000090H.3 SFRSYM    DATA     BIT       GP13
LX51 LINKER/LOCATER V4.66.1.0                                                         03/30/2017  09:01:59  PAGE 46


      00000080H.4 SFRSYM    DATA     BIT       GP04
      000000B8H.1 SFRSYM    DATA     BIT       PLVW1
      000000A8H.3 SFRSYM    DATA     BIT       SPIIE
      00000088H.5 SFRSYM    DATA     BIT       TSDIF
      000000B0H.2 SFRSYM    DATA     BIT       GP32
      000000A0H.3 SFRSYM    DATA     BIT       GP23
      00000090H.4 SFRSYM    DATA     BIT       GP14
      00000080H.5 SFRSYM    DATA     BIT       GP05
      00000084H   SFRSYM    DATA     BYTE      FLKEY
      000000B3H   SFRSYM    DATA     BYTE      TIM2_CMTRH
      000000B0H.3 SFRSYM    DATA     BIT       GP33
      000000A0H.4 SFRSYM    DATA     BIT       GP24
      00000090H.5 SFRSYM    DATA     BIT       GP15
      00000080H.6 SFRSYM    DATA     BIT       GP06
      00000088H   SFRSYM    DATA     BIT       IT00

      010006BAH   BLOCK     CODE     ---       LVL=0
      010006BAH   LINE      CODE     ---       #22
      010006BAH   LINE      CODE     ---       #23
      010006BAH   LINE      CODE     ---       #24
      010006BDH   LINE      CODE     ---       #25
      010006C4H   LINE      CODE     ---       #27
      010006C7H   LINE      CODE     ---       #28
      010006CBH   LINE      CODE     ---       #30
      010006CEH   LINE      CODE     ---       #31
      010006D2H   LINE      CODE     ---       #33
      010006D5H   LINE      CODE     ---       #34
      010006D9H   LINE      CODE     ---       #36
      010006DCH   LINE      CODE     ---       #37
      010006E1H   LINE      CODE     ---       #38
      010006E3H   LINE      CODE     ---       #40
      010006E6H   LINE      CODE     ---       #41
      010006EAH   LINE      CODE     ---       #43
      010006EDH   LINE      CODE     ---       #44
      010006F4H   LINE      CODE     ---       #45
      010006F6H   LINE      CODE     ---       #47
      010006F9H   LINE      CODE     ---       #48
      01000700H   LINE      CODE     ---       #49
      01000707H   LINE      CODE     ---       #51
      0100070AH   LINE      CODE     ---       #52
      01000711H   LINE      CODE     ---       #55
      ---         BLOCKEND  ---      ---       LVL=0

      ---         MODULE    ---      ---       FU68XX_OSC
      00000020H.6 PUBLIC    BIT      ---       ?SYSTEMFASTCLOCKSPD2CONFIG?BIT
      010008EDH   PUBLIC    CODE     ---       SYSTEMFASTCLOCKSPD2CONFIG
      00000020H.5 PUBLIC    BIT      ---       ?SYSTEMFASTCLOCKMCDCONFIG?BIT
      010008D4H   PUBLIC    CODE     ---       SYSTEMFASTCLOCKMCDCONFIG
      00000020H.2 PUBLIC    BIT      ---       ?EXTERNALSLOWCLOCKCONFIG?BIT
      0100091EH   PUBLIC    CODE     ---       EXTERNALSLOWCLOCKCONFIG
      00000020H.2 PUBLIC    BIT      ---       ?SYSTEMFASTCLOCKCONFIG?BIT
      01000934H   PUBLIC    CODE     ---       SYSTEMFASTCLOCKCONFIG
      00000020H.4 PUBLIC    BIT      ---       ?INTERNALFASTCLOCKCONFIG?BIT
      010008B9H   PUBLIC    CODE     ---       INTERNALFASTCLOCKCONFIG
      00000020H.0 PUBLIC    BIT      ---       ?EXTERNALFASTCLOCKCONFIG?BIT
      01000826H   PUBLIC    CODE     ---       EXTERNALFASTCLOCKCONFIG
      00000000H   SYMBOL    CODE     WORD      _ICE_DUMMY_
      01000826H   BLOCK     ---      ---       LVL=1
      00000020H.0 SYMBOL    BIT      BIT       Mode
      00000020H.1 SYMBOL    BIT      BIT       Status
      01000826H   LINE      CODE     ---       #22
      01000826H   LINE      CODE     ---       #23
      01000826H   LINE      CODE     ---       #24
      0100082BH   LINE      CODE     ---       #25
      0100082BH   LINE      CODE     ---       #26
LX51 LINKER/LOCATER V4.66.1.0                                                         03/30/2017  09:01:59  PAGE 47


      0100082EH   LINE      CODE     ---       #27
      01000831H   LINE      CODE     ---       #28
      01000840H   LINE      CODE     ---       #29
      01000843H   LINE      CODE     ---       #30
      0100084EH   LINE      CODE     ---       #31
      01000851H   LINE      CODE     ---       #32
      01000858H   LINE      CODE     ---       #33
      01000858H   LINE      CODE     ---       #34
      ---         BLOCKEND  ---      ---       LVL=0
      010008B9H   BLOCK     ---      ---       LVL=1
      00000020H.4 SYMBOL    BIT      BIT       Status
      010008B9H   LINE      CODE     ---       #43
      010008B9H   LINE      CODE     ---       #44
      010008B9H   LINE      CODE     ---       #45
      010008BEH   LINE      CODE     ---       #46
      010008BEH   LINE      CODE     ---       #47
      010008C1H   LINE      CODE     ---       #48
      010008CCH   LINE      CODE     ---       #49
      010008D3H   LINE      CODE     ---       #50
      010008D3H   LINE      CODE     ---       #51
      ---         BLOCKEND  ---      ---       LVL=0
      01000934H   BLOCK     ---      ---       LVL=1
      00000020H.2 SYMBOL    BIT      BIT       Mode
      01000934H   LINE      CODE     ---       #60
      01000934H   LINE      CODE     ---       #61
      01000934H   LINE      CODE     ---       #62
      01000942H   LINE      CODE     ---       #63
      ---         BLOCKEND  ---      ---       LVL=0
      0100091EH   BLOCK     ---      ---       LVL=1
      00000020H.2 SYMBOL    BIT      BIT       Status
      0100091EH   LINE      CODE     ---       #72
      0100091EH   LINE      CODE     ---       #73
      0100091EH   LINE      CODE     ---       #74
      01000929H   LINE      CODE     ---       #75
      01000933H   LINE      CODE     ---       #76
      ---         BLOCKEND  ---      ---       LVL=0
      010008D4H   BLOCK     ---      ---       LVL=1
      00000020H.5 SYMBOL    BIT      BIT       Status
      010008D4H   LINE      CODE     ---       #85
      010008D4H   LINE      CODE     ---       #86
      010008D4H   LINE      CODE     ---       #87
      010008D7H   LINE      CODE     ---       #88
      010008DAH   LINE      CODE     ---       #89
      010008E9H   LINE      CODE     ---       #90
      010008ECH   LINE      CODE     ---       #91
      ---         BLOCKEND  ---      ---       LVL=0
      010008EDH   BLOCK     ---      ---       LVL=1
      00000020H.6 SYMBOL    BIT      BIT       Status
      010008EDH   LINE      CODE     ---       #100
      010008EDH   LINE      CODE     ---       #101
      010008EDH   LINE      CODE     ---       #102
      010008F0H   LINE      CODE     ---       #103
      010008F3H   LINE      CODE     ---       #104
      01000902H   LINE      CODE     ---       #105
      01000905H   LINE      CODE     ---       #106
      ---         BLOCKEND  ---      ---       LVL=0

      ---         MODULE    ---      ---       FU68XX_POWER
      00000020H.2 PUBLIC    BIT      ---       ?VHALFCONFIG?BIT
      0100089BH   PUBLIC    CODE     ---       VHALFCONFIG
      00000020H.2 PUBLIC    BIT      ---       ?_VREFCONFIG?BIT
      01000761H   PUBLIC    CODE     ---       _VREFCONFIG
      010007E6H   PUBLIC    CODE     ---       _LVWPOWERDOWNWARNCONFIG
      010007A6H   PUBLIC    CODE     ---       _LVRPOWERDOWNRESETCONFIG
      00000021H.0 PUBLIC    BIT      ---       ?LVDPOWERDOWNWARNIECONFIG?BIT
LX51 LINKER/LOCATER V4.66.1.0                                                         03/30/2017  09:01:59  PAGE 48


      01000952H   PUBLIC    CODE     ---       LVDPOWERDOWNWARNIECONFIG
      00000020H.7 PUBLIC    BIT      ---       ?LVDPOWERDOWNDETECTCONFIG?BIT
      01000943H   PUBLIC    CODE     ---       LVDPOWERDOWNDETECTCONFIG
      00000000H   SYMBOL    CODE     WORD      _ICE_DUMMY_
      01000943H   BLOCK     ---      ---       LVL=1
      00000020H.7 SYMBOL    BIT      BIT       Status
      01000943H   LINE      CODE     ---       #22
      01000943H   LINE      CODE     ---       #23
      01000943H   LINE      CODE     ---       #24
      01000951H   LINE      CODE     ---       #25
      ---         BLOCKEND  ---      ---       LVL=0
      01000952H   BLOCK     ---      ---       LVL=1
      00000021H.0 SYMBOL    BIT      BIT       Status
      01000952H   LINE      CODE     ---       #35
      01000952H   LINE      CODE     ---       #36
      01000952H   LINE      CODE     ---       #37
      01000960H   LINE      CODE     ---       #38
      ---         BLOCKEND  ---      ---       LVL=0
      010007A6H   BLOCK     ---      ---       LVL=1
      00000007H   SYMBOL    DATA     BYTE      Value
      010007A6H   LINE      CODE     ---       #51
      010007A6H   LINE      CODE     ---       #52
      010007A6H   LINE      CODE     ---       #53
      010007A9H   LINE      CODE     ---       #54
      010007ACH   LINE      CODE     ---       #55
      010007BAH   LINE      CODE     ---       #56
      010007BAH   LINE      CODE     ---       #57
      010007BAH   LINE      CODE     ---       #58
      010007C0H   LINE      CODE     ---       #59
      010007C0H   LINE      CODE     ---       #60
      010007C2H   LINE      CODE     ---       #61
      010007C2H   LINE      CODE     ---       #62
      010007C8H   LINE      CODE     ---       #63
      010007C8H   LINE      CODE     ---       #64
      010007CAH   LINE      CODE     ---       #65
      010007CAH   LINE      CODE     ---       #66
      010007D1H   LINE      CODE     ---       #67
      010007D5H   LINE      CODE     ---       #68
      010007D7H   LINE      CODE     ---       #69
      010007D7H   LINE      CODE     ---       #70
      010007DEH   LINE      CODE     ---       #71
      010007E2H   LINE      CODE     ---       #72
      010007E2H   LINE      CODE     ---       #73
      010007E2H   LINE      CODE     ---       #74
      010007E2H   LINE      CODE     ---       #75
      010007E2H   LINE      CODE     ---       #76
      010007E5H   LINE      CODE     ---       #77
      ---         BLOCKEND  ---      ---       LVL=0
      010007E6H   BLOCK     ---      ---       LVL=1
      00000007H   SYMBOL    DATA     BYTE      Value
      010007E6H   LINE      CODE     ---       #90
      010007E6H   LINE      CODE     ---       #91
      010007E6H   LINE      CODE     ---       #92
      010007E9H   LINE      CODE     ---       #93
      010007ECH   LINE      CODE     ---       #94
      010007FAH   LINE      CODE     ---       #95
      010007FAH   LINE      CODE     ---       #96
      010007FAH   LINE      CODE     ---       #97
      01000800H   LINE      CODE     ---       #98
      01000800H   LINE      CODE     ---       #99
      01000802H   LINE      CODE     ---       #100
      01000802H   LINE      CODE     ---       #101
      01000808H   LINE      CODE     ---       #102
      01000808H   LINE      CODE     ---       #103
      0100080AH   LINE      CODE     ---       #104
LX51 LINKER/LOCATER V4.66.1.0                                                         03/30/2017  09:01:59  PAGE 49


      0100080AH   LINE      CODE     ---       #105
      01000811H   LINE      CODE     ---       #106
      01000815H   LINE      CODE     ---       #107
      01000817H   LINE      CODE     ---       #108
      01000817H   LINE      CODE     ---       #109
      0100081EH   LINE      CODE     ---       #110
      01000822H   LINE      CODE     ---       #111
      01000822H   LINE      CODE     ---       #112
      01000822H   LINE      CODE     ---       #113
      01000822H   LINE      CODE     ---       #114
      01000822H   LINE      CODE     ---       #115
      01000825H   LINE      CODE     ---       #116
      ---         BLOCKEND  ---      ---       LVL=0
      01000761H   BLOCK     ---      ---       LVL=1
      00000007H   SYMBOL    DATA     BYTE      Value
      00000020H.2 SYMBOL    BIT      BIT       Status
      01000761H   LINE      CODE     ---       #132
      01000761H   LINE      CODE     ---       #133
      01000761H   LINE      CODE     ---       #134
      0100076FH   LINE      CODE     ---       #135
      0100076FH   LINE      CODE     ---       #136
      0100076FH   LINE      CODE     ---       #137
      01000775H   LINE      CODE     ---       #138
      01000775H   LINE      CODE     ---       #139
      01000777H   LINE      CODE     ---       #140
      01000777H   LINE      CODE     ---       #141
      0100077DH   LINE      CODE     ---       #142
      0100077DH   LINE      CODE     ---       #143
      0100077FH   LINE      CODE     ---       #144
      0100077FH   LINE      CODE     ---       #145
      01000786H   LINE      CODE     ---       #146
      0100078AH   LINE      CODE     ---       #147
      0100078CH   LINE      CODE     ---       #148
      0100078CH   LINE      CODE     ---       #149
      01000793H   LINE      CODE     ---       #150
      01000797H   LINE      CODE     ---       #151
      01000797H   LINE      CODE     ---       #152
      01000797H   LINE      CODE     ---       #153
      01000797H   LINE      CODE     ---       #154
      01000797H   LINE      CODE     ---       #155
      010007A5H   LINE      CODE     ---       #156
      ---         BLOCKEND  ---      ---       LVL=0
      0100089BH   BLOCK     ---      ---       LVL=1
      00000020H.2 SYMBOL    BIT      BIT       Mode
      00000020H.3 SYMBOL    BIT      BIT       Status
      0100089BH   LINE      CODE     ---       #167
      0100089BH   LINE      CODE     ---       #168
      0100089BH   LINE      CODE     ---       #169
      010008AAH   LINE      CODE     ---       #170
      010008B8H   LINE      CODE     ---       #171
      ---         BLOCKEND  ---      ---       LVL=0

      ---         MODULE    ---      ---       ?C?FPDIV
      01000039H   PUBLIC    CODE     ---       ?C?FPDIV

      ---         MODULE    ---      ---       ?C?FCAST
      010000E0H   PUBLIC    CODE     ---       ?C?FCASTC
      010000DBH   PUBLIC    CODE     ---       ?C?FCASTI
      010000D6H   PUBLIC    CODE     ---       ?C?FCASTL

      ---         MODULE    ---      ---       ?C?FPGETOPN
      01000114H   PUBLIC    CODE     ---       ?C?FPGETOPN2
      01000149H   PUBLIC    CODE     ---       ?C?FPNANRESULT
      01000153H   PUBLIC    CODE     ---       ?C?FPOVERFLOW
      0100012BH   PUBLIC    CODE     ---       ?C?FPRESULT
LX51 LINKER/LOCATER V4.66.1.0                                                         03/30/2017  09:01:59  PAGE 50


      0100013FH   PUBLIC    CODE     ---       ?C?FPRESULT2
      01000150H   PUBLIC    CODE     ---       ?C?FPUNDERFLOW

      ---         MODULE    ---      ---       ?C_STARTUP
      01000000H   PUBLIC    CODE     ---       ?C_STARTUP

      ---         MODULE    ---      ---       ?C?ULDIV
      0100019AH   PUBLIC    CODE     ---       ?C?ULDIV

      ---         MODULE    ---      ---       ?C?LNEG
      0100022CH   PUBLIC    CODE     ---       ?C?LNEG

      ---         MODULE    ---      ---       ?C?LSTXDATA
      0100023AH   PUBLIC    CODE     ---       ?C?LSTXDATA

      ---         MODULE    ---      ---       ?C?LSTKXDATA
      01000246H   PUBLIC    CODE     ---       ?C?LSTKXDATA

      ---         MODULE    ---      ---       ?C?LIMUL
      01000277H   PUBLIC    CODE     ---       ?C?LIMUL

      ---         MODULE    ---      ---       ?C_INIT
      010005ABH   PUBLIC    CODE     ---       ?C_START



*** WARNING L16: UNCALLED FUNCTION, IGNORED FOR OVERLAY PROCESS
    NAME:    GPIOINIT/GPIOINIT

*** WARNING L16: UNCALLED FUNCTION, IGNORED FOR OVERLAY PROCESS
    NAME:    EXTERNALFASTCLOCKCONFIG/FU68XX_OSC

*** WARNING L16: UNCALLED FUNCTION, IGNORED FOR OVERLAY PROCESS
    NAME:    INTERNALFASTCLOCKCONFIG/FU68XX_OSC

*** WARNING L16: UNCALLED FUNCTION, IGNORED FOR OVERLAY PROCESS
    NAME:    SYSTEMFASTCLOCKMCDCONFIG/FU68XX_OSC

*** WARNING L16: UNCALLED FUNCTION, IGNORED FOR OVERLAY PROCESS
    NAME:    SYSTEMFASTCLOCKSPD2CONFIG/FU68XX_OSC

*** WARNING L16: UNCALLED FUNCTION, IGNORED FOR OVERLAY PROCESS
    NAME:    LVDPOWERDOWNDETECTCONFIG/FU68XX_POWER

*** WARNING L16: UNCALLED FUNCTION, IGNORED FOR OVERLAY PROCESS
    NAME:    LVDPOWERDOWNWARNIECONFIG/FU68XX_POWER

*** WARNING L16: UNCALLED FUNCTION, IGNORED FOR OVERLAY PROCESS
    NAME:    _LVRPOWERDOWNRESETCONFIG/FU68XX_POWER

*** WARNING L16: UNCALLED FUNCTION, IGNORED FOR OVERLAY PROCESS
    NAME:    _LVWPOWERDOWNWARNCONFIG/FU68XX_POWER

Program Size: data=16.1 xdata=60 const=0 code=2425
LX51 RUN COMPLETE.  9 WARNING(S),  0 ERROR(S)
